:020000040000FA
:10000000809B01202D220000A95E00005D220000DF
:100010005D2200005D2200005D2200005D220000E4
:10002000000000000000000000000000352000007B
:100030005D22000000000000DD1F0000855E000062
:10004000ED210000ED210000ED210000ED21000078
:10005000ED210000ED210000ED210000ED21000068
:10006000ED210000ED210000ED210000ED21000058
:10007000ED210000ED210000ED210000ED21000048
:10008000ED210000ED210000ED210000ED21000038
:10009000ED210000ED210000ED210000ED21000028
:1000A000ED210000ED210000ED210000ED21000018
:1000B000ED210000ED210000ED210000ED21000008
:1000C000ED210000ED210000ED210000ED210000F8
:1000D000ED210000ED210000ED210000ED210000E8
:1000E000ED210000ED210000ED210000ED210000D8
:1000F000ED210000ED210000ED210000ED210000C8
:10010000ED210000ED210000ED210000ED210000B7
:10011000ED210000ED210000ED210000ED210000A7
:10012000ED210000ED210000ED210000ED21000097
:10013000ED210000ED210000ED210000ED21000087
:10014000ED21000053B94AB9002908BF00281CBF9F
:100150004FF0FF314FF0FF3000F070B9ADF1080CF7
:100160006DE904CE00F006F8DDF804E0DDE90223D5
:1001700004B070472DE9F04F099E04468946002BD4
:1001800040F083808A42154645D9B2FA82F24AB1DC
:10019000C2F1200701FA02F39540944020FA07F7D4
:1001A00047EA03094FEA154E230C1FFA85F8B9FBFD
:1001B000FEFC0EFB1C990CFB08F143EA0943994233
:1001C0000AD9EB182CBF01200020994202D900283F
:1001D00000F01D810CF1FF3C591AA3B2B1FBFEF0F7
:1001E0000EFB101100FB08F843EA0144A04505D9B5
:1001F0002C1902D2A04500F20E810138A4EB0804AC
:1002000040EA0C4000271EB1D4400023C6E9004359
:100210003946BDE8F08F002A51D0B2FA82F2002AA6
:1002200040F0AF80491B4FEA154E1FFA85F80127B1
:10023000230CB1FBFEFC0EFB1C1108FB0CF043EA87
:10024000014398420AD9EB182CBF012100219842A2
:1002500002D9002900F0D7800CF1FF3C191AA3B293
:10026000B1FBFEF00EFB101108FB00F843EA01445D
:10027000A04505D92C1902D2A04500F2C180013851
:10028000A4EB080440EA0C40BDE78B4208D9002EDD
:1002900074D00027C6E9000138463946BDE8F08F22
:1002A000B3FA83F767B98B42C0F0A480824240F270
:1002B000A1803846002EABD0C6E90049A8E7FFDE92
:1002C000C7F12005BB4002FA07FC01FA07F4EA4037
:1002D00020FA05F8E94000FA07FE1A4348EA040448
:1002E0004FEA1248200C1FFA82F9B1FBF8FA08FB1A
:1002F0001A110AFB09FB40EA01418B450AD9511842
:100300002CBF012300238B4502D9002B00F08880ED
:100310000AF1FF3AA1EB0B01A4B2B1FBF8F008FB24
:10032000101100FB09F944EA0141894504D951182B
:1003300001D289457BD8013840EA0A40A1EB090186
:10034000A0FB0C89494544464B4602D306D1C6451D
:1003500004D20138B8EB0C0469EB0203002E5DD027
:10036000BEEB040261EB030101FA05F522FA07F383
:10037000F94000271D43C6E9005149E7374630469A
:1003800046E7C2F12000954001FA02F721FA00F396
:100390004FEA154E24FA00F11FFA85F894403943CC
:1003A000B3FBFEF00F0C0EFB103300FB08FC47EA1A
:1003B00003439C4507D9EB182CBF012700279C4518
:1003C00000D98FB30138A3EB0C0389B2B3FBFEF75E
:1003D0000EFB173307FB08FC41EA03418C4504D9A7
:1003E000691801D28C4525D8013FA1EB0C0147EAE1
:1003F00000471DE7841A61EB03030120994659E782
:1004000002382C443CE7ACF1020C2B4426E7ACF15B
:10041000020C2B44E0E602382C44EFE63746F7E6C0
:10042000AAF1020A114475E702382B44CBE70238DF
:10043000114481E7023F2944D7E700BF704700BF5E
:100440007FB5314B314A3248C3F800264921C3F801
:100450000426C3F80826C3F80C26C3F81026C3F8F0
:100460001426C3F81826C3F81C2605F0DFF900F09F
:100470007DF8284800F05EF828B9264A452126482C
:1004800005F0D4F9FEE701A800F0BAFC234B1B6885
:10049000834204D04521224805F0C8F9FEE7039ABB
:1004A0004921204805F0C2F949211F4805F0BEF94D
:1004B0004FF48031002002F077FE20B145211B4827
:1004C00005F0B4F9FEE769469DF8080000F03EF833
:1004D000009B039C1C44019B1D8966194FF0200260
:1004E000EFF3118382F31188BFF36F8F05F0CCFC1B
:1004F00000F028FF635983F3088873689847452103
:100500000B4805F093F9FEE7008001503546526E26
:10051000F48500000D860000208600005C47012065
:100520003F8600006286000091860000B6860000CB
:10053000E986000010B5044C236813B903F09AFF54
:100540002060206810BD00BF5847012008B540B1A9
:10055000024600230448452105F068F96FF01500B4
:1005600008BD0860FCE700BF0C8700004FF4C051D5
:10057000014803F081BA00BF3C5601202DE9F04F3D
:10058000774FF9B038A89246DDE984461D46DDF87C
:1005900018B2D7F8008007F01CFB002138A803F040
:1005A0007BFBB94634B1002E04DD3246214638A823
:1005B00007F013FB0026BAF80A30BAF808401C44CA
:1005C000DAF80C301C44B44248D80DA938A807F01A
:1005D00041FBBBF1000F04D020220DA9584605F0C5
:1005E0008FFC00232A46009351464FF6FF7307A85D
:1005F00004F061FE0346002840F0AC8006464FF050
:10060000FF34584F0DF1160305AA06A907A804F0F8
:100610009EFE031EC0F29E8040F09180BDF816A0A1
:10062000BAF1100F2FD1BDF81460202E40F0908049
:10063000334638AA0699284605F010FB03460028E1
:1006400040F08880324638A90DA804F0F9FE034630
:10065000454A126882427DD10126D3E7839BA71BBE
:100660009F4228BF1F46829A3B463146284605F0E6
:10067000F5FA034600286DD13A46829938A807F06A
:10068000ACFA3E449FE7BAF1010F37D1BDF8143000
:10069000202B5DD838AA0699284605F0DFFA0346D4
:1006A000002857D19DF814A0BAF1200F03D94FF0BC
:1006B000FF331C46A6E73A682C4C0292029A9342FA
:1006C000F5DA1DA8039307F084FA00211DA803F0B2
:1006D000E3FA62681DA8126854F8081B07F07DFA57
:1006E00015A91DA807F0B6FA524638A915A805F0B5
:1006F000F7FB039B0028DCD00133DFE7BAF1200FC2
:1007000080D1002C18DB3B68A34215DDBDF8143006
:10071000B3F5807F1CD138AA0699284605F09EFAC9
:100720000346B8B9E4B20094BDF8143038AA514673
:100730000DA800F01DF880464FF0FF3462E76EB15F
:10074000094B1B68434501D0D9F80080434601E0BE
:100750004FF0FF33184679B0BDE8F08F0123F9E779
:1007600000450120388200005C4701203C820000E7
:100770002DE9F04F17460022ADF54B7D1E466A4B22
:100780008046894627A811469DF850A31D6807F0AA
:10079000DCF9664B8AAA53F83A4003EBCA035B685C
:1007A00002941B6802A81C442146302305F0CFFEAA
:1007B00068BB029B8A9A13449C4228D129AA2146ED
:1007C00002A805F0D8FE10BB0DF1B00B5A46214629
:1007D00002A805F0D0FE8246C8B929A806F0B7FAEB
:1007E000029B28909C4212D1CDE900AB5346524661
:1007F00029A927A807F065F948B927A803F0EAF95D
:1008000028B929A806F0A3FA864228900AD027A87A
:1008100007F0A6F927A807F0A3F928460DF54B7DA8
:10082000BDE8F08FB6F5807F02D04FF0FF35F1E7DD
:10083000B9F1200FF9D18AAA394627A803F0EEF9B9
:1008400005460028F1D19DF82733BC2BEDD152AFDE
:10085000DF263C4603900CA807F0BBF900210CA84A
:1008600003F01AFA20220DF207310CA807F0B5F9AF
:10087000042203A90CA807F0B0F904A90CA807F0FA
:10088000E9F91F2ED4BFB1464FF020099DF80F3073
:10089000384601334A4604A9A6EB09068DF80F3005
:1008A00005F02EFB002E4F44D5DC20462246DF23E8
:1008B0008AAE117816F8017B013B81EA070102F844
:1008C000011BF6D1237803F07F03237010F8016B2E
:1008D000002EAAD10135BE2DF8D194F8BE30012BDF
:1008E000A3D10CA807F075F931460CA803F0D4F990
:1008F00008220F490CA807F070F9414620220CA8E5
:1009000007F06BF920220DF207210CA807F065F91A
:1009100004A90CA807F09EF920220DF2073104A8C3
:1009200004F08EFD054682E7004501203C82000070
:10093000328700002DE9F041032386B000250F46E1
:100940006E46DFF87080ADF800508DF8003001A9D8
:1009500016F8010B00F086FF0446D8B90198102361
:10096000816802AA103905F079F9044628B1019886
:1009700005F073F90EE00125E9E71022414602A8CF
:1009800005F0AEFA50B1019805F067F9002DF2D0EC
:100990004FF0FF34204606B0BDE8F081019805F025
:1009A0000FFD0423A0F108013A46019805F056F91D
:1009B0000446DCE7308400002DE9F041374B88B075
:1009C000804600200D461C6804F06CFC06A9C0B2ED
:1009D00000F048FF002855D1294604F063FC2C2480
:1009E00007A9C0B204FB058400F03CFF002834D006
:1009F0002C266E4308EB0607396911F0100137D138
:100A00004FF480730193264B22460093CDE90311E6
:100A10000291069B0846FFF7B1FD0446214B58F8AA
:100A2000062006989A420CD13A89FB68D1438B4242
:100A300007D813448268934203D21B4B1B68A3421E
:100A40001DD045B38268002105F04EF9174A4521B3
:100A5000174804F0EBFE012411E0079805F073F944
:100A60000646079805F0F9F8631EE21C93420DD183
:100A7000002DF0D00699404604F0E2FD2C46069881
:100A800005F0EBF8204608B0BDE8F08113F8011F2F
:100A9000B142EBD0ACE7074AD9E700BF00450120DF
:100AA0003C7201203DB8F3965C4701206987000045
:100AB0007B8700007387000073B50D460021044654
:100AC0002846CDE9001104F07AFD30B3164E2268B5
:100AD000B24203D101AA204604F0E9FCE36AB34222
:100AE00004D16A460121204604F0E1FCDDE9003230
:100AF000934288BF0193019BAB60019A294620462F
:100B000000F020FB094B1A68002A03DD5721084832
:100B100004F08CFE002002B070BD05F10801FFF763
:100B200009FFAB680193E8E73DB8F396C04F012099
:100B30003A8700002DE9F84F894692469B460026E9
:100B40001A4F1B4C1B4D0B9B9E4201D3002010E003
:100B50000B9B164AA3EB0608B8F5806F28BF4FF42D
:100B6000806806EB0B014346484605F077F810B164
:100B70000120BDE8F88F0A9943463A46711850465D
:100B800005F089F80028F3D1C4F800564644C4F8AB
:100B90000456C4F80856C4F80C56C4F81056C4F8E5
:100BA0001456C4F81856C4F81C56CCE73C6E012005
:100BB000008001503546526E2DE9F043884B0446C3
:100BC000602285B00F4600211E6805F0C3F90021A0
:100BD000844B08466362844B236504F063FB04F195
:100BE0002001C0B200F03EFE0121002004F05AFBBB
:100BF00004F14C01C0B200F035FE0546204604F079
:100C0000B6FC024630B180225721784804F00EFE2F
:100C100001238CE00146204604F091FC804618B187
:100C2000002257217248F1E7204600F0A3F900287E
:100C3000EED0684604F0BAFC6946204604F054FD44
:100C400018B1424657216B48E0E7684604F0B7FC0C
:100C500080F001016A46C9B2204604F070FC0246E9
:100C60000028DDD1684604F0AAFC804660BB6946D6
:100C70002046FFF721FF9DF8073084F85830033BEA
:100C8000012B06D8404604F07DFD10B1FF2384F807
:100C900058309DF80730023B022B0BD8002004F09F
:100CA0005FFD38B1FF2384F858304521524804F0E5
:100CB000BDFDFEE794F85830FF2BF6D06A460021C0
:100CC000204604F03CFCA3E79DF80790B9F1010F22
:100CD00022D1104602F0EEFA831E022B80460DD878
:100CE00049462046FFF768FE444B1B68984205D0F2
:100CF00001280CBF4FF001084FF0050884F8588018
:100D000094F858308DF80730013B042B26D8DFE8E3
:100D100003F02B111111340001212046FFF74CFE86
:100D2000364B1B68984214BF05239DF8073084F8A2
:100D30005830E5E769462046FFF7BEFE94F8583084
:100D40000546DA1E012A0DD8002004F01BFD0546D9
:100D500020B9002004F004FD054628B1FF2384F8E3
:100D6000583001E0022BF4D094F85830FF2B08D112
:100D70004521214804F05AFDFEE7002004F002FD61
:100D8000EAE7012B06D06A460021204604F0D7FB93
:100D90000546B8B900212046FFF70EFE0646DFF8EB
:100DA0005C80D8F8003083420CD1102200216846C4
:100DB00005F0D0F8236AD8F800605A783A715B6879
:100DC0003C60BB60E06C04F048FF206A04F045FF23
:100DD000002D14BF2846304605B0BDE8F08300BFA3
:100DE00000450120C0470120C04B0120A38700001F
:100DF000E5870000118800003B8800005C47012067
:100E000008B501460148FFF7D7FE08BD604701203D
:100E100073B516461D4633B3436A5C686B79012B84
:100E200015D101BB1F4B2A681B689A4298BF00244A
:100E3000002004F037FA01A9C0B200F013FDF0B1B0
:100E40000124019804F009FF204602B070BD022B76
:100E500009D12B68012B08D9124A1268934202D893
:100E6000B1FA81F149090024E2E7FCD10029DFD081
:100E70000129F8D12979023918BF0121F3E7214668
:100E800020233246019804F0E9FE04460028D7D119
:100E9000002DD6D03468044BE41A18BF4FF0FF344D
:100EA000CFE700BF044501203DB8F3962DE9F04F90
:100EB000814685B00C4601460020164604F0C7FA6C
:100EC000051E50DB4846E46D04F0CBFA5FFA84F867
:100ED0004FF0000A4FF0010B4FF0FF346F1E08FB7C
:100EE00007079DB9BAF1010F03DD4521204804F041
:100EF0009DFC631C06D07F2C2ADC40F201130134D8
:100F00003460B380284605B0BDE8F08F6B1E0093B7
:100F10000DF10F0201233946484604F09FFE031EDF
:100F2000019322DB01220DF10F01484605F05AFA28
:100F3000019B40B19B4501D00AF1010AA7EB0807CC
:100F4000009D9B46CDE7B4F1FF3F08BF2C46F5E777
:100F50000223803C7371631004F0010401330134F7
:100F600033603471CEE70725CCE70125CAE700BF1F
:100F7000DA88000070B5826A456DAA4208D06B1C01
:100F8000934205D05721134804F050FC002070BD57
:100F9000802A1BD957211048F6E7446A066DD9000C
:100FA0000C44314464684968A14202D057210B487F
:100FB000EAE70133AB42F0D19A4205D9426A02EB2B
:100FC000C3035B689C42F1D10120E0E700231C468B
:100FD000F0E700BF478800007F880000AE8800006F
:100FE00000B589B004A9032005F02FFA9DF8102060
:100FF000012A41D0254B2649032A18BF0B469DF8EC
:101000001320492102929DF81220224801929DF856
:1010100011200092204A04F009FC06A9072005F0DF
:1010200014FA9DF81820012A28D0184B1849032AD1
:1010300018BF0B469DF81B20492102929DF81A20EB
:10104000144801929DF819200092144A04F0EEFB16
:101050009DF81030012B13D19DF81230032B0FD1C6
:101060009DF81830012B0BD00D48492104F0DEFB10
:10107000022009B05DF804FB0A4BC0E7094BD9E731
:101080000948492104F0D2FB0020F2E73189000031
:1010900037890000498900003B8900008A890000E7
:1010A0009A8900002C890000B989000070B51446A7
:1010B0004A680D461D4902F0FF228A4286B0064664
:1010C0002FD12A68012A2CD104A9184605F0BDF9B0
:1010D0009DF81020012A26D0154B1649032A18BF67
:1010E0000B469DF81320492102929DF812201248C8
:1010F00001929DF811200092104A04F097FB9DF890
:101100001030032B0DD12146304604F099FA2046C9
:1011100005F08BF9A968204604F0BAF9204602F0E0
:101120006BF806B070BD064BDBE700BF00010004A2
:101130003189000037890000498900008A89000050
:101140002C890000436A2DE9F04F0C465E68054685
:10115000012300218BB03144914203F1010011D3EE
:10116000754F20463B6004F02AFABA46C8B1E86DD4
:1011700004F068F90022AB6A013B3244904203D983
:10118000013BFAE70346E6E7DAF800209A4208D383
:1011900057216A4804F04AFB0123E3710BB0BDE814
:1011A000F08F08A9032000F05DFB09A9072000F0DB
:1011B00059FB0723099A21462846FFF777FF6379F1
:1011C000012B08D1DAF80070DFF874B1DAF80030DA
:1011D000A7B90123236002230127DFF8649163711B
:1011E0000693DAF80030DDF820809F424BD9404664
:1011F00004F033FD099804F030FDCFE72268013395
:101200009B1A9F423DD86B6A012A196853F8370030
:1012100003EBC70353F8083CDDF82080A3EB010380
:10122000A0EB0109039312D1E268099B022A0AD0BC
:1012300041462846049304F003FA224641462846D4
:1012400004F033FA049B1946284604F0F9F93246B3
:101250004946404604F0F2F9039B42464146CDE937
:1012600000962846FFF766FC2146284604F0B4F9AC
:1012700023680133236020B1DBF800300133CBF861
:101280000030013FA2E723689F4252D36A6AFB0005
:1012900052F83710083B05911168DDF824B004912D
:1012A000296DC8580968411A0391217901293ED155
:1012B000D358049A40469B1A19463246079304F0C5
:1012C000BDF9079B424600935946039B0196284669
:1012D000FFF730FC2146284604F07EF9069B237177
:1012E00020B1D9F800300133C9F8003032460399F3
:1012F000584604F0A3F9039B414600930196DDE9AB
:10130000042328469B1A5A46FFF714FC2146284618
:1013100004F062F92368013323604FF00103237165
:1013200038B1D9F800300133C9F8003001E00229A2
:10133000DCD0013755E700BF04450120FD880000DF
:10134000C04F01200122124B12491A604FF0FF33A7
:10135000C1F84833C1F8083301F5805104310A60FF
:1013600000210D4AC2F84833C2F80833A2F55042B2
:10137000C2F80015C2F8083302F58052C2F8001511
:10138000C2F808334FF05022C2F80833704700BF4C
:101390000440015000400150005001500B680133DF
:1013A0000B60014B1B68184708450120014B186072
:1013B000704700BF08450120002307B5024601938E
:1013C00003480B4601A900F0E3F803B05DF804FB05
:1013D0009D1300002DE9F84FB0F81890044619F05D
:1013E00008080DD001290CBF49F0100949F0200967
:1013F000A0F8189082F31188BFF36F8FBDE8F88FC3
:1014000009F00709022907D1204604F01CFA002838
:10141000F0D00128238B4AD16769238B002F15DA7E
:101420002568C4E9008823F0070343F00103238300
:101430000026238B03F0070ACA4502D0A1680029C1
:1014400056D10DB9002E6DD0002152E003F00701F6
:10145000481F01281CD823F00703062925689BB2E2
:10146000C4E900880AD13DB12846618B006801318A
:1014700089B20028FAD1618343F002032383204616
:1014800004F0E1F90028D3D0238B43F02003CEE70A
:1014900004290AD123F0070399B22183204604F0DE
:1014A000D2F910B141F0200121830025C0E70328C3
:1014B00009D1216923F007030E6843F006030025D4
:1014C00023832F46B5E7042806D1216923F00703BB
:1014D0004E6843F00403F2E7052806D1216923F0A2
:1014E00007038E6843F00503E9E700252E46E8E789
:1014F000012143F00803238382F31188BFF36F8F28
:10150000F9B985BB16B121492046B0474FF02003F9
:10151000EFF3118283F31188BFF36F8F238B23F0D6
:1015200008032383238BD90627D5012123F0100339
:101530002383B4F8189009F0070900297FF462AFFB
:1015400058E7A1680029DCD0D1F80090D1F804B0A8
:101550003B4652462046D847B9F1000FD1D0494604
:10156000D9F80090F2E7D5F8009029463B4652465C
:10157000204604F084F94D46C3E713F020011EBF56
:1015800023F0200323830221D3E700BFAB580000E0
:101590002DE9F04F00258046894693461F464FF0BF
:1015A000FF36AA462C468DB00B959BF8000018B963
:1015B0000B980DB0BDE8F08F54B9252800F00D81CF
:1015C0004946C0470B9A01320B920BF1010BECE735
:1015D000642861D020D839280ED8312859D22D2836
:1015E00000F00181302843D025280BD14946C0475F
:1015F0000B9A01320B927DE0582800F0CE806328D0
:1016000000F0E38049462520C0470B9A4946013245
:101610000B929BF80000EAE7702800F082800DD85A
:10162000692839D06C2803D16C2D1DD14C25CCE70D
:101630006828E7D1682D17D14825C6E775282BD033
:101640000DD87328DED157F8044B2346194613F8FA
:10165000010B002840F0B1800A1BB21A77E078280D
:1016600000F09B807A28CDD1002DCBD10546ACE788
:10167000002E04DABAF1000F00F0B88000260A222A
:101680003038BAF1000F02FB060608BF4FF0020A1D
:101690009BE726EAE676F2E77A2D06D13C4654F837
:1016A000042BD317752828D10FE06C2DF6D04C2DC4
:1016B00005D1FC1D24F00704F4E80223F2E77528A5
:1016C00007F104043A6817D10023BAF1030118BFE7
:1016D0000121BAF1010F0CBF30202020CDE901100B
:1016E0000A210BAFCDE9036700914046494604F05B
:1016F00030FA2746002468E7D317002A73F1000167
:10170000E3DA49462D20CDE90623C047DDE906236B
:101710000B99524201F101010B9163EB4303013E2E
:10172000D3E757F8044B334B334A002C18BF13460A
:1017300013F8010B494606930993C0470B99069B82
:1017400001310B9119780029F2D174B9721FBAF1E5
:10175000030FCFD11446002CCCDD49462020C047D2
:101760000B9A013C01320B92F5E722460B46023EF2
:10177000BAF1030118BF0121BAF1010F0CBF3020EB
:101780002020CDE9011010210BAC0091CDE90364BC
:101790004946404604F0DDF9ACE76C2D03D157F81B
:1017A000042B0023E4E74C2DF9D1FC1D24F00703A2
:1017B0001F465B6857F8082BDAE749460693C0478F
:1017C0000B99069B01310B9140E7494657F8040BF2
:1017D000C0470B9B01330B938CE72546A2464FF085
:1017E000FF360124F1E64FF0030AEEE64FF0010A5E
:1017F000EBE600BFDE8A0000E48A00004FF0200222
:10180000EFF3118382F31188BFF36F8F0121044A34
:10181000C2F8401583F31188BFF36F8F0020704723
:101820000090035020B1034B800143F0010318479F
:10183000704700BF30820000084B30B51D68084B70
:10184000196800239D4202DC0022104630BD1C01B5
:101850000A190C5D8442F8D00133F3E7E8820000F6
:101860000C450120084B10B51B680C462BB1FFF747
:10187000E3FF28B12060002010BD6FF00C00FBE7F3
:101880006FF00100F8E700BF0C45012030B589B0CA
:101890000C4615460190FFF7CFFFB8B143682268A8
:1018A00002938368C068CDE9033500230593CDE931
:1018B000062304F0B2F960B101AA074904F0CFFB96
:1018C000079808B9059B236009B030BD6FF015007B
:1018D000FAE76FF01200F7E71F5C000008B5044656
:1018E0004FF02002EFF3118382F31188BFF36F8F63
:1018F00004F0CAFA204600F07FFE034803F096FF8A
:1019000000F008FCFCE700BFF18A00000A2838B5A7
:101910000446064D03D10D21286804F01DFA2868FD
:10192000E1B204F019FA204638BD00BFC44F0120CF
:1019300010B5074802F09EFD064C074B1860204684
:1019400000F0E0FF2046FFF731FD002010BD00BF92
:101950001A8B00000D190000C44F012070B5054618
:101960000C240D480E462B1A9A100C4B4021534361
:10197000DBB25C4304F14003184404F0F9F9011EA2
:1019800004DB074B23445B68984700212846334615
:10199000BDE87040184700BFD84F0120B76DDBB6D7
:1019A000008300002DE9F0410F4C104D031B9B10EC
:1019B0005D43EBB20C255D43074605F140000E4642
:1019C0002044402104F0EDF9011E08DB084B2C44B3
:1019D000C4E90E36074B5B59BDE8F041184738465D
:1019E0003346BDE8F0411847D84F0120B76DDBB64C
:1019F0000B5E00000083000070B500220121044648
:101A0000052000F045FB052000F024FB0F4801F005
:101A10006FFD0F4B984215D104F03CFDE6680D496F
:101A2000304603F05FFF00280BDB01253564E468D6
:101A3000084904F11C0003F055FF002801DB0020D9
:101A4000E56470BD6FF00400FBE700BFF11A000011
:101A50000000AD0B1883000001460C2300224B430D
:101A6000084870B5C4184033D4E90E561844A26330
:101A700004F0B5F92DB132462B46BDE8704002485E
:101A8000184770BDD84F01200846012008B54FF017
:101A90002003EFF3118183F31188BFF36F8F124A94
:101AA000136843F0020013F0010310600CD04FF0F4
:101AB0005022D2F80C34D2F80C2413F0010303D0D6
:101AC0000A4804F08CF9012381F31188BFF36F8F6A
:101AD00023B1BDE808400020FFF7BEBF0120BDE8EC
:101AE000084001F015BD00BF28500120185001200A
:101AF00010B1012804D07047034B1B6C5B0701D168
:101B0000FFF7AABF704700BFD84F0120074BD3E8AB
:101B1000EF2F22F00201C3E8E01F0028F7D1D3071E
:101B200002D4012001F026BD704700BF28500120DB
:101B30002DE9F843012205463849D1E8EF3FC1E8D5
:101B4000E02F0028F9D133B9354936484B60CB60D6
:101B50008A6003F0DAFE6B1E012B30D8012D07D10D
:101B60004FF05023D3F81C3403F00303022B26D08C
:101B700006F0BDF918B92C4B1B78002B46D14FF05D
:101B80002003EFF3118983F31188BFF36F8F0124D2
:101B9000264E274FDFF89C804FF05022D2F81834A1
:101BA000D2F81824D2030CD503F00303022B01D082
:101BB000012D06D124B389F31188BFF36F8FBDE8DF
:101BC000F883C4B1484600F0B3FA4FF05022D2F87F
:101BD0001835DBB2012BDFD131680029DCD00021C0
:101BE000316031680221C2F818152022C7F880211F
:101BF000C8F80030D0E70021212002F0FBFFE4E725
:101C00004FF050230222C3F80423D8E74FF05023AB
:101C100002220446C3F808238146B9E72C5001206C
:101C2000C84F0120F44F01207E7301200451005061
:101C300000E100E008500050044A1368C91A21F07E
:101C40007F400344136003F0F9B800BF3C5001200B
:101C50002DE9F0474FF48037850000F1500405F17D
:101C60005025A40005F58035A4B204F15024D5F820
:101C70004025DFF86C80DFF86C9021F07F4604F59A
:101C800080348740D8F804A5A2EB0A0222F07F42F4
:101C90002AF07F43012AC5F8403502D1132006F00F
:101CA0002CF90AF10202B31A23F07F434B4528BFF7
:101CB000164600232360236826F07F43C8F8447348
:101CC000C5F84035D8F804359A4507D0F31A023BD9
:101CD00023F07F43B3F5000F3246D3D8BDE8F08739
:101CE0000050015001008000F8B5002427460F4E37
:101CF0000F4B104A1D68184604B1F8BDD2F8041302
:101D0000C903FAD531680029F7D0346031684FF43F
:101D10008031C2F84813D2F84015012425B11F6064
:101D20005A680020A847E3E70560E6E74051015004
:101D3000305001200050015038B500244FF480335A
:101D40004FF400120D4D0121C5F80845C5F80433C4
:101D50000B4B1520C3F88021224600F099F915207D
:101D600000F078F90123074A02201360064A2B602D
:101D70001360FFF7DDFE204638BD00BF0050015064
:101D800000E100E00850015038500120134BB0F141
:101D9000FF3F08BF1846013800281CDD9842A8BF45
:101DA00018460F4BD3F804250E4B1968521A12F43B
:101DB000000F18BF002022F07F4301330A4A03447A
:101DC0000A48106000205060044A934294BFC9182A
:101DD0008918FFF73DBF0020E3E700BFFFFF7F004A
:101DE000005001503C50012030500120391C0000AF
:101DF0004FF02002EFF3118382F31188BFF36F8F4E
:101E0000064AD2F80405064A1268801A20F07F407C
:101E100083F31188BFF36F8F704700BF00500150EC
:101E20003C500120014803F0CFB800BF24830000DC
:101E300008B5B0B14368042B0DD100220368D3E884
:101E4000EF1F012903D1C3E8E02F0028F7D107488D
:101E500008BF104608BD3BB1006802F0C9FC002075
:101E6000F8E76FF4E040F5E70148F3E7E98FFFFF9B
:101E7000EA8FFFFF10B5044618B90D4B0D485B689B
:101E80009847616808290DD031F004030AD011F099
:101E9000020108D02146084802F008FC0023236014
:101EA0000023636010BD1422206804F053F8F7E7A4
:101EB000A84501204B8B00004050012010B504467E
:101EC00018B9164B16485B6898476368042B23D0F3
:101ED000082B21D0CBB92368BBB94FF0FF324FF0AC
:101EE000FF3321460F4802F0AFFB08B923681BB946
:101EF0000A4B0D485B68984714220021206804F0C3
:101F000029F8636843F002036360206805F041FF2D
:101F1000636843F00103636010BD00BFA845012062
:101F20004B8B000040500120718B000008B5D8B1E8
:101F30004368042B0CD101220368D3E8EF1F00296A
:101F400003D1C3E8E02F0028F7D10BD1002008BD52
:101F50006BB100684FF0FF324FF0FF3302F0D0FB5F
:101F60000028F3D00348F2E76FF4E040EFE70248BF
:101F7000EDE700BFE98FFFFFEA8FFFFF08B50649D5
:101F800040231422054805F0E9FEBDE80840044955
:101F9000044803F06BB800BF5C50012040500120A2
:101FA0003C8300002C830000094A0A4993680968B1
:101FB0009867D96708494B6843F080534B6000230A
:101FC00083F31188BFF36F8F9368D86F704700BF9A
:101FD000F05501205485000000ED00E013498A68A7
:101FE0004FF038001044EFF3098C80E8F01F2020F8
:101FF00080F31188BFF36F8F0D4F4FF000664A6A70
:102000008A603E60906F0023936780F3118802F12D
:10201000380090E8F01F8CF3098802F1000004B545
:1020200003F03AFFBDE8044070470000F05501207E
:1020300004ED00E01EF0040F0CBFEFF30880EFF397
:102040000980816911F8021C0229FFD001B503F053
:1020500027FF01BD43B2002B08DB012200F01F0067
:1020600002FA00F0024A5B0942F82300704700BF01
:1020700000E100E0054B420953F82220012300F063
:102080001F0003FA00F01040704700BF00E100E0BD
:1020900043B2002B01F10101A8BF03F160434FEAF5
:1020A0004111B8BF054BC9B2ABBF03F5614300F0A6
:1020B0000F0083F800131954704700BF14ED00E0BF
:1020C00080B51D4604460F46164600F0D5FA00239B
:1020D00083F30B880B4B31462A463846A3F520562E
:1020E000202586F30B8883F3098863B64FF000033D
:1020F00083F31188BFF36F8FA04785F31188BFF377
:102100006F8FFEE7809B0120014910220A60704713
:1021100010ED00E072B6404080F31188BFF36F8F7E
:10212000BFF34F8F30BF62B6BFF36F8F704700BFF2
:1021300072B6494081F3118820BF80F3118862B6DE
:10214000704700BF37B505460C46C9B18B681048CB
:102150000093D1E90023452103F068FB6369452121
:102160000093D4E903230B4803F060FBE2694521A7
:10217000094803F05BFBA2694521084803F056FBC0
:102180002146284603B0BDE8304002F09BB900BFAD
:102190009E8B0000D28B0000068C00001A8C000081
:1021A00030BFFFF7FDBF00BF0E4A08B50E4B22F04F
:1021B0007F029A60BFF34F8FBFF36F8FD3F88820F1
:1021C00022F47002C3F88820EFF3148323F0040391
:1021D00083F3148802F0C4F902F044FD00F01EFA03
:1021E00002F0E0F90000000000ED00E001B572B679
:1021F0000B4A106A00281EBF0021116205F0ACFDD9
:1022000062B6EFF30580A0F110004FEAC000054967
:10221000014409C99847BDE8014003490847000047
:10222000F0550120B47F0000F525000003F0F0FC1C
:10223000202080F3118808484FF40061401880F393
:102240000988EFF314800221084380F31488BFF358
:102250006F8FFFF7A9FF0000809B0120EFF308803C
:10226000EFF3098101B5724600F008F901BD00BF26
:1022700070B5224C06460D462148452103F0D6FA9A
:10228000A26AD00603D545211E4803F0CFFAA36AFF
:10229000190703D545211C4803F0C8FA174CA36A57
:1022A0009A0710D54521194803F0C0FA626BA36A5A
:1022B0001B0608D54521164803F0B8FA1EB1A36ADB
:1022C00023F08003A3620D4CA26AD00703D54521F9
:1022D000104803F0ABFAA36A990603D545210E48CE
:1022E00003F0A4FA0020054B9A6AD20658BF9A6AF6
:1022F0009A6A42F0FF029A62287070BD00ED00E019
:10230000F38C00000E8D0000468D00005E8D0000F5
:102310007B8D0000968D0000BA8D000070B5234CB7
:1023200006460D462248452103F080FAA26AD104F0
:1023300003D545211F4803F079FAA36A1A0503D58E
:1023400045211D4803F072FA184CA36A9B0510D56D
:102350001A48452103F06AFAA26BA36A180408D54B
:102360004521174803F062FA1EB1A36A23F4004323
:10237000A3620E4CA36A590503D54521114803F009
:1023800055FAA36ADA050BD545210F4803F04EFA3A
:102390000020064A936A43F47F439362287070BD1D
:1023A000A36A9B04F4D545210848EFE700ED00E05F
:1023B0004D8C0000688C0000468D00007E8C000073
:1023C0009C8C0000B68C0000D68C0000BA8D0000FA
:1023D00038B5214C4521214803F028FAA26A95011D
:1023E00003D545211E4803F021FAA36ADC0103D579
:1023F00045211C4803F01AFA174DAC6A14F48014F6
:1024000004D04521184803F011FA0224AB6A1803DE
:1024100003D54521154803F009FA0F4DAA6A510367
:1024200003D54521124803F001FAAB6A9A0303D59C
:102430004521104803F0FAF9074DAB6ADB0303D5D9
:1024400045210D4803F0F2F9AB6A20466FEA0343D9
:102450006FEA1343AB6238BD00ED00E0EE8D000083
:102460000B8E0000238E0000428E0000718E000053
:10247000948E0000BE8E0000DD8E00002DE9F0433A
:102480004A4B8BB0D3F804900025C9F3080885F3B4
:102490001188BFF36F8F02F07F43B3F17F4F07D1F5
:1024A00002F00C03082B05D14521414803F0BEF989
:1024B0002F4604E012074EBF0F46074601250022B3
:1024C000A8F103068DF807201446092E5BD8DFE833
:1024D00006F0054F53335A5A5A5A5A574521354830
:1024E00003F0A4F9314B8DF80740DC6A14F00204C4
:1024F00005D04521304803F099F900241FE0DB6A3C
:102500005B001CD545212D4803F090F92C4B1B781E
:102510002BB101200DF10701FFF7AAFE0EE0294BB8
:102520001B782BB101200DF10701FFF7F7FE05E045
:10253000254B1B889BB213B1FFF74AFF04469DF859
:10254000073093B92022394602A803F0D9FC099B31
:1025500035B3C3F3080222B96FEA53236FEA43236A
:10256000099302A92046FFF7EDFD0BB0BDE8F0830B
:102570000DF107010020CFE70DF107010020D4E79E
:1025800045211248B7E7124919F4F87F114AA8F11A
:10259000100308BF0A461048452103F047F9ACE78D
:1025A00023F4FF7323F00103DAE700BF00ED00E03E
:1025B0003B8F00006B8F0000878F0000AD8F000005
:1025C00028ED00E029ED00E02AED00E0D18F0000C9
:1025D0000D8F0000228F00000C900000044B5A6900
:1025E00042F010025A615A6942F480625A6170479F
:1025F00000ED00E0704700BFBFF34F8F0549064B69
:10260000CA6802F4E0621343CB60BFF34F8F00BF90
:10261000FDE700BF00ED00E00400FA0500232021E3
:102620000348C2180133412B82F80013F9D17047D7
:1026300000E100E008B50E4B9B68834207D1EFF341
:10264000058393B10B4A536843F08053536002F003
:10265000C3F94FF02003EFF3118083F31188BFF328
:102660006F8FBDE8084005F09BBB02F0DBFA00BFAE
:10267000F055012000ED00E0024B034A0121034820
:1026800000F036B90000042000450120508300000E
:1026900010B50B680C7A23F01F0204F01F031A43D5
:1026A000CB68640923F01F03044943EA440343F061
:1026B00001038860CA600B6110BD00BF90ED00E0AF
:1026C00030B54B6885B00C689DF808200D890094E2
:1026D000498924F01F04013B234465F3040261F39C
:1026E000471223F01F030F288DF808200393044698
:1026F00009D902464521064803F098F86FF0150401
:10270000204605B030BD6946FFF7C2FFF8E700BFBD
:10271000289000002DE9F04F8946144606464FF0F8
:102720000008534D85B0C84523DA7768002F42D0A2
:102730001F2F17D9FB0615D1D6F800A01AF01F0FCE
:1027400010D1504603F0B7FB834607EB0A0001386F
:1027500003F0B1FB834510D06FF0150B5A464521AD
:10276000444802E042464521434803F05FF86FF0D9
:102770001504204605B0BDE8F08F1BF1160FEDD013
:10278000631E5B45EADBC5F808B0E968C5F808B028
:102790002F6921F01F01D6E900321A44994247F00F
:1027A0001F0702F1FF3A1CD1574508D131465FFAA5
:1027B0008BF0FFF785FF08F101080C36B3E73146CF
:1027C000C5F808B0EB6822F01F0203F01F031A439C
:1027D000EA60E0B2FFF774FF10F1160FC7D0441C97
:1027E000E9E7013B5745E0B223F01F03C5F808B005
:1027F00006D12A69314602F01F0213432B61E9E733
:10280000296901F01F010B432B613146FFF758FF87
:1028100010F1160FABD0C5F808B0EA689DF8083083
:10282000013F62F304038DF808302B699DF80820FE
:102830005B0863F347128DF80820D6E90032134491
:10284000009323F01F033B440130A3EB0A0AC4B2F8
:102850002AF01F030F2C039303D922464521074872
:1028600083E720466946FFF713FF0134A3E700BF63
:1028700090ED00E07B900000539000002890000055
:102880000522034B5A60BFF34F8FBFF36F8F704722
:1028900090ED00E0BFF35F8F0022014B5A6070475C
:1028A00090ED00E070B50E4D2E68102E15D8002466
:1028B000FFF7F0FF0B4B0C4A1A63A64205D10B4BF6
:1028C0001E70FFF7DDFF002070BD6968204601EB38
:1028D0000411FFF7DDFE0134EFE74FF0FF30F3E7BF
:1028E0005C83000090ED00E0AAFF44003C730120EF
:1028F00010B5034C2278FFF70DFF207010BD00BF0C
:102900003C730120014B1860704700BF3045012027
:10291000064B00F01F0003EB8000D0F8003223F4D8
:10292000403343EA0141C0F800127047002584504B
:1029300008B5094B1A786AB901210D2019700521D3
:10294000FFF7A6FB0D20FFF785FB4FF00042034B7E
:10295000C3F80423002008BD3D73012000D00050BF
:1029600073B50D46416805F01F04097AB2F5A03F22
:10297000C66844EA41140AD15C4804F01F01803162
:1029800050F82110C80707D56FF0220091E0B2F58A
:10299000005FF16800F08F800121F068A9400143D9
:1029A000F16001217069A940B2F5A03F0CBF084356
:1029B000884370610020B269B3F5C02F0CBF0A4391
:1029C0008A43B2613269B3F5802F0CBF114322EA0A
:1029D0000101474A3161D2F80433DBB200F5A2713C
:1029E00052F82110C1F304218C4269D123FA00F17D
:1029F000C90765D5830003F1A04303F55043D3F81D
:102A0000101521F00101C3F8101501238340C2F80D
:102A10000833C0B200F042FE20460021FFF778FFE5
:102A2000F068E84010F0010043D07069E84010F011
:102A300001024ED0B369EB40DB0745D4336923FA7A
:102A400005F515F0010F14BF012502250DF1070052
:102A500000F046FE274B984238D100209DF8071021
:102A600024028B0003F1A04303F55043D3F8102553
:102A700004F4F85422F4473222F44072C3F81025CB
:102A8000D3F8102514438A0002F1A04202F5514206
:102A900044EA0544C3F8104510601268D3F81025C5
:102AA00042F00102C3F810250123114A8B40C2F8FD
:102AB000043302B070BD0120A84021EA00016FE795
:102AC000013008288AD1A7E70325BFE76FF012007D
:102AD000EFE73369204623FA05F515F0010F0CBF27
:102AE00003210221FFF714FF1046E2E7002584507E
:102AF00000D000500000AD0B284B70B51340B3F56B
:102B0000801F46683BD007D8022B3AD0062B13D043
:102B100093B16FF0150031E0B3F5800F33D004D8D6
:102B20001F488342F5D1072306E01E4883422CD07C
:102B3000B3F5A00FEDD10323D00654BFC2F3401567
:102B4000032582F4807412F4007FC2F34020C4F3A2
:102B5000002406D012F4006F766818D001228A4053
:102B6000B26040EA440040EA0323002001F01F0164
:102B70000D4A43EA8503803142F8213070BD0123BC
:102B8000DAE70423D8E70223D6E70523D4E7520582
:102B900042BF01228A40F260E3E700BF0600F00076
:102BA0000600100002004000002584502DE9F0418D
:102BB0003A4E3568002D4CD001274FF00008384BB5
:102BC000DA68D3E90510014322EA010235491B699D
:102BD0000C695C4022EA040472BB32603368002353
:102BE00001261F463048D0F8042306FA03F11142AB
:102BF00011D09A0002F1A04202F55142116851B180
:102C000003F5A27150F821101760C1F3042106FAF0
:102C100001F112680C430133082BE4D1DCB94DB14A
:102C2000012500261E4CE268D4E90510014322EA82
:102C300001020ABBBDE8F0813A4206D0002108F04B
:102C40001F00FFF765FE22EA070208F101087F0076
:102C5000C2E72C46C3E7124B59680029DFD00E6843
:102C6000124F8A68224002D04B6838469847002E9F
:102C7000D5D031463668F4E715420CD0236906F00A
:102C80001F00F34013F0010F0CBF03210221FFF7D7
:102C90003FFE22EA050201366D00CAE77CD10050F2
:102CA0005C5501200025845000D00050484601208A
:102CB000024B0B6001231360704700BF7855012061
:102CC00000487047CC83000010B503F0F4FB034CC0
:102CD000206003F0EDFB6060002010BD78550120FE
:102CE000F8B50F46144603F0E3FB21460646384686
:102CF00003F0A2F93D46F8B1B7FBF6F306FB1373F8
:102D000023B9B4FBF6F006FB104040B123463A4627
:102D100045210C4802F08AFD6FF015000BE0B4422B
:102D200009D303F0C5FB0646284600F025FDA41B89
:102D30003544F9D12046F8BD23463A46452102489C
:102D4000E8E700BFB9900000DD90000070B50D46C7
:102D50001946284616461C4603F06EF940B9094844
:102D600023462A46452102F061FD6FF0150070BD33
:102D700034B122462946304603F0C2F80020F6E777
:102D80002046F4E7DD900000F8B50E4619463046BF
:102D900017461C4603F050F940B9234632464521F8
:102DA000124802F043FD6FF01500F8BD44EA060535
:102DB00015F0030504D02346324645210C48F0E7C0
:102DC0008CB124F00304A54205EB060006D1094AA4
:102DD000D2F80034DB07FBD50020E6E7795900F094
:102DE000E9FC0435EFE72046DFE700BFDD90000097
:102DF000FF90000000900350F0B54B79012B27D0D5
:102E0000032B22D110268B79032B1ED1CC7924B130
:102E1000012C1AD143681B79BBB10A7912B1022A7D
:102E200013D10E2247F612270B684568BB422D6866
:102E300063D029D8B3F5965F62D014D8B3F5167F66
:102E400060D007D8B3F5967F5FD06FF0220053E0D3
:102E50000026D8E7B3F5966F5AD0B3F5166FF4D1C4
:102E60004FF41D233CE0B3F5615F54D004D8B3F5B3
:102E7000165FEAD1334B33E0B3F5964F4DD0B3F53F
:102E8000E14FE2D1304B2BE0B3F5E13F47D012D810
:102E90004DF6C027BB4245D005D8B3F5164FD4D167
:102EA0004FF41D031CE0B3F5614F3ED0B3F5963FE0
:102EB000CBD1264B14E0B3F5E12F39D008D8B3F5C8
:102EC000613F38D0224FBB42BFD14FF0806307E053
:102ED000B3F5612F32D01F4FBB42B6D14FF08053B4
:102EE000C5F82435C36834432243043303C9C5F805
:102EF0006C2583E803000020F0BD4FF40003EFE7EA
:102F0000154BEDE74FF41C33EAE74FF4A033E7E746
:102F10004FF49E23E4E7114BE2E7114BE0E74FF05B
:102F2000EB73DDE74FF46503DAE74FF46B03D7E7A4
:102F30004FF0E863D4E74FF06C73D1E74FF0706364
:102F4000CEE700BF0050270000C0750000903A0196
:102F500090D0030040420F0000B0130000F03A0090
:102F600000A04E002DE9F04106460F46C56804F06A
:102F7000BEFFB8B9294B1B7883F00103726814684F
:102F800093B14FF02003EFF3118183F31188BFF366
:102F90006F8F304603F0DEF848BB81F31188BFF332
:102FA0006F8FEEE70123E9E74FF06408304603F046
:102FB000D1F878B9012003F06BFAB8F10108F5D126
:102FC0000021212001F016FEEEE781F31188BFF306
:102FD0006F8FF5E74FF02003EFF3118183F3118832
:102FE000BFF36F8F304603F0B5F80028EDD0012312
:102FF000002205F8147FC4F84455C4F84835C4F8D5
:103000002021D4F82001C4F85821D4F85821A36015
:1030100081F31188BFF36F8FBDE8F0817E730120CB
:103020004FF0000C43682DE9F041C5681C680F465D
:10303000C4F800C506462860086801213E4B00F030
:103040001F02914099600321803243F822107A6870
:10305000511C1EBF02F01F01803143F821C0B96826
:10306000C4F80C05481C18BF0020C4F814251EBF66
:1030700001F01F02803243F82200F868421C0CD095
:103080004FF0010C00F01F020CFA02FCC3F808C05C
:103090004FF0030C803243F822C0C4F80805C4F88E
:1030A0001015F16830460431FFF7A6FE804678B966
:1030B00073689B79E3B105F1160000F0D1FA1F4B5C
:1030C000984208D045211E4802F0B0FB6FF004087A
:1030D0004046BDE8F081AB7D43F00043C4F8A03129
:1030E000C4F88C300123AA7D9340164AC2F80435F7
:1030F0000823C4F800357B6801330CD00023C4F8E2
:103100001031D4F8103105F11503C4F8343501231A
:10311000C4F83835236073689B791BB94FF480730A
:10312000C4F8043300231435C4F84455C4F84835B2
:103130000123A360E360CBE7002584500000AD0BC2
:10314000439100000070015030B585B06C460546D3
:10315000084B0FCB84E80F00002201210820FEF766
:1031600097FF0820FEF776FF21462846FFF758FF15
:1031700005B030BD1082000030B585B06C46054604
:10318000084B0FCB84E80F00002201210920FEF735
:103190007FFF0920FEF75EFF21462846FFF740FF2C
:1031A00005B030BD2082000040EA0103C3F30E03E6
:1031B00030B58BB940F21515094CC90BC0F3C730B7
:1031C000994201D1002030BDC218D2B202F5C072BE
:1031D00044F822500133F3E76FF01500F3E700BF26
:1031E00000300050034808B5452102F01FFB0020C5
:1031F000FFF702FA67910000816808B5044A1023BE
:10320000103902F048FD003018BF012008BD00BF92
:103210003084000030B50C46816887B0102302AAC4
:103220001039054602F01AFD002811DB102202A910
:10323000284603F089F868B103232370A9680123A5
:103240000DF107022839284602F008FD00280BDAA4
:1032500001202AE01022164902A802F041FE0028AF
:1032600014BF02230123E8E79DF807300DF10701A1
:1032700003F00F021B09627023710122284603F03C
:1032800063F810B96378042B03D90123637000231A
:103290002371AA68A11C203A284603F0A9F8002847
:1032A000D6D1E11C284603F0CCF807B030BD00BFF2
:1032B000308400002DE9F04385B06946032003F017
:1032C000C4F818B1FF2005B0BDE8F08302A90720BB
:1032D00003F0BBF80028F5D102469DF800509DF898
:1032E00008609DF803709DF80B809DF802901E4CBD
:1032F0002946207803F067F800B33146607803F080
:1033000062F8D8B1A378042B01D0BB4216D1E37880
:10331000042B01D0434511D12379042B0CD16379BF
:10332000022B16D1114A1248492102F07FFA607926
:10333000831E022BC7D9C5E74B45F0D00132032AC3
:1033400004F10604D4D10B48492102F06FFA0120A0
:10335000B9E7032B05D0084A0849042B18BF0A46D1
:10336000E1E7074ADFE700BF94910000AD9100005C
:10337000C9910000DC910000A6910000B791000007
:10338000B2910000054B1868043B1B68092B03D160
:10339000431E584258417047002070473401FF00D7
:1033A00008B5474B1B68092B01BF4FF05023002283
:1033B000C3F81421C3F81821FFF7E4FF30B101234B
:1033C000404A1360A2F63822C2F878353C4B1B689D
:1033D000092B07D13C4B1B68012B1EBF01223B4B25
:1033E000C3F87825FFF7CEFF10B10E22384B1A60D4
:1033F000334B1B68092B04D10022364B1A60012283
:103400005A600022D30003F57F03D3F80013013183
:1034100008D0D3F800130132D3F80433B2F5807F1B
:103420000B60EFD12C4BDA69D1073BD52B4B1946FA
:10343000D3F80024012AFBD1C3F80425D1F80034C5
:10344000012BFBD1244BDA69D20708D5DA6923496D
:1034500022F00102DA61D1F80024012AFBD11A6AB4
:1034600001320AD11A6A22F0FF0242F020021A62E7
:103470001A4AD2F80034012BFBD10022174BC3F8B3
:103480000425D3F80024012AFBD1BFF34F8F144940
:10349000144BCA6802F4E0621343CB60BFF34F8F52
:1034A00000BFFDE71B6A0133C0D00D4AD2F88C3053
:1034B00043F44063C2F88C300B4B0C4A1A6008BDD1
:1034C0003001FF00384A00503401FF000040005036
:1034D000E4AE03500C4700500080FF000090035002
:1034E00000ED00E00400FA058C4501200090D003B7
:1034F000044B1A7922B9012218601A7102487047E8
:1035000002487047805501200000AD0B0C00AD0B48
:1035100010B1012820D070474FF05022D2F8183453
:10352000D2F81814C90311D503F00303022B0DD1EF
:10353000C2F8183500220D4B1A601B6802224FF0AA
:103540005023C3F8042301229A6070474FF05023A0
:103550000122C3F81825EDE70022054B1A601B680D
:103560004FF05023C3F80403186070470451005013
:103570000051005038B510B1012818D038BD4FF0B7
:1035800050230222012142F210751C46C3F8082381
:10359000154A10601268154A1160D4F81834DB031C
:1035A000ECD5012002F074FF013DF6D1E6E74FF0C3
:1035B0005024002242F210750D4BC4F808031A6023
:1035C0001B680C4B1860D4F80C34D4F80C2403F0AE
:1035D0000103D203D2D5002BD0D0012002F058FF36
:1035E000013DF0D1CAE700BF045100500C5000501B
:1035F0000051005004500050164B10B51A6852B1DB
:10360000002018601B6801224FF05023C3F80823E4
:10361000114B1B689847114B1A688AB100221A6037
:103620001B684FF05023D3F81824D3F8181402F075
:103630000302012A4FF0020103D1C3F818159A6062
:1036400010BDC3F80813044B0120BDE810401B68EF
:10365000184700BF00510050805501200451005010
:103660000B4A70B51668F14389B271B10025ECB20E
:1036700021FA04F3DB0705F10105F8D50123A34086
:10368000334304700348136070BD0348FCE700BF78
:10369000885501200000AD0B0200AD0B012303FA99
:1036A00000F010F0FF0F12D04FF02003EFF3118164
:1036B00083F31188BFF36F8F064AD36C23EA0000AF
:1036C000D06481F31188BFF36F8F034870470348BC
:1036D000704700BF8C5501200000AD0B0400AD0BFE
:1036E0002DE9F041FF22002401258646144E15489D
:1036F000154FE3B24FF02001EFF3118881F31188E9
:10370000BFF36F8F22FA03F1C9070BD5F16C05FAED
:1037100003FC11EA0C0F01BF384641EA0C01F164C9
:103720008EF8003088F31188BFF36F8FB84205D050
:1037300005FA03F39A4304F10104DAD1BDE8F081FC
:103740008C5501200200AD0B0000AD0B0022034B95
:10375000C3F88425C3F80425704700BF00900350C8
:10376000044AD2F80834DB07FBD50160BFF35F8F52
:10377000704700BF0090035008B5C0F30B0383B936
:103780000222094BC3F88425C3F804254FF0FF3209
:103790000260D3F80024D207FBD5FFF7D7FF034818
:1037A00008BD0348FCE700BF009003500000AD0BCC
:1037B0000A00AD0B012208B5054BC3F88425C3F8F8
:1037C0000425FFF7CDFFBDE80840FFF7BFBF00BFEE
:1037D0000090035002680E4B9A4215D1C269A3F1C2
:1037E0001023A3F1EF139A420ED18368012B0BD85B
:1037F000C36813B10269934206D0436933B180694B
:10380000C31A584258417047012070471846704704
:1038100055AA00FF38B50D4B9D68A5B12846FFF7A6
:10382000D9FF014678B9EB686BB92C690CB9084629
:1038300038BD2046FFF7CEFF28B9E368AB4202D17E
:1038400025462469F2E70121F1E700BFDC5501209C
:103850002DE9F843404D2C68D4B1AC68C4B10028C0
:103860004DD000294BD001FB00F6B6FBF0F08842AA
:1038700045D1301D43D8B1070DD026F003070437DA
:10388000EC6803E06368BB423BD2A469002CF9D129
:103890002046BDE8F8833746F2E7E86044E007F1E8
:1038A000200C04EB0C03203959600021DFF8B0E054
:1038B000C3E902142169196144F80CE0DFF8A4C0DF
:1038C000C3F81CC001B1CB60C3E90520AAB1936164
:1038D0009A6902B15361236100234FF00109C4E9E1
:1038E00005332B69C4E90179DB072DD5FFF792FF7A
:1038F00050B31A4B48461B6825E0EB60E8E700240C
:10390000C6E7A3681BB1154B01201B689847D4E993
:103910000520616804F12008C91B2329BFD80123B1
:10392000A360002AB9D09061A36903B15A61002352
:10393000C4E905332B69DA0706D5FFF76BFF18B129
:103940000120064B1B6898473246002140464446FA
:1039500002F000FB9CE700BFDC55012094450120EC
:1039600055AA00FF669911EE2DE9F041074600289F
:103970007CD03F4D2B68002B78D0AA68002A75D0E8
:10398000834203D86A681344984203D3394B012019
:103990001B689847A7F120042046FFF71BFF18B1CA
:1039A000344B01201B68984757F8183C012B03D073
:1039B000304B01201B689847002357F8146C47F8D8
:1039C000183CAEB1B26892B957F81C3C03F1200222
:1039D00073681344736057F8103C336103B1DE60C1
:1039E00020462022002102F0B5FA234634461E4626
:1039F0002069002832D08368002B2FD16368426889
:103A00002033134463600369D4E905212361DAB9E3
:103A100001BB426981696261A161EAB19461A269F5
:103A200002B1546103B1DC602022002102F092FA5D
:103A30002B699B071AD5FFF7EDFEB8B1BDE8F04141
:103A40000C4B01201B6818479161A1690029E0D047
:103A50004A61DEE7E960F8E7EC60E0E7002EE7D1D5
:103A6000EB68A36103B15C61EC60E1E7BDE8F08164
:103A7000DC5501209445012038B50D461422002163
:103A80000446124802F066FA1149124800F032F872
:103A9000232D1AD914F003031FBF043DED18C3F101
:103AA0000403E4182A460021204602F053FA074B8B
:103AB000094AC3E900459C602260A2F11022203D22
:103AC000A2F1EF126560E261DC6038BDDC550120D7
:103AD000693900005138000055AA00FF014B1B68EE
:103AE000184700BF90450120014B1B68184700BFD5
:103AF00098450120024B1860024B00201960704766
:103B000090450120984501200A4619B1024B002139
:103B10001B681847704700BF9C450120F8B500F1AD
:103B200008054768044628460E4603F010F9874208
:103B300016D16368B3F5807F12D80021284603F0C0
:103B400076FA00280CDD0021284603F0D4F838B1BD
:103B500046B9002104F1140003F069FA00281EDCC4
:103B60001B481EE004F12C050021284603F05FFAF3
:103B70000028F5DD0021284603F0BDF80028EFD02D
:103B800004F138050021284603F051FA0028E7DD4A
:103B90000021284603F0AFF80028DAD1E0E70EB99B
:103BA0000020F8BD002104F1440003F040FA002891
:103BB000D6DD002104F1500003F039FA0028CFDDF2
:103BC000002104F15C0003F032FA0028E8DCC7E7CA
:103BD00080BFFFFF70B500210446FFF79FFF054639
:103BE000B8B904F10806304603F095F87F2810D9DB
:103BF00014342946204603F07EF850B1204603F0E5
:103C00008AF8012805D93146204603F0CDF900286D
:103C100000DB014D284670BD00BEFFFFF0B50C462D
:103C200087B0002105461646FFF778FF80BB03A842
:103C300002F0DBFF21466A6803A803F08EF8044611
:103C4000D0B905F10804214603A803F0ADF9002816
:103C50001BDA05F1680303A9009305F1140223465A
:103C600008466F6803F02CFD044628B93A463146F1
:103C700003A803F0AAF8044603A802F0BCFF0CB1A5
:103C8000A4F58544204607B0F0BD6FF00304F3E7C8
:103C9000004CF7E780BFFFFF0023C0E90033C1B944
:103CA000194A1A4BDFF88CC0C0E90223184B194A95
:103CB000C0E904C3184BC0E90623184B036203F1A3
:103CC0007453A3F52303A3F6924343628166002055
:103CD0007047134B134ADFF860C0C0E9022303F1B9
:103CE000794303F5740303F5016303610E4BC0E9E7
:103CF00005C303F1D14303F5C01303F51E63C3618C
:103D00000A4B03620A4BE0E767E6096A85AE67BBC8
:103D10003AF54FA57F520E518C68059BABD9831F96
:103D200007D57C36D89E05C1310BC0FFA78FF9643B
:103D3000A44FFABE72F36E3C39590EF72DE9F04FDD
:103D400000F10803D1B0059308AB019300F12803FB
:103D50000693019A059B53F8040B42F8040B06984E
:103D60009842F8D10DF140094A4601F140004B78E4
:103D70000C781B0443EA0463CC780431234311F824
:103D8000024C884243EA042342F8043BEFD1A14CA1
:103D9000CA46A446019B019A01990198D3F81C8058
:103DA000D2F818E04F69D0F810B0DB689268496823
:103DB00000680294DCF80040DAF800504FEAFB2675
:103DC00086EABB162C4486EA7B6626448EEA070404
:103DD00004EA0B0484EA0E04264440EA01054FEA93
:103DE0007034B04484EAB00400EA0106154084EA65
:103DF000B054354325444344DCF80440A844DAF881
:103E000004508BEA07062C44A6441E404FEAF324D4
:103E10007E4084EAB314B64484EA7364744448EA86
:103E200000054FEA783E08EA00068EEAB80E0D401B
:103E300035438EEAB85EAE44A6442244DCF808500E
:103E4000DAF808400CF1200C25442F4483EA0B05D6
:103E5000154085EA0B06BD194FEAF22787EAB2172B
:103E600087EA72672F4448EA0E044FEA7E3508EA73
:103E70000E0685EABE050440344385EABE55DAF8ED
:103E80000C6025445CF8144C39443444A34483EA60
:103E900002040C403D4484EA03070BEB07044FEA9D
:103EA000F12B8BEAB11B8BEA716BA3444EEA05063A
:103EB0004FEA75340EEA050784EAB50406EA0806F7
:103EC0003E4384EAB5545CF8107C3444DAF8106060
:103ED0005844374482EA01063B4406404FEAF02743
:103EE000564087EAB0175C44334487EA70671F4442
:103EF00045EA04064FEA743305EA040B83EAB40387
:103F000006EA0E0646EA0B0683EAB45333443B4402
:103F1000B8445CF80C6CDAF8147081EA000B3E448B
:103F200032440BEA080B4FEAF8268BEA010B86EACB
:103F3000B8165A4486EA7866164444EA03074FEAFC
:103F4000733204EA030B2F4082EAB30247EA0B07FD
:103F500082EAB3523A443244B644DAF818705CF854
:103F6000086C80EA080B3E4431440BEA0E0B4FEA22
:103F7000FE268BEA000B86EABE16594486EA7E6668
:103F80000E44AF194FEA723143EA0205254003EAB5
:103F9000020B81EAB20145EA0B0581EAB2512944DC
:103FA00031445CF8045CDAF81C600AF1200A3544FC
:103FB000054488EA0E00384080EA080B05EB0B0048
:103FC0004FEAF72585EAB71585EA7765054404EBDE
:103FD000050B4FEA713042EA010480EAB1001C404F
:103FE00002EA0106344380EAB15020440A4C2844D6
:103FF00064457FF4DFAECDE90D7ECDE90801CDE962
:104000000A2309F1C004CDF83C80CDF830B0079404
:1040100004E000BF4084000080840000D9F83840EC
:10402000D9F804604FEAF44C8CEA744CD9F800508B
:104030008CEA942CD9F824404FEAB64A2C448AEAF8
:10404000F61A8AEAD60AA4444FEAFB250CEB0A04C6
:1040500085EABB15049485EA7B648EEA070505EAC8
:104060000B0585EA0E052544029C09F12009246C04
:104070002C44049D2C44A04403EB080C40EA0104AA
:104080004FEA7033C9F8205083EAB00300EA010513
:10409000144083EAB0532C431C44D9F81C30A0448C
:1040A0004FEAF34585EA734585EA9325D9F8083048
:1040B00059F8184C33442B44029D4FEAB4466D6CBA
:1040C00086EAF41686EAD4063344AE448BEA070641
:1040D0000EEB030506EA0C064FEAFC2E7E408EEA44
:1040E000BC1E8EEA7C6E2E440EEB060502EB050A22
:1040F0004FEA783E40EA080200EA08068EEAB80E67
:104100000A4032438EEAB85E9644049AAE444FEABF
:10411000F24585EA724585EA9225D9F80C2059F8CE
:10412000146C22442A444FEAB644029D84EAF614F1
:1041300084EAD604AD6C22448BEA0C0404EA0A0437
:104140003D44154484EA0B042C444FEAFA2585EAE1
:10415000BA1585EA7A652C44214448EA0E054FEAEF
:104160007E37039187EABE0708EA0E01054087EA19
:10417000BE570D433D444FEAF34787EA7347C9F8FA
:10418000243087EA9323D9F8107059F8101C37446B
:104190003B444FEAB14787EAF11787EAD1071F444A
:1041A000039B8CEA0A061E40029B2544DC6C86EACF
:1041B0000C065C44E3191E44039BC9F828204FEA0F
:1041C000F32484EAB31484EA7364A31900EB030BA9
:1041D0004FEA75344EEA05000EEA050684EAB50496
:1041E00000EA0800304384EAB55404441C444FEA12
:1041F000F24383EA724383EA9222D9F8143059F8E1
:104200000C0C1944039BC9F82C700A448AEA030673
:104210004FEAB041029B81EAF01181EAD0011B6DA7
:10422000114406EA0B060B44634486EA0A061E4460
:104230004FEAFB2383EABB1383EA7B639A1945EABF
:1042400004064FEA743305EA040C83EAB40306EA71
:104250000E0646EA0C0683EAB453334413449044F2
:1042600059F808CCD9F818204FEAF74686EA77467D
:1042700086EA972716184FEABC4282EAFC1282EAC5
:10428000DC023E441644039AC9F8301082EA0B0758
:1042900007EA08075740029AC9F83460526D324461
:1042A000524417444FEAF82282EAB81282EA78624E
:1042B000D01944EA03074FEA733204EA030A2F4095
:1042C00082EAB30247EA0A0782EAB3523A44024456
:1042D00086444FEAF147D9F81C0059F804AC87EA44
:1042E000714787EA912100EB0C070F444FEABA416E
:1042F00081EAFA1181EADA010F4402998BEA080C8B
:10430000886D0399384408440CEA0E0C4FEAFE21EC
:104310008CEA0B0C81EABE11604481EA7E6108449C
:10432000C9F838704FEA72312F1843EA0205254068
:1043300003EA020C81EAB20145EA0C0581EAB251B6
:10434000294401444FEAF64080EA7640D9F800500B
:1043500080EA9626049888EA0E0C82444FEAB5401B
:1043600080EAF51080EAD505029856442E44C56DC2
:104370000CEA070C35444FEAF7205D448CEA080C40
:1043800080EAB71080EA77606544054404EB050BCA
:104390004FEA713042EA0104C9F83C6080EAB1009A
:1043A0001C4002EA0106344380EAB1502044029CDA
:1043B000284420340294079C4C457FF42FAECDE96D
:1043C0000D7ECDE90801CDE90A23CDF83C80CDF87A
:1043D00030B0059B01991B6851F8042B1344059AD2
:1043E000019142F8043B069B05929342F1D10020D3
:1043F00051B0BDE8F08F00BFF8B5104B104F53F827
:104400002050013053F82060AE4200D8F8BDD5E905
:1044100000342046984770B16CB10123E41B24118D
:10442000084A610952F8210004F01F0403FA04F459
:10443000044342F821400835E6E700BF408500000C
:104440000846012078460120084BC01A0011084B8D
:10445000420953F82220012300F01F0003FA00F064
:1044600010420CBF18460020704700BF08460120CC
:1044700078460120114970B505460E46104C8C4215
:1044800004D10F4CB4420AD1002414E02046FFF7B7
:10449000DBFF10B12368AB420DD01034EFE72046AC
:1044A000FFF7D2FF08B91034ECE72168284601F085
:1044B0000BFD0028F7D1204670BD00BF78460120D3
:1044C00008460120F7B505460E464FF02003EFF3EE
:1044D000118783F31188BFF36F8F00F09DFB0022DB
:1044E000042D98BF184B044694BF53F82530174B42
:1044F000009245212A46164801F098F93EB1F36929
:10450000C3F308031BB14521124801F08FF934B100
:10451000204603F0F6FC034608B1027802B90E4BC0
:10452000224645210D4801F081F931462846FEF723
:1045300059FE87F31188BFF36F8F204603B0BDE8A3
:10454000F040FEF777B800BF588500003B920000AE
:10455000519200007E92000049920000A492000057
:104560000248034A0021121A01F0F4BCD04601208F
:1045700080730120012208B5084B02201A70FFF752
:104580003BFF00F063FB0320FFF736FFFBF758FF0C
:10459000034A137B23F00103137308BD7E730120CC
:1045A000D046012008B5144B03F5006282F3088859
:1045B00083F30A880025E023104C84F82230E57745
:1045C00025766576A576636A43F4E0236362FEF799
:1045D00005F8FDF799FD4FF0FF332846A362E3622B
:1045E000FFF70AFF0120FFF707FF2B462A4629465F
:1045F0000348FDF765FD00BF809B012000ED00E052
:104600007545000070B50E4B0E4CA34201D300203F
:1046100070BDD3E9030141EA000212F003020BD19D
:104620009D685A61AA4201D11C33EEE75E690132EE
:104630000E6059610144F5E76FF01500E8E700BF2F
:104640007C4601207C460120D3B50C4616461F4609
:104650004FF02003EFF3118183F31188BFF36F8FC5
:1046600043695BB123601B684361836901338361E4
:10467000002081F31188BFF36F8F11E056EA070223
:1046800003D123606FF00B00F3E70246CDE900672A
:10469000044800F05BFA18B9034B9B685B69236020
:1046A00002B0D0BD7F730120F0550120F8B504465B
:1046B0000D464FF02003EFF3118683F31188BFF30B
:1046C0006F8F47696FB903F0EDFB50B12A68C76778
:1046D000426103F08FFB3146BDE8F840074800F027
:1046E000CBB82B6862691A602B686361A369013BD0
:1046F000A36186F31188BFF36F8FF8BD7F7301202C
:104700002DE9F341044616461F464FF02003EFF310
:10471000118883F31188BFF36F8FC368324A6BB17E
:1047200080689168884219D056EA070318D188F347
:104730001188BFF36F8F6FF00F000CE0916891F953
:104740000E100133E36093682161A36088F3118840
:10475000BFF36F8F002002B0BDE8F0812169F0E760
:1047600090F90E3091F90E109942A8BF194621EA2E
:10477000E17199422CDA00F0F9F90546CDE90067BC
:1047800022464146194800F0E1F90028E3D04FF0F5
:104790002003EFF3118683F31188BFF36F8F236833
:1047A0002169A34207D033B193F90E309942A8BFD3
:1047B000194621EAE171A06890F90E30994209D1B9
:1047C0006DB13146094800F057F86FF00A00C2E7B2
:1047D0000025D3E700F0CAF90028F2D1F0E786F30C
:1047E0001188BFF36F8FF0E7F05501207F73012030
:1047F00038B583680446002B33D01D4A9268934233
:1048000032D1C368012B05D0013BC36003F0DEFA4F
:10481000002038BD4FF02003EFF3118583F311889A
:10482000BFF36F8F0169806890F90E30994201D013
:1048300000F09CF9204603F035FBA06058B190F9D8
:104840000E2022610022C26703F0D4FA29460948EB
:1048500000F012F8DAE7E06085F31188BFF36F8F9C
:10486000D4E76FF01500D4E74FF0FF30D1E700BF79
:10487000F05501207F73012049B9EFF3058030B96D
:10488000054B5A6A9B689A4201D0FDF78DBB81F3B4
:104890001188BFF36F8F7047F0550120094B03F16A
:1048A0002802824205D19B688B4202D14B7BDB06FA
:1048B00006D1D1E9003213605A600023C1E9003308
:1048C000704700BFF05501200F4A10B51369044628
:1048D0000BB1D0680DE002F1280003F085FA916871
:1048E0004B7B13F0200F1CBF43F008034B730028D1
:1048F000EFD03CB99368597BC90603D1816900297F
:1049000008BF1846506210BDF055012070B4437BBB
:104910001A0629D4DB0627D183692BBB134A02F17F
:104920002801D2E90A348B4218D0BBB190F90E505D
:1049300093F90E60AE420CDD5A68C0E90032106097
:104940005860437B63F07F03437370BC0020FFF724
:10495000BBBF9C4202D01B68002BE9D1C0E9001408
:10496000D36A1860D062ECE770BC7047F055012044
:1049700070B50446183003F0C6FA4FF02003EFF389
:10498000118683F31188BFF36F8F94F90D30002BDC
:1049900007DA21460E48FFF781FF637B03F07F03B0
:1049A00063730C4D637BA86843F010036373031BB0
:1049B00058425841FFF788FF86F31188BFF36F8F85
:1049C000AB68A34203D1BDE8704003F0F5B970BDF8
:1049D00018560120F05501202DE9F04104464FF012
:1049E0002003EFF3118283F31188BFF36F8F437BB2
:1049F00013F0280F05D082F31188BFF36F8FBDE845
:104A0000F08143F02003437382F31188BFF36F8F6B
:104A1000183003F078FA4FF02003EFF3118683F398
:104A20001188BFF36F8F637BD80616D1A269A2B934
:104A3000190607D521462248FFF730FF637B03F0B4
:104A40007F0363731F4B9868021B50425041FFF76E
:104A50003BFF04F1300800271DE09B07F9D52146F4
:104A6000A068FFF71BFF637B23F00203637300233F
:104A7000A360EEE705F1180003F045FAA86829469F
:104A8000FFF70CFF6B7BAF6023F002036B73EF67E4
:104A90002846FFF73BFF256B454501D0002DE9D1A6
:104AA000637B43F008036373236E86F31188BFF3BF
:104AB0006F8F002BA3D02046BDE8F041184700BF00
:104AC00018560120F055012010B590F90D3004461C
:104AD000002B07DA01460848FFF7E0FE637B03F08E
:104AE0007F036373054B9868031B58425841BDE828
:104AF0001040FFF7E9BE00BF18560120F055012015
:104B00002DE9F041064614461D464FF02003EFF311
:104B1000118783F31188BFF36F8F03F09BF987F33D
:104B20001188BFF36F8F6B1C08BFB4F1FF3F08D033
:104B300022462B4606F118000349BDE8F04100F07B
:104B4000F3B8BDE8F08100BF157E000010B50C463B
:104B500005481146DDE902238068FFF7D1FF2046B2
:104B6000BDE81040FDF720BAF05501202DE9F041D5
:104B700004464FF02003EFF3118883F31188BFF34D
:104B80006F8F437B4EB2DB062ED1836963BB184D1A
:104B9000014605F128073846FFF780FEAB6AA67389
:104BA000BB422A4619D0C3B1E96A93F90E00B0425C
:104BB0000EDD5A68C4E9003214605C600120FFF722
:104BC00083FE012088F31188BFF36F8FBDE8F08169
:104BD000994202D01B68002BE7D1D36A276063603B
:104BE000D36A1C60D462E9E7A6730020EAE700BF3D
:104BF000F0550120013108BFB0F1FF3F08B506D1E3
:104C0000044B9868FFF7B4FE4FF0FF3008BD00205A
:104C1000FCE700BFF0550120014B9868704700BFCA
:104C2000F055012008B54FF02003EFF3118483F312
:104C30001188BFF36F8F044B98681861FFF798FED7
:104C40002046FDF7B1F900BFF0550120024A0349A3
:104C5000034800F0EBBD00BFA3920000C492000027
:104C6000D192000008B50648064A0749121A01F019
:104C700047F9BDE80840054A0549064801F040B932
:104C800000450120CC4601201093000000000000E8
:104C9000F892000000450120034B1B680BB9FDF79B
:104CA000A7B80020704700BF2056012030B5036828
:104CB00068B10A4A5268904209D043B1D3E904214D
:104CC000D0E90445121945EB0101C3E9042142680A
:104CD00013605A600023C0E9003330BDA0450120B5
:104CE00038B5104B1C689C4208BF0024FFF7D4FF66
:104CF00094B1D4E90423141A63EBE075012C75F127
:104D000000030CDB6FF000420023A242204673EB4D
:104D1000050400DA104638BD6FF00040FBE70020C4
:104D2000F9E700BFA04501202DE9F74F0191591C7B
:104D300008BFB2F1FF3F82466ED0541C43F100051C
:104D40006FF001034FF0FF3BB3EB04086BEB050979
:104D5000B8F1000F79F100030FDBFFF79DFF6FF053
:104D60000103344AD2E9001C5B1A6BEB0C021E1BD8
:104D700062EB0507341A67EBE075019BCAF808304F
:104D80004FF02003EFF3118683F31188BFF36F8F89
:104D9000FFF782FF012C75F100032146B8BF012106
:104DA0002A46B8BF0022244B0C1842EBE0751A6863
:104DB000CAE904459A4201D05F6852B95A68CAF8F4
:104DC0000030CAF804205A68C2F800A0C3F804A052
:104DD00014E0D2E90489DAE90445444575EB090198
:104DE0001DDAB8EB040069EB0501C2E90401516862
:104DF000CAE90021C1F800A0C2F804A01A689A42CA
:104E000006D0924504D1FFF76BFF0021FCF7BEFFEF
:104E100086F31188BFF36F8F03B0BDE8F08FB4EB5A
:104E2000080065EB0901BA42CAE90401C6D012685C
:104E3000C3E700BF50470120A04501202DE9F74FEF
:104E40004FF02003EFF3118583F31188BFF36F8FC9
:104E50002C4BDFF8B4909846CB46DFF8B0A0186032
:104E6000D8F800C0DAF800406646D9E90023544576
:104E7000CDE900234FEAE6770CD05CB1D4E9041207
:104E80008C4577EB02031BDAB1EB0C0062EB0701F8
:104E9000C4E904010024009BC8F80040F218019BFB
:104EA00047EB0303CBE90023FFF71AFF2146FCF78A
:104EB0006DFF85F31188BFF36F8F03B0BDE8F08FEE
:104EC0000022DDE9006700237618ACEB010047EB18
:104ED000E177C8F80000C4E904232046C9E9006767
:104EE000FFF7E4FE85F31188BFF36F8FA36898473F
:104EF0004FF02003EFF3118583F31188BFF36F8F19
:104F0000AEE700BF2056012050470120A0450120F8
:104F100038B5064C064DAC4201D3002038BDD4E96B
:104F20000112204603F005F81434F4E77C46012012
:104F30007C46012010B50A4C23681BB101230020D8
:104F4000236010BD00F0AEF80028F7D00138062825
:104F500003D8044B53F8200010BD034810BD00BF18
:104F6000245601206C850000FE8FFFFFBFF34F8F9A
:104F70000549064BCA6802F4E0621343CB60BFF3F5
:104F80004F8F00BFFDE700BF00ED00E00400FA0511
:104F90004FF0FE33002130B4064A074D074C2B601A
:104FA00013602360064A074CEB606368C2F8001583
:104FB00030BC1847041484500014845008148450E2
:104FC00000008450A8450120024BD0E90012C3E93B
:104FD00000127047A845012048B143682BB1BFF3C8
:104FE0005F8F0023036018467047024870476FF4D4
:104FF000E0407047EA8FFFFF10B5044628B16368B0
:1050000013B100232360636010BD024B02485B684C
:105010009847F4E7A84501208885000010B50446AC
:1050200030B100226368226043F00103636010BD69
:105030000148FFF7ADFFF4E7B085000080B1436899
:1050400063B10122D0E8EF3FC0E8E12F0029F9D198
:10505000012BF7D0BFF35F8F0020704702487047E5
:105060006FF4E040704700BFEA8FFFFF70B40B4B56
:105070000668C268D0E90154C3E90242C3E9006589
:10508000D1E903020E68064BD1E90154C3E900657A
:10509000C3E902401A6170BC704700BFB8450120E7
:1050A000C845012010B500F033F820B1032400F00A
:1050B00067F8204610BD00F035F890B900F0B0F860
:1050C00090B90F4B1B681B0EF02B08D10D4A0E4BED
:1050D00012689A420AD0072400F01CF8E7E7062479
:1050E000FAE70424204610BD0024F5E7012000F073
:1050F00097F804460028F7D1044B1860D9E700BFA1
:1051000028198450241A84500000E0200C1A84507E
:105110000020704700207047014B1860704700BFA7
:10512000041A845010B5114800F048F800B110BDC1
:105130000F4800F043F80028F9D10E4C204600F04B
:105140003DF80028F3D10C4B0C481C6000F036F8F9
:1051500001460028EBD100F02DF8044608B12046A6
:1051600010BD00F03FF82046FAE700BF00460120DE
:10517000F4450120FC45012004460120F8450120AA
:1051800008B5084800F024F8074800F021F807485F
:1051900000F01EF8064800F01BF8BDE8084000F0DB
:1051A0000BB800BF00460120F4450120FC4501205A
:1051B000F845012000207047704700BF08B5034B39
:1051C00002681B6810689847002008BDB845012098
:1051D00008B5034B02685B6810689847002008BD5B
:1051E000B845012070B5094C094D2069AB68984756
:1051F00018B1084B08485B6898470021074AEB68DC
:1052000011602069BDE87040184700BFC845012003
:10521000B8450120A8450120D4850000385601205A
:1052200070B51A4D1A4E0446B26828699047F0B915
:105230005CB1184C2368ABB1012B1AD0013B236041
:105240002869F3689847002070BD124C216839B96D
:105250000120114B114AC3F800051368002BFCD143
:1052600001312160F36828699847002070BD0C481F
:1052700070BD0A4A1368002BFCD1074A6FF07E40CC
:10528000C2F80035FFF748FF2368D7E7C84501207B
:10529000B845012038560120000084501019845070
:1052A000E98FFFFF29B101290CBF07206FF015001E
:1052B0007047032070472DE9F7430E46174699467D
:1052C000044628B94FF0FF38404603B0BDE8F083EC
:1052D0000029F7D0002AF5D0CB680D8938461D4447
:1052E000042329460DEB030200F0B8FC8046002899
:1052F000E8D146F60812BDF804107389914223D113
:10530000BDF806109942DDD1042329440DEB0302B8
:10531000384600F0A3FC0028D4D146F60713BDF8A8
:1053200004209A42CED19DF82830BDF80620A37201
:105330007389C4E900672B44E36004351344A4F87F
:10534000089063612561BFE7002BE6D0BAE72DE93D
:10535000F3410E4617461D46044620B94FF0FF3074
:1053600002B0BDE8F0810368002BF7D04368002B42
:10537000F4D04FF6FF78D4E904239A4216D223687A
:105380005B8923B1E368934204BF043323610423A0
:1053900021690DEB0302606800F060FC0028DDD19C
:1053A000A27A236922B1E2689A4201D80120D7E7A4
:1053B000B4F808C0BDF80620C44502F1040103D0CA
:1053C000BDF804E0E6450BD11DB1BDF804C0A5F859
:1053D00000C0043333603A8022690A442261BFE787
:1053E0000B442361C7E72DE9F74306460F46914674
:1053F0001D4600F09FFC082804461ED8304600F0E9
:10540000A2FCAC4238BF2C468046E4B22A4649464C
:10541000684600F075FD621B41460DEB050000F08B
:1054200099FD23466A463946304600F034FC003088
:1054300018BF012003B0BDE8F0834FF0FF30F9E75B
:1054400000F04EBD4FF4C0735843303070470B78B6
:1054500003F0FB03032B14BF4FF0FF304FF4C07079
:10546000704710B5044600F065FC4FF4C072A368A5
:10547000303B02FB103010BD012307B5816801AA43
:1054800020398DF80430FFF7AEFF03B05DF804FB60
:1054900013B50446019100F093FF0423A0F1080125
:1054A0000DEB03022046FFF79EFF02B010BDF7B5DB
:1054B000044600200D461746FFF7F4FE6946C0B2C9
:1054C000FCF7D0F930B10126009800F0C6FB304659
:1054D00003B0F0BD2C2303FB05452989EB68009838
:1054E000CC18042321460DEB030200F0B7FB06465F
:1054F0000028E8D146F60813BDF804206D899A42C9
:105500001AD1BDF806309D4201D00326DCE7042302
:1055100029190DEB0302009800F0A0FB0028D2D15E
:1055200046F60713BDF804209A42EED1BDF80610E6
:10553000294421443960C7E7002DF1D0E5E7F8B5EB
:1055400013460F461646002102460546FBF760FC4F
:10555000044650B9334605F12C0201212846FBF7D9
:1055600057FC10B1002F18BF04462046F8BD37B5D0
:1055700080250446426A01A903200195FCF786F9BB
:1055800048B9019B226DA36201A907200195FCF790
:105590007DF9054608B1012505E0019B206A636598
:1055A00000F0C8FBE065284603B030BD012303606E
:1055B00003F1012343600023C0E9023370474379BC
:1055C000012B07D10368012B04D10079431E5842F7
:1055D00058417047002070477FB506460D460320AE
:1055E00001A9FCF73FF938BB0198FFF73AFFF16DCD
:1055F0000446284600F0E4F80444019800F09AFBC1
:105600000646019800F09FFB082201460DEB0200C0
:1056100000F0A0FC2B7921468DF8083002AA334611
:10562000019800F038FB041C18BF0124019800F019
:1056300014FB204604B070BD0124F7E700F054BB12
:105640002DE9F8430F46002106460846FFF72AFEDB
:10565000044601210020FFF725FE3B789C4220D024
:10566000984220D101242C2303FB0464F06DA56A29
:10567000FFF7E8FE00268146013D636A384603EBEA
:10568000C50253F83510D2F804801B684246C91A87
:105690004644FFF7D3FFB14505F1FF35EDD8BDE82E
:1056A000F8830024DFE70120F9E737B515460C46FB
:1056B0000720694600F0C9FEE979012903D00022DC
:1056C000204600F0D6FE9DF80330012B02D1204683
:1056D00000F0ABFEA9682046FFF7DAFE2046FDF792
:1056E0008BFD002003B030BD73B50D460646FBF7B9
:1056F00077FC0446E86038B102282FD101A90320C5
:10570000FCF7B0F818B10124204602B070BD2A465B
:1057100031460198FBF7CAFB0446D8B9019800F05E
:105720004FFE012301460DF10302019800F096FAA5
:1057300004460028E7D101220DF10301019800F091
:1057400051FE10B101238DF803309DF8033003F0B2
:105750000F03EB71019800F080FAD5E70724D3E737
:1057600013B5032001A9FCF77DF848B90198FFF7AC
:1057700083FE0446019800F070FA204602B010BD86
:105780000124FAE71FB5032001A9FCF76BF8A8B9BB
:1057900002A90198FDF73EFD044668B99DF80B305B
:1057A000032B03D1019800F040FE0446019800F05D
:1057B00054FA204604B010BD0124F7E70124F8E7AD
:1057C00030B543790468012B0ABF0122022200256B
:1057D00001FB02F204F1FF3402FB04F2037918BF6B
:1057E000CD01013B01FB0323581930BD60B1436873
:1057F00003F00303012B03D0032B05D103681BB176
:1058000000238360184670476FF0150070474268A8
:10581000034602F00302032A4FF0000281600CBF2E
:10582000006810465A607047002070470FB407B5F3
:1058300004A951F8040B0191FBF7BEFD03B05DF81C
:1058400004EB04B07047038B13F0070305D1036822
:10585000002B0CBF002003207047022B05D1438B87
:10586000002B14BF002004207047012B05D10368D2
:10587000002B0CBF002005207047002070472DE949
:10588000F0410D4607461946281D90461E46FFF773
:10589000BEFF044638B13346424629463846A44640
:1058A000BDE8F0416047BDE8F08110B44FF020043E
:1058B000EFF3118284F31188BFF36F8F416110BC45
:1058C0000121FBF787BD10B50C4640B139B1081D69
:1058D000FFF78CFF28B9A36833F0030301D06FF002
:1058E000150010BD38B50C46054658B151B10B68CE
:1058F00043B14B6833B11C22002100F02BFB002088
:105900002C6138BD6FF01500FBE770B504460D46FD
:10591000FFF7D9FF061E31DB4FF02003EFF31181B3
:1059200083F31188BFF36F8F4FF6FF76638B208B65
:10593000B34200F007022ED0022A0ED10133638356
:105940001646012381F31188BFF36F8FB3B1002393
:1059500029462046FFF793FF10E0830701D0062A6F
:105960000ED100232B60636893B9C4E90055164635
:1059700062B90A4620460221FBF72CFD304670BD75
:10598000052A0CBF6FF022066FF004060023D9E74A
:105990001D606560EBE76FF00A06F7E7836800EBD0
:1059A000C101B3F5004F2CBF51F8220031F81200AD
:1059B000704700EBC1018068B0F5004F2CBF41F883
:1059C000223021F81230704708B50122FFF7E6FFB8
:1059D000400808BD836800EBC101B3F5004F08D350
:1059E0004B681AB143F001034B60704723F0010389
:1059F000FAE74B881AB143F001034B80704723F05C
:105A00000103FAE753000122FFF7D3BF8368481C64
:105A1000B3F5004F2CBF02230123C01AB0FA80F067
:105A2000C0F11F0070472DE9F04104460D46FFF715
:105A3000CBFFA3680146B3F5004F01D3012835D051
:105A40002046FFF7E3FF04EB800216699EB90123AD
:105A500003FA00F0E36829460343E360204615613A
:105A60002B460222FFF7A5FF032229462046BDE868
:105A7000F041FFF79EBF022231462046FFF78EFF1E
:105A800007460346022229462046FFF792FF334687
:105A9000032229462046FFF78CFF032239462B4676
:105AA0002046FFF786FF02223146DFE7BDE8F0819E
:105AB000B2F5802FF8B52CBF082504250023551B0F
:105AC0000022CC1D0D4424F0070425F007052D1BF2
:105AD000ED0804602946C4E90023C4E902522046C7
:105AE000FFF794FF134686001B36471CF60804F1A7
:105AF0001001BB4229DB324620460021FFF782FF1E
:105B0000AF1B204601220021FFF764FF3A463146D1
:105B1000FFF778FF3346314620460022FFF749FF62
:105B2000294620460022FFF76DFF3B4629462046C6
:105B30000022FFF73EFF294620460122FFF74AFFD9
:105B40003146BDE8F840FFF76EBF41F8042B013342
:105B5000CFE72DE9F04F8BB09B469DF854300E46B1
:105B60000393149B92461946002205460024CDE972
:105B700000129DF85880189F0DF11009DDE90023EF
:105B800050465946FAF7DEFAD3B2092B84BF2732C2
:105B9000D3B2303309F8013BDDE900239B4508BF50
:105BA000924504F1010423D2179BA3EB040A2AEACD
:105BB000EA7AD346AAEB0B09BBF1000F01D0039B95
:105BC000CBB9A2460AF1FF3A04AB314613F80A00FA
:105BD000A847BAF1000FF5D1DA46BAF1000F10D19B
:105BE0003B681C444C445C443C600BB0BDE8F08F07
:105BF00082468B46C2E731464046A8470BF1FF3B41
:105C0000D8E731464046A8470AF1FF3AE5E7704732
:105C1000FDF7C6BB8368DB681847FEF72BBC70B581
:105C200002684C68A24216D38B6823449A4206D27B
:105C3000D1E90435AB4204D36FF00B038B61002034
:105C40000AE0CD68121B45F83320426805EBC30615
:105C5000013372600B61012070BD70472DE9F04186
:105C60001E46836805468B420C4617460FD37218B2
:105C700093420CD3C068FFF7D0FF69682144836862
:105C80003A461C683346A446BDE8F04160476FF0D1
:105C90001500BDE8F0812DE9F84398468368074672
:105CA0008B420D4691461CD308EB0102934218D358
:105CB000C068FFF7B2FF06460021FFF7ABFF0446BE
:105CC00060B979682944B3684A465C6830464346FF
:105CD000A047044601213046FFF79CFF2046BDE85F
:105CE000F8836FF01504F9E783682DE9F0418B42E2
:105CF00007460D4690461AD30A44934217D3C0680C
:105D0000FFF78BFF06460021FFF784FF044658B9D2
:105D100079682944B36842469B68304698470446F0
:105D200001213046FFF776FF2046BDE8F0816FF095
:105D30001504F9E708B5C068FFF76FFF83681B69B2
:105D40009847007808BD08B5C068FFF766FF83680C
:105D50001B699847007908BD83685B6818470C2366
:105D6000C268C9B201FB0323186C00F0070070473A
:105D70004FF02003EFF3118283F31188BFF36F8F8D
:105D8000036813F0C00301D08B4207D101230360E5
:105D9000002082F31188BFF36F8F70474FF0FF3000
:105DA000F7E710B54FF02003EFF3118283F311886A
:105DB000BFF36F8F036803F00704012C06D1016065
:105DC000002082F31188BFF36F8F10BD03F0C00372
:105DD0008B4214BF4FF0FF306FF04400F1E74FF0FB
:105DE0002003EFF3118283F31188BFF36F8F0368F1
:105DF00003F0C00343F00203036082F31188BFF392
:105E00006F8F70476FF022007047C3681C2010B47A
:105E1000CCB204FB0030002110BC10470020FDF77D
:105E200077BB0020FDF7A6BB38B50C24C9B24C43A4
:105E30000546C06804F1400380211844FFF798FF2D
:105E4000002804DB69680C4463689847002038BD6B
:105E50002DE9F0410C24C9B24C43C568064604F153
:105E600040008021284490461F46FFF79AFF0028F3
:105E700006DB2544C5E90E8773681B599847002047
:105E8000BDE8F0817047704770470020FBF726BDE2
:105E900000210120FCF756B9836E83F30B8870470D
:105EA00001460068FCF74EB908B5FCF779F9BDE882
:105EB0000840FCF79FBB40E800F313F4803FD8B2E2
:105EC00008BF6FF0150070470138013910F8013F25
:105ED00011F8012F934201D1002BF7D1981A704786
:105EE00010B55AB10139841810F8012B11F8013F8F
:105EF000A04201D09A42F7D0D01A10BD1046FCE75C
:105F0000F0B581EA0004A50703460BD0013B0A4423
:105F100091421AD1F0BD002AFCD011F8014B013A90
:105F200003F8014B9C07F6D19508AC001E1F0F1912
:105F3000B94205D16FF00306234406FB0522E5E7CD
:105F400051F804CB46F804CFF2E711F8014B03F8FF
:105F5000014FDDE7034670B5C9B29C0710D141EA95
:105F6000012444EA0445940803EB8406B3420DD1AE
:105F70006FF0030505FB04241C44A34209D170BD46
:105F8000002AFCD003F8011B013AE6E743F8045B62
:105F9000ECE703F8011BF0E74FF0FF307047436870
:105FA00000205B681B690B60704743685B6858683A
:105FB00042400A4042405A60002070474368002037
:105FC0005B6899607047436800205B68D9607047E0
:105FD000436800205A685368594051607047C3684D
:105FE00030B5586858B10024814213D108685CB9B3
:105FF0009C685860A14200D198600020086072B986
:10600000002030BD2846EFE720609868814208BF35
:106010009C60F2E705680446002DF3D13AB15A6856
:106020000A60986859600028EAD19960E9E76FF042
:106030001500E6E70020704738B504460D4600F02D
:1060400034FA844209D2002C07DBA84205D32C4441
:1060500084428CBF0020012038BD0020FCE72DE9E0
:10606000F0470024836886B0894692465B6902AA9D
:1060700001A99847A0462546029BAB4202D806B02C
:10608000BDE8F0870026019F07EBC5077B680493F6
:106090003A6808EB0603B24202D801359846EBE7AE
:1060A000514603A803940593C8470028E7D0049BF2
:1060B00001361C44ECE7436810B41B68D3F8042392
:1060C000D20518D5D3F82021AAB14FF02001EFF363
:1060D000118281F31188BFF36F8FD3F8201131B192
:1060E0000021C3F82011D3F820110121D96082F3D7
:1060F0001188BFF36F8FC268D2685AB1D3F85811B4
:1061000051B10021947B116134B14FF48000C3F888
:106110000803917310BC7047D3F8241121B10021FA
:10612000C3F82411D3F824311368002BF2D051683E
:1061300010BC18470A46C368043393E8030082E89A
:1061400003000020704743681B68D3F88004C3F83D
:106150008004704742681368D3F8580138B99279BF
:1061600032B9D3F82001003018BF01207047012058
:1061700070474368C2681B68D3F8100148B100201B
:10618000527D0A70C3F81001D3F8102101221A6061
:1061900070474FF0FF307047F8B54368C6681D6818
:1061A000F3689C8910339442A8BF14460122D3E8B7
:1061B000EF7F002F04D1C3E8EC2FBCF1000FF6D124
:1061C0000CBF13460023E3B91C462046F8BDF26815
:1061D000CF5C9268D7540133A342F8DB4FF0200321
:1061E000EFF3118183F31188BFF36F8FFFF7B2FFD5
:1061F000F36840B90446186181F31188BFF36F8FCB
:10620000E3E70023E8E79B68C5F844350023C5F8B9
:106210004845C5F82031D5F82021C5F85831D5F8C2
:1062200058310123AB60E7E743681A68D2F81031B0
:1062300053B1C3680020C2F81001D2F81001012048
:106240005B7D0B7010607047184670474368C168EB
:106250001A684FF02000EFF3118380F31188BFF329
:106260006F8F0020C96888734FF48001C2F804134F
:1062700083F31188BFF36F8F70470122C368DB6817
:106280009A737047C368DB689A7B02F0FF0162B9BA
:1062900042681268D2F8580140B1D2F8040310F4F1
:1062A000800003D0196101207047002070474368C7
:1062B0001B68D3F81001003018BF0120704710226E
:1062C00043681B68C3F804237047102243681B68A7
:1062D000C3F8082370474FF4007243681B68C3F883
:1062E000042370474FF4007243681B68C3F8082307
:1062F000704701207047C368DB68C3E9001270472C
:1063000038B5436804461D68D5F804335B0205D4EC
:10631000D5F8040310F0100006D138BDFFF7B2FF26
:106320000028F5D00120F8E72046FFF7C0FF003035
:1063300018BF0120F1E708B5FBF774FDFBF71EFE5F
:10634000BDE80840FEF7F6BD38B50C461546FFF728
:10635000FAFC21462544A94201D1012038BD11F89B
:10636000013B9842F7D00020F8E72DE9F3410546BC
:106370000E469046FFF7DEFC082804461DD8284646
:10638000FFF7E1FC002C08BF01240746012241462B
:106390006846FFF7B5FD621E39460DF10100FFF7B3
:1063A000D9FD23466A4631462846FFF774FC003083
:1063B00018BF012002B0BDE8F0814FF0FF30F9E7CF
:1063C00080682838704704280AD0052804D111F1C4
:1063D000FF3018BF01207047431A58425841704798
:1063E0000120704711B10AB1FFF7AEBF002070471E
:1063F00038B50C460123114622460546FFF72EFC10
:10640000002810DB012221462846FFF7EBFF18B1D8
:1064100003230020237038BD2378012B0CBF0123F8
:1064200002232370F7E70120F5E7012307B5816810
:1064300001AA18398DF80430FFF797FF03B05DF813
:1064400004FB8268183AFFF7D3BF13B50C46C0B2FD
:1064500001A9FBF707FA50B921460198FCF7DAFECB
:1064600004460198FFF7F9FB204602B010BD012455
:10647000FAE707B541EA021281688DF8072028394A
:106480000DF10702FFF771FF03B05DF804FB004751
:1064900001F033BD08B50520FBF7ECFD20B9BDE8E0
:1064A00008400520FBF7D6BD08BD4FF480107047AB
:1064B0004FF4805070474FF4807070470020704751
:1064C000036830B5CD1A002D0CDD1C7814F0800F58
:1064D0000BD15C1C04601B7813600368C91A136835
:1064E0008B4232D96FF05F0030BD04F07F04013C75
:1064F000032C27D8DFE804F00209121E012DF1D089
:106500005C78023314600360E7E7022DEADDB3F83C
:106510000140033364BAA4B21460F4E7032DE1DD53
:106520009C785D78240244EA0544DD7804332C43EA
:106530001460E8E7042DD5DDD3F80140053324BA13
:106540001460E0E76FF06300CEE70020CCE770B4A2
:1065500004680E1B002E07DD26789E4208D1013408
:10656000046070BCFFF7ACBF6FF05F0070BC704799
:106570006FF06100FAE737B50223154601AA044619
:10658000FFF7E5FF40B9019A2168284600F0E5FBD6
:106590002368019A1344236003B030BD0023F0B593
:1065A0001D460439854201D11846F0BD4F68FC1ADA
:1065B00041F8044F52F825600135B4422CBF4FF02A
:1065C000000C4FF0010CA41B9F422CBF63460CF142
:1065D00001030C60E6E72DE9F04384460D464FF0D9
:1065E000000E02F14004BCF10F0F54F8408C05F18D
:1065F000400504F1400400F2BF806FF00F044FEA41
:10660000101C04FB0C004FEA8C1C072801EB0C0546
:1066100002EB0C0440F29C8051F80C600838A3FB9C
:1066200006671EEB060E2CBF4FF001094FF0000964
:1066300018EB0E0142F80C102CBF012200226E68EC
:10664000B944A3FB06674A4492192CBF01210021DB
:1066500001EB070C6168203552182CBF0121002185
:10666000626055F8186C6144A3FB066789192CBF5A
:106670000122002202EB070CA268203489182CBFEB
:106680000122002244F8181C55F8146C6244A3FB44
:10669000066792192CBF0121002101EB070C54F869
:1066A000141C52182CBF0121002144F8142C55F859
:1066B000106C6144A3FB066789192CBF01220022DC
:1066C00002EB070C54F8102C89182CBF0122002271
:1066D00044F8101C55F80C6C6244A3FB0667921931
:1066E0002CBF0121002101EB070C54F80C1C52189F
:1066F0002CBF0121002144F80C2C55F8086C614492
:10670000A3FB066789192CBF0122002202EB070CAC
:1067100054F8082C89182CBF0122002244F8081CC8
:1067200055F8046C6244A3FB066792192CBF4FF026
:10673000010E4FF0000E54F8046C0EEB0701921995
:106740002CBF4FF0010E4FF0000E44F8042C8E4485
:106750002146800005EB000C654551F8042B40F004
:106760009A810444236813EB0E0344F8043B4FF072
:10677000010EF7D2BDE8F08355F8406CACF1100C77
:10678000A3FB06671EEB060E2CBF4FF001094FF06E
:1067900000091EEB08062CBF4FF001084FF000085F
:1067A00044F8806C55F83C6CB944A3FB0667C844B8
:1067B00018EB06082CBF4FF0010E4FF0000E54F8F6
:1067C0007C6C0EEB070916EB08062CBF4FF0010E90
:1067D0004FF0000E44F87C6C55F8386CCE44A3FBA7
:1067E00006671EEB060E2CBF4FF001084FF00008A5
:1067F00008EB070954F8787C17EB0E072CBF4FF015
:1068000001084FF0000844F8787C55F8346CC8440F
:10681000A3FB066718EB06082CBF4FF0010E4FF0E4
:10682000000E54F8746C0EEB070916EB08062CBF2B
:106830004FF0010E4FF0000E44F8746C55F8306CB8
:10684000CE44A3FB06671EEB060E2CBF4FF00108DB
:106850004FF0000808EB070954F8707C17EB0E079F
:106860002CBF4FF001084FF0000844F8707C55F839
:106870002C6CC844A3FB066718EB06082CBF4FF02E
:10688000010E4FF0000E54F86C6C0EEB070916EB7E
:1068900008062CBF4FF0010E4FF0000E44F86C6C50
:1068A00055F8286CCE44A3FB06671EEB060E2CBFE2
:1068B0004FF001084FF0000808EB070954F8687C16
:1068C00017EB0E072CBF4FF001084FF0000844F8FB
:1068D000687C55F8246CC844A3FB066718EB0608CF
:1068E0002CBF4FF0010E4FF0000E54F8646C0EEB0D
:1068F000070916EB08062CBF4FF0010E4FF0000EF3
:1069000044F8646C55F8206CCE44A3FB06671EEB7C
:10691000060E2CBF4FF001084FF0000808EB0709E6
:1069200054F8607C17EB0E072CBF4FF001084FF0B6
:10693000000844F8607C55F81C6CC844A3FB06674B
:1069400018EB06082CBF4FF0010E4FF0000E54F864
:106950005C6C0EEB070916EB08062CBF4FF0010E1E
:106960004FF0000E44F85C6C55F8186CCE44A3FB55
:1069700006671EEB060E2CBF4FF001084FF0000813
:1069800008EB070954F8587C17EB0E072CBF4FF0A3
:1069900001084FF0000844F8587C55F8146CC844BE
:1069A000A3FB066718EB06082CBF4FF0010E4FF053
:1069B000000E54F8546C0EEB070916EB08062CBFBA
:1069C0004FF0010E4FF0000E44F8546C55F8106C67
:1069D000CE44A3FB06671EEB060E2CBF4FF001084A
:1069E0004FF0000808EB070954F8507C17EB0E072E
:1069F0002CBF4FF001084FF0000844F8507C55F8C8
:106A00000C6CC844A3FB066718EB06082CBF4FF0BC
:106A1000010E4FF0000E54F84C6C0EEB070916EB0C
:106A200008062CBF4FF0010E4FF0000E44F84C6CDE
:106A300055F8086CCE44A3FB06671EEB060E2CBF70
:106A40004FF001084FF0000808EB070954F8487CA4
:106A500017EB0E072CBF4FF001084FF0000844F869
:106A6000487C55F8046CC844A3FB066718EB06087D
:106A70002CBF4FF0010E4FF0000E54F8446C7744D9
:106A800016EB08062CBF4FF0010E4FF0000E44F835
:106A9000446CBE44A7E555F8046BA3FB06781EEBD7
:106AA000070E2CBF0126002612EB0E022CBF4FF062
:106AB000010E4FF0000E464441F8042CB6444BE65C
:106AC00073B501F18041013900EB8101814201D2AE
:106AD00002B070BD03680025019304230DEB03028F
:106AE000144612F8016B013B13F0FF0346EA05253B
:106AF000F7D10A680192042214F8016B013A12F0EE
:106B0000FF0246EA0323F7D140F8043B41F8045959
:106B1000DCE72DE9F04F8B46914685B00E9C019045
:106B20006268A068920000210393FFF713FADBF874
:106B30000430D9F80480A568434528BF43462E4653
:106B40000024029308F101039B000093019BA045E0
:106B5000186821D1009B1F1FEE193A463146FFF7F6
:106B6000CFF955F81730D9F80820013345F8173018
:106B700031462046FFF712FD55F81730181A019BD1
:106B800045F817001D680023C0B2C0F101079C4200
:106B900020D105B0BDE8F08FDBF8081050F824A034
:106BA00033680F68324607FB0A37039B02985F433E
:106BB0005346FFF710FD32463B46D9F808104046D1
:106BC000FFF709FD009B46F804AB1A460023013489
:106BD000B350BBE756F8231055F82320414302FB7E
:106BE000071245F823200133D1E7002301228360F7
:106BF000C0E90023704710B5044668B1806830B121
:106C000061688900FCF780FFA068FCF76DFF002336
:106C10000122C4E90023A36010BD42F2107399421F
:106C200070B504460D4602D96FF00F0070BD436881
:106C30008B4216D204212846FCF750FF0646002856
:106C4000F2D0A16859B162689200FFF759F9616802
:106C5000A0688900FCF758FFA068FCF745FFC4E96D
:106C600001560020E2E7884270B505460E4603D083
:106C70004C683CB9FFF7BFFF002011E0B36853F840
:106C8000243013B9013C002CF8D16A680134336810
:106C9000A2422B6005D221462846FFF7BEFF40B135
:106CA00070BDA868121B9200002100EB8400FFF762
:106CB00051F9A200B168A868FFF722F9DCE770B5C6
:106CC0000E4601210446FFF7A8FF054688B9626811
:106CD00001469200A068FFF73DF9A36886EAE672D4
:106CE000002EA2EBE6721A60B4BF4FF0FF3301230F
:106CF0002360284670BD4368B1EB431F3FBF8368E4
:106D00004A0953F8220001F01F013ABFC84000F0C1
:106D100001000020704743688BB18268013B83B952
:106D200052F8231000204FF00042114204D10130EC
:106D300020284FEA5202F8D10133C0EB4313184622
:106D4000704752F823100029EAD1013BE7E708B564
:106D5000FFF7E1FF0730C00808BD2DE9F04112F050
:106D6000030418BF0124436804EB9204A3420746BE
:106D70008846154608D100213846FFF7A0FF064691
:106D800088B13046BDE8F081FFF735FF00230122CE
:106D9000BB60C7E9002321463846FFF73EFF0646A1
:106DA0000028E8D0EDE7B8F1000FEAD0BB68C5EBEA
:106DB00084002A4641461844FFF7A2F8002CE0D090
:106DC0002146B868FFF77CFEDBE7F8B505466C683E
:106DD0000846A40094421CD2121B8E180021FFF713
:106DE000B9F830462246002310449A4213D10020BD
:106DF000F8BDAF6803F0030123F0030CCE0057F891
:106E00000C10F14011F0FF0F11D10133A342F0D16A
:106E1000E9E71346FAE7AF6803F0030123F003063E
:106E2000CC00B9590133E14000F8011DDDE76FF0F6
:106E30000700DDE7F8B505460E464C0901F01F07CF
:106E4000FFF769FF6B683044B0EB431F04D81F2E77
:106E50000ED89FBB00200AE010F01F0118BF0121CF
:106E600001EB50112846FFF7D8FE0028EFD0F8BDFF
:106E70006FF0030161436B689A00A342A2F1040220
:106E800007D800229B00043B191DE2D0A968CA5014
:106E9000F9E7A868013B861876588650EDE7A868A0
:106EA00050F8241001FA07F3134340F8243021FA74
:106EB00006F201346B68A342F1D8CBE70022C7F198
:106EC0002006F7E74368F0B44C09A34201F01F0223
:106ED00001D304D18AB3F0BC0021FFF7F0BE1F2913
:106EE00015D90023A5004168091B994201D8002447
:106EF0000AE081684E59043541F823600133F2E716
:106F0000816841F82340013341689942F8D812B9A9
:106F1000F0BC0020704700244368C2F1200713F141
:106F2000FF33F5D3866856F8235025FA02F1214342
:106F300046F8231005FA07F4F1E71F29E8D91346AC
:106F4000D5E730B543682BB94A6862B9181C18BF39
:106F5000012028E0826802EB830252F8042C002A08
:106F6000F2D1013BEFE78C6804EB820555F8045C35
:106F700085B9013AE9E7826852F8231054F82320D2
:106F8000914205D803F1FF330AD24FF0FF300AE0F7
:106F9000012008E00BB19342FAD89342F5D3013BAC
:106FA0005A1CE8D1002030BD30B5436823B94A6887
:106FB0005AB9002B38D131E0826802EB830252F8D3
:106FC000042C002AF3D1013BF0E78C6804EB820526
:106FD00055F8045C25BB013AEAE79342096801D2FF
:106FE0004A4222E00268002A03DD002913DA012266
:106FF0001BE000290FDD72B14FF0FF3215E0816810
:1070000051F8235054F823108D420ED803F1FF336A
:1070100002D2524209E0013B591CF0D1002204E0A7
:10702000002BDAD09342D8D90268104630BD1FB584
:1070300081EAE173A3EBE17300290093B4BF4FF041
:10704000FF3301230193012301A90293CDF80CD052
:10705000FFF7AAFF05B05DF804FB90422DE9F0416F
:1070600006460C46154602D0884229D12C460123FB
:107070006568336065BB29463046FFF7CEFD07469D
:1070800018BBA1680446B36885422AD103EB850387
:10709000DCB1726805F10108AA4208D841463046C1
:1070A000FFF7BBFD00282FD1B36803EB85031A68F7
:1070B0004546141943F8044B2CBF01240024E7E78C
:1070C000FFF7D1FD07460028D0D03846BDE8F08153
:1070D000A36803EB850353F8043C002BCBD1013D9F
:1070E000C8E753F8202012EB040C51F820202CBFE5
:1070F000012400241CEB020243F820202CBF0122B3
:10710000002201301444BFE70746DEE7F0B516461B
:107110000023012285B0B04205460F46CDE9012388
:10712000039306D1014601A8FFF79DFD044620BB4D
:1071300001AEBD421AD1D6E9014201232B6014BB36
:10714000A9682046FFF72AFA70B14FF0FF316B684B
:10715000A34224D9AB6853F82420E2B1AA6852F8BC
:107160002430013B42F82430002406E0394628460A
:10717000FFF779FD04460028DDD001A8FFF73BFDAD
:10718000204605B0F0BD02EB840353F8043C002B0D
:10719000D6D1013CD3E743F824100134D7E7DDD141
:1071A0006FF00904ECE7F8B50C6813680546634313
:1071B0000F46164616D511463846FFF7C2FE002880
:1071C00006DB324639462846FFF7A0FF40B1F8BD3E
:1071D0003A4631462846FFF799FF0028F7D1644226
:1071E0002C60F4E7FFF739FFF0E7F8B50C68136897
:1071F00005466343002B0F46164616DD11463846FA
:10720000FFF79FFE002806DB324639462846FFF787
:107210007DFF40B1F8BD3A4631462846FFF776FF7C
:107220000028F7D164422C60F4E7FFF716FFF0E77F
:107230002DE9F04300231646012287B0884280469C
:107240000F46CDE90023CDE90232CDE9043305D163
:107250006846FFF708FD0546E8B96F46B04506D118
:10726000414603A8FFF7FFFC0546A0B903AED7F8D7
:107270000490B9F1000F18D1746804BB09EB040144
:107280004046FFF7CAFC054628B901464046FFF7CD
:1072900016FD054638B303A8FFF7ADFC6846FFF7B7
:1072A000AAFC284607B0BDE8F083BB6803EB89035E
:1072B00053F8043C002BDFD109F1FF39D9E7B3685B
:1072C00003EB840353F8043C002BD7D1013CD4E7F3
:1072D000B368D8F8082053F8243002EB8402B96868
:1072E0004846FFF778F914F1FF34F1D23A68336871
:1072F0005343C8F80030CEE71FB50123009201AA1E
:10730000CDE90133CDF80CD0FFF792FF05B05DF861
:1073100004FB2DE9F04F824697B0884618460021BD
:1073200091460293FFF783FE002800F09481002429
:10733000012502994846CDE90754CDE90945CDE933
:107340000B44CDE90D54CDE90F45CDE91144CDE90C
:1073500013541594FFF7F5FDA04229DABAF1000F96
:1073600007D1B8F1000F1BD10024204617B0BDE8AB
:10737000F08F21465046FFF7A2FC04460028F0D0CB
:1073800007A8FFF738FC0AA8FFF735FC0DA8FFF7A0
:1073900032FC10A8FFF72FFC13A8FFF72CFCE4E742
:1073A00049464046FFF75FFC04460028E8D1DBE78A
:1073B000494607A8FFF757FC04460028E0D10AAF6A
:1073C00002993846FFF74FFC04460028D8D1D9F877
:1073D00004100DA802310A950795FFF71EFC04461C
:1073E0000028CDD101460DA8FFF769FC044600280E
:1073F000C6D1022110A8FFF710FC04460028BFD117
:10740000032113A8FFF709FC04460028B8D1384629
:10741000FFF781FC00F01F001F286DD0C0F11F0393
:10742000194607A80093FFF705FD04460028A7D1D9
:1074300000993846FFF7FEFC04460028A0D1089EBC
:107440000B9D3846A6EB050B4FEA4B1319460193EB
:10745000FFF7F0FC0446002892D14FEA8B0B394627
:1074600007A8FFF7A1FD002848DA01993846FFF781
:1074700029FD0446002883D16B1E01939B00771ED3
:10748000039306F1804605F18043023B013E9B00D9
:10749000751B0593AD00019B9F423ED8BAF1000FCA
:1074A0000BD00DA95046FFF7DEFB18BB029BD9F8A5
:1074B00000201B685343CAF80030B8F1000F3FF4B6
:1074C0005FAF009907A8FFF7FDFC98B9D9F8003025
:1074D00007A940460793FFF7C6FB0146002840F086
:1074E000B8804046FFF7A3FD00287FF449AF012391
:1074F000C8F80030044643E70094A0E70F9951F81C
:107500000B20013241F80B2007A93A460846FFF745
:107510006CFE04460028A2D032E70398099B0C9A1F
:10752000BE00125853F82710301F04900F98914254
:1075300000EB050B77D34FF0FF334351DBF80030FE
:107540000133CBF80030A6F1080B0F9A00215359F4
:1075500010A8013B5351FFF7B2FB0028CAD1019B91
:107560000C9A002B73D0059BD158129B196003997C
:10757000525810A95A600F9B08465A59FFF7BCFE93
:107580000146002865D113A8FFF799FB0028B1D167
:10759000099A012F18BF52F80B00159B0499186027
:1075A000515810A85960925913A99A60FFF7FCFC32
:1075B0000028CADC0F9B0AA95A5910A8FFF79CFEA5
:1075C000002897D1EE00314610A8FFF733FC0028C1
:1075D00090D107A9084610AAFFF707FE0146002828
:1075E00037D107A8FFF723FD002819DA0AA910A848
:1075F000FFF739FB00287FF47DAF314610A8FFF775
:1076000019FC00287FF476AF07A910AA0846FFF7F7
:10761000CAFD00287FF46EAF0F9A5359013B5351B6
:10762000013F043D37E7049818586AB10023F8F782
:1076300089FD00234FF0FF328B4208BF824200D207
:107640001046CBF8000079E74FF0FF30F9E70199D9
:107650008BE70C4694E66FF00B0486E670B50446A3
:107660000D46104600211646FFF7E1FC002824DBFA
:107670002A46334621460020FFF74BFE054638B127
:10768000284670BD324621462046FFF78CFD90B952
:1076900000212046FFF7CBFC0028F3DB31462046D3
:1076A000FFF782FC0028EBDB324621462046FFF73D
:1076B0009CFD0028F2D00546E2E76FF00905DFE700
:1076C0002DE9F04FADF2646D04900F46184600218D
:1076D00006921E46FFF7ABFC002840F3EB81B3682F
:1076E0001C6814F00103089300F0E481002106985F
:1076F000FFF79DFC0028C0F2DD810321A51C6D0071
:1077000005F00805254405FB04F30139C3F1020324
:1077100003FB05F5F7D101234FF4C06218A8CDE9AA
:107720000C31CDE90E13CDE91011CDE912311491D0
:10773000FEF710FC0698FFF7EEFAB0F5287F80F010
:10774000F180EF2800F2F0804F2800F2EF80172838
:10775000089B88BF032303937368049803F101080F
:107760004146FFF75AFA0446002840F0B9804146E6
:107770001BA8FFF752FA0446002840F0B1804FEAF8
:1077800048010FA8FFF749FA0446002840F0A880F6
:107790003B68079301330AD1394612A8FFF763FA11
:1077A0000446002840F09C80012312AF1293DDF8BC
:1077B00088361BB19B68002B40F0BA8001210CA8D1
:1077C000FFF77DFA0446002840F08A8071680CA813
:1077D0008901FFF72FFB0446002840F081800CA9A7
:1077E00032460846FFF73AFF0446002878D1DDF814
:1077F000883623B10C2218460CA9FEF781FB3146CE
:107800003846FFF7D1FB0028C0F297803246394650
:107810001BA8FFF723FF0446002861D16D420DF13C
:107820003C082B4632460CA91DA8CDF80080FFF776
:1078300070F90CA90498FFF716FA044600284FD1F6
:1078400001270BAB1793049BCDF8008008330593F9
:1078500032462B4615A905980B97CDE91577FFF70A
:1078600058F9039BBB426DD14FF0000AD046D34676
:107870005746069BD3F80490BBF1000F40F0B98047
:10788000B9F1000F40F0B1804FF0010B039B0DF1F7
:107890003C0A0BFA03FBC14540F0EE8001230BAA22
:1078A0000B93CDE9153317922B46CDF800A0324645
:1078B00015A90598FFF72DF9079B013310D1069BF9
:1078C0005B686BB1069B9B681B68DB0708D5049B54
:1078D00031461A46079B10461360FFF764FC0446C6
:1078E000039B0C275D1E0123039A03FA05F503FA97
:1078F00002F6AE4200F2D7801BA8FFF77CF90FA872
:10790000FFF779F912A8FFF776F9DDF888360BB1A1
:107910009B6813B90CA8FFF76EF920460DF2646D51
:10792000BDE8F08F062316E7052314E7042312E7CA
:107930000C22DDF888160CA85FE739461BA8FFF774
:1079400092F968E7039B716803F1FF3907FA09F3BD
:107950000C27099307FA09F718AB1F440131384681
:10796000FFF75BF90028BAD11BA93846FFF77BF96E
:107970000028B4D1A24607F1080BCDF800802B46B1
:107980003246394658460AF1010AFFF7C2F8CA459D
:10799000F3D34FF0010B099B0DF13C0A03F10108F1
:1079A000039B0BFA03FBC3457FF65EAF716807F1DB
:1079B0000C0901314846FFF730F900288FD13946CC
:1079C0004846FFF750F9002889D107F11400CDF897
:1079D00000A02B4632461BA9FFF79BF808F10108CF
:1079E0004F46E0E74FF0020A46E74FF0200B09F15F
:1079F000FF39069B0BF1FF3B9B6853F8293023FAB4
:107A00000BF313F001030FD1BAF1000F3FF434AFC1
:107A1000BAF1010F08D1DDE904100FAB0093324633
:107A20002B46FFF776F827E7039A08F10108A2EB47
:107A3000080293401F43039B4345D3D14FF0000AF4
:107A4000DDE904100FAB009332462B460AF1010A20
:107A5000FFF75FF8D045F3D80C2118A801FB070108
:107A600000270FAB009332462B460598FFF751F8DD
:107A7000B846DDF820A0FFE6CDF800A02B46DDE9F2
:107A8000041032467F00FFF744F81BEA070F07D0C7
:107A9000CDF800A02B4632461BA90598FFF739F810
:107AA00009F10109F7E618AB07FB0530FFF7A3F86A
:107AB00001351EE76FF003042FE700207047704781
:107AC00070472DE9F8430446DDE90876914698466B
:107AD0000D4679B9B9F1000F15D1B8F1000F1AD1DF
:107AE0000FBB46BB7DB304F10800FFF730F96060BF
:107AF000002006E00830FFF7B6F80028EAD0A0F52D
:107B00008140BDE8F883494604F12C00FFF7ABF84B
:107B10000028E2D0F3E7414604F13800FFF7A3F86C
:107B20000028DDD0EBE7394604F12000FFF79BF891
:107B30000028D6D0E3E7314604F11400FFF793F8AC
:107B40000028CFD0DBE72846DBE770B504460E46B9
:107B500015460021AC22FEF7FDF9C4E9296570BD88
:107B600010B50446A0B38C30FFF745F804F1980037
:107B7000FFF741F804F16800FFF73DF804F1200039
:107B8000FFF739F804F13800FFF735F804F12C005D
:107B9000FFF731F804F11400FFF72DF804F10800A5
:107BA000FFF729F804F18000FFF725F804F17400CD
:107BB000FFF721F804F15C00FFF71DF804F1500015
:107BC000FFF719F804F14400BDE81040FFF713B8BF
:107BD00010BD6C220021FEF7BDB92DE9F843054622
:107BE0000F46144612B90020BDE8F883036803F07D
:107BF0003F06D318036022BF436801334360A6B138
:107C0000C6F140094A4510D300F128084A4608EB5E
:107C10000600FEF775F941462846FCF78FF8002864
:107C2000E2D1344406464F44403C274405E0284610
:107C3000FCF784F80028D7D1403C3F2CA7EB040187
:107C4000F5D8002CCFD005F1280022463044FEF7AD
:107C500057F9C8E770B50D468021036800F1280682
:107C600003F03F035A1C382A0344044683F82810C3
:107C700006EB020061D80021C2F13802FEF76AF972
:107C8000D4E900315A0F42EAC102DB0012BA1BBA32
:107C90002266636631462046FCF750F800284BD137
:107CA000E37A2B7063896B70A3681B0AAB70A368BF
:107CB000EB70E37B2B71E3896B71E3681B0AAB719B
:107CC000E368EB71E37C2B72638A6B7223691B0A96
:107CD000AB722369EB72E37D2B73E38A6B73636989
:107CE0001B0AAB736369EB73E37E2B74638B6B745A
:107CF000A3691B0AAB74A369EB74E37F2B75E38B59
:107D00006B75E3691B0AAB75E369EB7594F8233077
:107D10002B76638C6B76236A1B0AAB76236AEB7631
:107D2000A36E4BB994F827302B77E38C6B77636A9B
:107D30001B0AAB77636AEB7770BD0021C2F140028A
:107D4000FEF708F931462046FBF7F8FF0028F3D18B
:107D500001463822304691E7FEF795B830B5002449
:107D6000846141EA020414F00304C0E902320161B3
:107D70000CD14461A34203D1C0E90000002030BD12
:107D8000456901340D6041611144F3E76FF015005E
:107D9000F5E703460020C3E90033C3E9020070475A
:107DA000034620B9EFF305820AB9FAF7FDB883F369
:107DB0001188BFF36F8F70474FF02003EFF31180EE
:107DC00083F31188BFF36F8FFFF7EABF704710B5D9
:107DD000044601468068FCF761FD637B23F00203E3
:107DE00063730023A36010BD0368984214BF184654
:107DF0000020704710B54FF02003EFF3118483F398
:107E00001188BFF36F8FFCF781FD84F31188BFF3F6
:107E10006F8F10BD70B504464FF02003EFF311864D
:107E200083F31188BFF36F8F50F8103CA0F1180551
:107E300013B12846FFF7CBFF14F80B3C284623F07C
:107E4000140304F80B3CFCF761FD86F31188BFF3C3
:107E50006F8F70BD38B504460D46FCF735FE637B69
:107E600043F0020363737DB12B68A5609D4212D07D
:107E70008BB194F90E2093F90E10914205DD5A68EA
:107E8000C4E9003214605C6038BD69688B4202D07E
:107E90001B68002BEFD16B68256063606B681C600A
:107EA0006C60F1E738B54FF02003EFF3118283F3F4
:107EB0001188BFF36F8FFFF797FF044682F3118895
:107EC000BFF36F8F88B14FF02003EFF3118583F379
:107ED0001188BFF36F8FFFF77AFF85F31188BFF327
:107EE0006F8F04F1180000F00EF8204638BDEFF354
:107EF0000580003018BF0120704708B1F9F792BC27
:107F000070470020704710B54FF02002EFF3118446
:107F100082F31188BFF36F8F03683BB1FCF7C6FE95
:107F2000002084F31188BFF36F8F10BD6FF0150030
:107F3000F7E710B400F10C04C0E9034410BCFDF7EE
:107F4000B7BD70473082FF7F01000000FD170000C1
:107F5000000000000546000000000000114F000076
:107F600000000000A528000000000000F919000032
:107F700008460120793100001846012049310000EF
:107F8000284601203119000000000000391D0000C2
:107F900038460120BD6400000000000031290000C7
:107FA000484601203763000058460120C92C0000D4
:107FB0006846012000000000915E00000000000003
:107FC000915E000000000000915E000000000000D3
:107FD000915E000000000000915E0000F935000095
:107FE0008F64000000000000915E000000000000AF
:107FF000915E000028460120B7600000184601206D
:10800000B760000000000000915E0000000000006A
:10801000915E000000000000915E00000000000082
:10802000AD2B000000000000915E00000000000089
:10803000915E000000000000915E00000000000062
:10804000915E000000000000915E00000000000052
:10805000915E000000000000915E00000000000042
:10806000E91C000000000000915E0000000000001C
:10807000915E000000000000915E00000000000022
:10808000915E000000000000915E00000000000012
:10809000915E000000000000915E00000000000002
:1080A000915E000000000000915E000000000000F2
:1080B000915E000000000000915E000000000000E2
:1080C000915E000000000000915E000000000000D2
:1080D000915E000000000000915E000000000000C2
:1080E000915E000000000000915E000000000000B2
:1080F000915E000000000000915E000000000000A2
:10810000915E000000000000915E00000000000091
:10811000915E000000000000915E00000000000081
:10812000915E000000000000915E00000000000071
:10813000915E000000000000915E00000000000061
:10814000915E000000000000915E00000000000051
:10815000915E000000000000915E00000000000041
:10816000915E000000000000915E00000000000031
:10817000915E000000000000915E00000000000021
:10818000915E000000000000915E00000000000011
:10819000915E000000000000915E00000000000001
:1081A000915E000000000000915E000000000000F1
:1081B000915E000000000000915E0000338B000023
:1081C000030000007D9100000300000022910000E8
:1081D000030000000487000003000000249000005A
:1081E00003000000C192000003000000EB8A0000C1
:1081F00003000000E78A0000030000003391000044
:1082000001000000FFFFFFFFFFFFFFFFFFFFFFFF79
:108210001D0000001C0000001A0000001B000000F0
:1082200001000000000000000F0000000E00000030
:108230000338FDD87047000001000000D08900001D
:10824000448200000E010000000000000000000059
:1082500000C000000D8600000100000000C000000A
:10826000004000000D860000020000000000010038
:10827000000200000D860000030000000000010065
:10828000000007000D86000004000000000201004D
:1082900000FE06000D86000005000000000201003F
:1082A00000C000000D8600000600000000C20100B2
:1082B000003E06000D8600000700000000000800D8
:1082C000000007000D8600000800000000000F00FD
:1082D00000E000000D8600000900000000E00F0033
:1082E000002000000D8600000A000000055E00006E
:1082F000295E0000515E0000000000005F5D00008C
:108300008D1A00000D1B0000278B00001D5E000071
:10831000235E00002D8B0000A51900005D190000F0
:1083200000000000000000008B5E0000BD1E000089
:10833000751E00002D1F0000311E00002845012081
:1083400010450120204501200000000018450120B3
:1083500000450120000000000600010002000000AE
:108360006483000000000000A390000002000000F1
:10837000E0FF0F00E8440120AB9000002100000066
:10838000E0FF0320F92A00009F5F0000AB5F0000C0
:10839000BD5F0000C75F0000D15F000061290000E1
:1083A000DF5F000000000000FFFFFFFF002584509A
:1083B000000000004D2D0000892D0000E12C000080
:1083C00035600000C12C0000B12C0000040000004A
:1083D000FF00000073610000652F0000476100008E
:1083E000F92D00003561000099610000296200004C
:1083F0004D6200007B62000085620000BF620000E9
:10840000CB62000085620000AF620000D76200000E
:10841000E562000001630000F3620000F762000003
:10842000008000500600010000900050060001008E
:1084300077C295F360D2EF7F3552500F2CB679801A
:10844000982F8A4291443771CFFBC0B5A5DBB5E9BF
:108450005BC25639F111F159A4823F92D55E1CAB33
:1084600098AA07D8015B8312BE853124C37D0C55C1
:10847000745DBE72FEB1DE80A706DC9B74F19BC109
:10848000C1699BE48647BEEFC69DC10FCCA10C24F9
:108490006F2CE92DAA84744ADCA9B05CDA88F976DD
:1084A00052513E986DC631A8C82703B0C77F59BF47
:1084B000F30BE0C64791A7D55163CA066729291473
:1084C000850AB72738211B2EFC6D2C4D130D385310
:1084D00054730A65BB0A6A762EC9C281852C7292D2
:1084E000A1E8BFA24B661AA8708B4BC2A3516CC700
:1084F00019E892D1240699D685350EF470A06A1039
:1085000016C1A419086C371E4C774827B5BCB03487
:10851000B30C1C394AAAD84E4FCA9C5BF36F2E6825
:10852000EE828F746F63A5781478C8840802C78CB4
:10853000FAFFBE90EB6C50A4F7A3F9BEF27871C6B7
:108540004C7F00008C7F0000947F0000B47F00000F
:10855000B47F0000F5FFFFFFF1910000FF910000E4
:1085600013920000229200002E920000FF8FFFFF66
:10857000FF8FFFFFFE8FFFFFFE8FFFFFFD8FFFFFCF
:10858000FC8FFFFFFC8FFFFF6D757465785F66726F
:1085900065652063616C6C65642077697468204E42
:1085A000554C4C20706172616D65746572000000FD
:1085B00043616E277420696E697469616C697A65BC
:1085C000206D757465782C20776173204E554C4C66
:1085D0000D0A0000436F756C64206E6F74206C6F21
:1085E000636B20706F7765722073617665206D759F
:1085F0007465780025633A205374617274696E67FC
:1086000020626F6F746C6F616465720A004E52462F
:108610005F464C4153485F4452565F4E414D4500C2
:1086200025633A20466C61736820646576696365EA
:10863000202573206E6F7420666F756E640A0025A6
:10864000633A20556E61626C6520746F2066696EB6
:108650006420626F6F7461626C6520696D6167652B
:108660000A0025633A20426F6F746C6F6164657213
:1086700020636861696E6C6F616420616464726517
:108680007373206F66667365743A20307825780AB4
:108690000025633A204A756D70696E6720746F20FB
:1086A00074686520666972737420696D61676520FE
:1086B000736C6F740A0025633A2050726F7465639F
:1086C00074206D6375626F6F7420666C61736820CF
:1086D0006661696C65642C2063616E63656C2073F0
:1086E0007461727475702E0A0025633A204E6576A7
:1086F00065722073686F756C6420676574206865A7
:1087000072650A006D6375626F6F740025633A20AD
:10871000696E76616C696420666C61736820494497
:108720002025643B2065787065637465642025644A
:108730000A00000000000000000025633A202564C4
:108740002073746174757320777269746520666133
:10875000696C7320706572666F726D696E672074E4
:10876000686520737761700A007365636F6E64617A
:108770007279007072696D6172790025633A2049DF
:108780006D61676520696E207468652025732073AC
:108790006C6F74206973206E6F742076616C6964ED
:1087A000210A0025633A204661696C656420726580
:1087B0006164696E6720736563746F72733B2042F6
:1087C0004F4F545F4D41585F494D475F53454354A8
:1087D0004F52533D2564202D20746F6F20736D61BF
:1087E0006C6C3F0A0025633A204661696C65642021
:1087F00072656164696E6720696D6167652068658F
:1088000061646572733B20496D6167653D25750A3A
:108810000025633A204661696C6564207265616475
:10882000696E6720626F6F74207374617475733B37
:1088300020496D6167653D25750A0025633A207002
:10884000616E6963210A0025633A2043616E6E6F91
:108850007420757067726164653A206E6F74206170
:1088600020636F6D70617469626C6520616D6F75F6
:108870006E74206F6620736563746F72730A0025CF
:10888000633A2043616E6E6F742075706772616425
:10889000653A206D6F726520736563746F72732023
:1088A0007468616E20616C6C6F7765640A00256383
:1088B0003A2043616E6E6F742075706772616465F3
:1088C0003A206E6F742073616D6520736563746FF9
:1088D00072206C61796F75740A0025633A204465D3
:1088E00074656374656420696E636F6E7369737415
:1088F000656E7420737461747573210A0025633A80
:10890000204E6F7420656E6F7567682066726565AE
:1089100020737061636520746F2072756E207377A9
:10892000617020757067726164650A00676F6F64BB
:1089300000756E73657400626164005072696D61E8
:10894000727920696D6167650025633A2025733A65
:10895000206D616769633D25732C20737761705FBB
:10896000747970653D307825782C20636F70795F5D
:10897000646F6E653D307825782C20696D61676580
:108980005F6F6B3D307825780A005365636F6E64C6
:1089900061727920696D6167650025633A20426FD5
:1089A0006F7420736F757263653A207072696D61C0
:1089B000727920736C6F740A0025633A20426F6FDE
:1089C0007420736F757263653A206E6F6E650A006E
:1089D0003082010A0282010100D106081A18442CD3
:1089E00018E8FBFDF70DA34F1FBBEE5EF9AAD24BB3
:1089F00018D35AE96D188019F9F09C341BCBF3BCDD
:108A000074DB42E78C7F10537E435E0D572C44D1BC
:108A100067080F0DBB5CEEECB399DFE04D840BAA49
:108A2000774160ED152849A701B43C10E6698C2F09
:108A30005FAC414D9E5C14DFF2F8CF3D1E6FE75BEB
:108A4000BAB4A9C8887E473C94C37767544BAA8DB3
:108A50003835CA62617EB7E115DB7773D4BE7B72AD
:108A600021896924FBF8656E643EC80ED785D55C04
:108A70004AE4530D2FFFB7FDF31339833FA3AED262
:108A80000FA76A9DF9FEB8CEFA2ABEAFB8E0FA8207
:108A90003754F43EE12BD0D3085818F65E4CC88802
:108AA0008131AD5FB08217F28A692723F3AB873E2D
:108AB000931A1DFEE8F81A246659F81CABDCCE6840
:108AC0001B666435ECFA0D119DAF5C3AA7D167C601
:108AD00047EFB14B2C62E1D1C90203010001286EBE
:108AE000696C2900307800736F6300706F7765726E
:108AF000004661696C656420746F207265626F6FF7
:108B0000743A207370696E6E696E6720656E646C6E
:108B10006573736C792E2E2E0A00554152545F30C6
:108B200000434C4F434B006866636C6B006C66639C
:108B30006C6B00636C6F636B5F636F6E74726F6CF2
:108B4000007379735F636C6F636B006D7574657828
:108B50005F696E69742063616C6C65642077697409
:108B600068204E554C4C20706172616D6574657261
:108B700000436F756C64206E6F7420616C6C6F6362
:108B8000617465206D75746578206265666F7265C5
:108B900020696E697469616C697A696E6700256322
:108BA0003A2072302F61313A2020307825303878E1
:108BB000202072312F61323A2020307825303878E9
:108BC000202072322F61333A2020307825303878D7
:108BD0000A0025633A2072332F61343A202030781E
:108BE00025303878207231322F69703A2020307861
:108BF00025303878207231342F6C723A202030784A
:108C0000253038780A0025633A2020787073723A4C
:108C100020203078253038780A0025633A204661D4
:108C2000756C74696E6720696E73747275637469AC
:108C30006F6E206164647265737320287231352F02
:108C40007063293A203078253038780A0025633A55
:108C5000202A2A2A2A2A20425553204641554C547C
:108C6000202A2A2A2A2A0A0025633A20202053741F
:108C700061636B696E67206572726F720A002563AB
:108C80003A202020507265636973652064617461C5
:108C900020627573206572726F720A0025633A2034
:108CA00020204246415220416464726573733A2029
:108CB000307825780A0025633A202020496D7072AB
:108CC00065636973652064617461206275732065F2
:108CD00072726F720A0025633A202020496E737405
:108CE00072756374696F6E20627573206572726F3E
:108CF000720A0025633A202A2A2A2A2A204D505532
:108D0000204641554C54202A2A2A2A2A0A00256343
:108D10003A202020537461636B696E67206572721C
:108D20006F722028636F6E7465787420617265615C
:108D3000206D69676874206265206E6F74207661AB
:108D40006C6964290A0025633A202020556E7374EB
:108D500061636B696E67206572726F720A002563CA
:108D60003A2020204461746120416363657373205D
:108D700056696F6C6174696F6E0A0025633A202032
:108D8000204D4D46415220416464726573733A2010
:108D9000307825780A0025633A202020496E7374C4
:108DA00072756374696F6E204163636573732056D7
:108DB000696F6C6174696F6E0A0025633A20202028
:108DC000466C6F6174696E672D706F696E74206C8C
:108DD000617A79207374617465207072657365724D
:108DE000766174696F6E206572726F720A00256316
:108DF0003A202A2A2A2A2A2055534147452046410B
:108E0000554C54202A2A2A2A2A0A0025633A20206F
:108E1000204469766973696F6E206279207A657281
:108E20006F0A0025633A202020556E616C69676ED9
:108E30006564206D656D6F7279206163636573731E
:108E40000A0025633A202020537461636B206F76FB
:108E50006572666C6F772028636F6E746578742016
:108E600061726561206E6F742076616C6964290A95
:108E70000025633A2020204E6F20636F70726F636D
:108E80006573736F7220696E737472756374696F42
:108E90006E730A0025633A202020496C6C65676177
:108EA0006C206C6F6164206F66204558435F5245AB
:108EB0005455524E20696E746F2050430A0025634A
:108EC0003A202020496C6C6567616C2075736520C1
:108ED0006F662074686520455053520A0025633A36
:108EE000202020417474656D707420746F20657843
:108EF000656375746520756E646566696E6564206A
:108F0000696E737472756374696F6E0A005265736B
:108F1000657276656420457863657074696F6E204C
:108F2000280053707572696F757320696E7465726D
:108F3000727570742028495251200025633A2053DD
:108F40005053454C20696E20746872656164206DD1
:108F50006F646520646F6573206E6F7420696E6442
:108F60006963617465205053500A0025633A202AD2
:108F70002A2A2A2A2048415244204641554C54204E
:108F80002A2A2A2A2A0A0025633A202020427573B9
:108F9000206661756C74206F6E20766563746F72E5
:108FA000207461626C6520726561640A0025633A11
:108FB0002020204661756C7420657363616C617458
:108FC000696F6E20287365652062656C6F77290A6A
:108FD0000025633A202A2A2A2A2A204465627567D6
:108FE000206D6F6E69746F72206578636570746947
:108FF0006F6E20286E6F7420696D706C656D656E84
:1090000074656429202A2A2A2A2A0A0025633A201C
:109010002A2A2A2A2A20257320256429202A2A2A56
:109020002A2A0A006D70750025633A204661696C32
:10903000656420746F20616C6C6F63617465206E71
:109040006577204D505520726567696F6E202575D4
:109050000A0A0025633A20506172746974696F6E60
:109060002025753A2073616E6974792063686563A1
:109070006B206661696C65642E0A0025633A20499D
:109080006E76616C696420756E6465726C79696E68
:109090006720726567696F6E20696E646578202548
:1090A000750A00464C4153485F30005352414D5FB2
:1090B00030004750494F5F300025633A20756E619C
:1090C0006C69676E656420616464726573733A20CD
:1090D00030782530386C783A257A750A0025633A5D
:1090E00020696E76616C6964206164647265737373
:1090F0003A2030782530386C783A257A750A002580
:10910000633A206E6F7420776F72642D616C6967AB
:109110006E65643A2030782530386C783A257A7557
:109120000A00666C6173685F6E7266005541525446
:109130005F3100756172745F6E7266785F7561721F
:1091400074650025633A204661696C656420746F1C
:1091500020616C6C6F6361746520505049204368D6
:10916000616E6E656C0A0025633A20526573657402
:1091700074696E672073797374656D0A0066617433
:10918000616C5F6572726F720048575F434333587A
:10919000585F3000040104030402040104010403C5
:1091A00001030304010472657665727400746573CB
:1091B00074007065726D004255473B2063616E27F5
:1091C000742068617070656E0025633A2053776182
:1091D0007020747970653A2025730A0025633A205F
:1091E0005377617020747970653A206E6F6E650AEE
:1091F0000043505520657863657074696F6E005543
:109200006E68616E646C656420696E7465727275F7
:10921000707400537461636B206F766572666C6F57
:1092200077004B65726E656C206F6F7073004B65D5
:10923000726E656C2070616E696300556E6B6E6F47
:10924000776E206572726F7200756E6B6E6F776EDF
:109250000025633A203E3E3E205A45504859522050
:10926000464154414C204552524F522025643A20E9
:109270002573206F6E204350552025640A00256316
:109280003A204661756C7420647572696E67206956
:109290006E746572727570742068616E646C696E4C
:1092A000670A0A0025633A2043757272656E74205E
:1092B0007468726561643A20257020282573290A34
:1092C000006F730076322E342E39392D6E63733170
:1092D000002A2A2A20426F6F74696E67205A6570CF
:1092E000687972204F53206275696C642025732061
:1092F0002573202A2A2A0A00FFFFFFFFFFFFFFFF36
:10930000FFFFFFFFFFFFFFFFFFFFFFFFFFFFFFFF6D
:10931000FFFFFFFFFFFFFFFF29580000488200000A
:109320007C46012001000000904601200100000061
:10933000A446012001000000B84601200100000001
:10934000995F000000000000000000003E73012053
:1093500020000000000000000000000000000000ED
:109360005E730120200000000000000000000000EB
:1093700000C201000001030034450120000000008C
:10938000000000000000000000C201000001030016
:109390004845012000000000000000000090D003BC
:1093A000BB7A0000BF7A0000C17A0000555F000060
:1093B000A0450120A0450120000000006D4F0000E5
:1093C00028560120010000001D500000F94F000048
:1093D0003D500000D94F0000EC450120B045012070
:1093E000E445012000000000DC4501202C5601204E
:1093F0000100000030560120010000003456012019
:1094000001000000CC450120D8450120D0450120B5
:10941000C8450120FC450120218B0000008300008D
:10942000EC820000D84F01202C910000288400001D
:10943000D4830000744501201A8B000020840000B2
:10944000D48300005C450120418B00000000000037
:109450000000000000000000B2900000A88300009F
:10946000848300005C550120899100000000000009
:1094700000000000000000000D8600000000000059
:10948000B483000000000000000000007C460120C2
:109490007C4601200000000000000000FFFFFFFFED
:1094A00090460120904601200000000000000000CE
:1094B000FFFFFFFFA4460120A4460120000000009A
:1094C00000000000FFFFFFFFB8460120B846012062
:0C94D0000000000000000000FFFFFFFF94
:020000040001F9
:100000003DB8F3960000000000020000D8E90300AC
:1000100000000000000000000000000000000000E0
:10002000FFFFFFFFFFFFFFFFFFFFFFFFFFFFFFFFE0
:10003000FFFFFFFFFFFFFFFFFFFFFFFFFFFFFFFFD0
:10004000FFFFFFFFFFFFFFFFFFFFFFFFFFFFFFFFC0
:10005000FFFFFFFFFFFFFFFFFFFFFFFFFFFFFFFFB0
:10006000FFFFFFFFFFFFFFFFFFFFFFFFFFFFFFFFA0
:10007000FFFFFFFFFFFFFFFFFFFFFFFFFFFFFFFF90
:10008000FFFFFFFFFFFFFFFFFFFFFFFFFFFFFFFF80
:10009000FFFFFFFFFFFFFFFFFFFFFFFFFFFFFFFF70
:1000A000FFFFFFFFFFFFFFFFFFFFFFFFFFFFFFFF60
:1000B000FFFFFFFFFFFFFFFFFFFFFFFFFFFFFFFF50
:1000C000FFFFFFFFFFFFFFFFFFFFFFFFFFFFFFFF40
:1000D000FFFFFFFFFFFFFFFFFFFFFFFFFFFFFFFF30
:1000E000FFFFFFFFFFFFFFFFFFFFFFFFFFFFFFFF20
:1000F000FFFFFFFFFFFFFFFFFFFFFFFFFFFFFFFF10
:10010000FFFFFFFFFFFFFFFFFFFFFFFFFFFFFFFFFF
:10011000FFFFFFFFFFFFFFFFFFFFFFFFFFFFFFFFEF
:10012000FFFFFFFFFFFFFFFFFFFFFFFFFFFFFFFFDF
:10013000FFFFFFFFFFFFFFFFFFFFFFFFFFFFFFFFCF
:10014000FFFFFFFFFFFFFFFFFFFFFFFFFFFFFFFFBF
:10015000FFFFFFFFFFFFFFFFFFFFFFFFFFFFFFFFAF
:10016000FFFFFFFFFFFFFFFFFFFFFFFFFFFFFFFF9F
:10017000FFFFFFFFFFFFFFFFFFFFFFFFFFFFFFFF8F
:10018000FFFFFFFFFFFFFFFFFFFFFFFFFFFFFFFF7F
:10019000FFFFFFFFFFFFFFFFFFFFFFFFFFFFFFFF6F
:1001A000FFFFFFFFFFFFFFFFFFFFFFFFFFFFFFFF5F
:1001B000FFFFFFFFFFFFFFFFFFFFFFFFFFFFFFFF4F
:1001C000FFFFFFFFFFFFFFFFFFFFFFFFFFFFFFFF3F
:1001D000FFFFFFFFFFFFFFFFFFFFFFFFFFFFFFFF2F
:1001E000FFFFFFFFFFFFFFFFFFFFFFFFFFFFFFFF1F
:1001F000FFFFFFFFFFFFFFFFFFFFFFFFFFFFFFFF0F
:1002000088180020692501009F5B0100C9250100B5
:10021000C9250100C9250100C9250100C925010022
:100220000000000000000000000000007923010031
:10023000C92501000000000021230100C959010067
:100240002925010029250100292501002925010072
:100250002925010029250100292501002925010062
:100260002925010029250100292501002925010052
:100270002925010029250100292501002925010042
:100280002925010029250100292501002925010032
:100290002925010029250100292501002925010022
:1002A0002925010029250100292501002925010012
:1002B0002925010029250100292501002925010002
:1002C00029250100292501002925010029250100F2
:1002D00029250100292501002925010029250100E2
:1002E00029250100292501002925010029250100D2
:1002F00029250100292501002925010029250100C2
:1003000029250100292501002925010029250100B1
:1003100029250100292501002925010029250100A1
:100320002925010029250100292501002925010091
:100330002925010029250100292501002925010081
:10034000292501000000000000000000000000005E
:10035000000000000000000000000000000000009D
:10036000000000000000000000000000000000008D
:10037000000000000000000000000000000000007D
:10038000000000000000000000000000000000006D
:10039000000000000000000000000000000000005D
:1003A000000000000000000000000000000000004D
:1003B000000000000000000000000000000000003D
:1003C000000000000000000000000000000000002D
:1003D000000000000000000000000000000000001D
:1003E000000000000000000000000000000000000D
:1003F00000000000000000000000000000000000FD
:10040000DEE61E284CBBCE8F025B00003C000000E5
:10041000007E000001000000000201000002010057
:10042000FFFF02910000000000000000000000003B
:1004300000000000000000000000000053B94AB9AD
:10044000002908BF00281CBF4FF0FF314FF0FF30DC
:1004500000F070B9ADF1080C6DE904CE00F006F8BB
:10046000DDF804E0DDE9022304B070472DE9F04F28
:10047000099E04468946002B40F083808A42154637
:1004800045D9B2FA82F24AB1C2F1200701FA02F369
:100490009540944020FA07F747EA03094FEA154EC2
:1004A000230C1FFA85F8B9FBFEFC0EFB1C990CFB14
:1004B00008F143EA094399420AD9EB182CBF0120FD
:1004C0000020994202D9002800F01D810CF1FF3C68
:1004D000591AA3B2B1FBFEF00EFB101100FB08F895
:1004E00043EA0144A04505D92C1902D2A04500F2E7
:1004F0000E810138A4EB080440EA0C4000271EB12D
:10050000D4400023C6E900433946BDE8F08F002AF5
:1005100051D0B2FA82F2002A40F0AF80491B4FEA74
:10052000154E1FFA85F80127230CB1FBFEFC0EFBCC
:100530001C1108FB0CF043EA014398420AD9EB185E
:100540002CBF01210021984202D9002900F0D78058
:100550000CF1FF3C191AA3B2B1FBFEF00EFB101117
:1005600008FB00F843EA0144A04505D92C1902D242
:10057000A04500F2C1800138A4EB080440EA0C4019
:10058000BDE78B4208D9002E74D00027C6E90001D0
:1005900038463946BDE8F08FB3FA83F767B98B4226
:1005A000C0F0A480824240F2A1803846002EABD039
:1005B000C6E90049A8E7FFDEC7F12005BB4002FA03
:1005C00007FC01FA07F4EA4020FA05F8E94000FACE
:1005D00007FE1A4348EA04044FEA1248200C1FFAA7
:1005E00082F9B1FBF8FA08FB1A110AFB09FB40EA91
:1005F00001418B450AD951182CBF012300238B459B
:1006000002D9002B00F088800AF1FF3AA1EB0B0120
:10061000A4B2B1FBF8F008FB101100FB09F944EAA1
:100620000141894504D9511801D289457BD8013847
:1006300040EA0A40A1EB0901A0FB0C894945444668
:100640004B4602D306D1C64504D20138B8EB0C04A0
:1006500069EB0203002E5DD0BEEB040261EB0301E7
:1006600001FA05F522FA07F3F94000271D43C6E910
:10067000005149E73746304646E7C2F12000954031
:1006800001FA02F721FA00F34FEA154E24FA00F1BD
:100690001FFA85F894403943B3FBFEF00F0C0EFBB4
:1006A000103300FB08FC47EA03439C4507D9EB18CD
:1006B0002CBF012700279C4500D98FB30138A3EB3D
:1006C0000C0389B2B3FBFEF70EFB173307FB08FCE4
:1006D00041EA03418C4504D9691801D28C4525D8DB
:1006E000013FA1EB0C0147EA00471DE7841A61EBCB
:1006F00003030120994659E702382C443CE7ACF14A
:10070000020C2B4426E7ACF1020C2B44E0E6023845
:100710002C44EFE63746F7E6AAF1020A114475E7E2
:1007200002382B44CBE70238114481E7023F2944C9
:10073000D7E700BF704700BF2DE9E04F2746A0462E
:10074000A146A246A346A4462DED108B4FF000050E
:1007500045EC185B45EC195A45EC1A5A45EC1B5A06
:1007600045EC1C5A45EC1D5A45EC1E5A45EC1F5AE7
:10077000F1EE105A4FF66076C0F6FF763540E1EEA6
:10078000105A84F3008825462646A447BDEC108BFA
:10079000BDE8E08F0B6801330B60014B1B68184705
:1007A00000000020014B1860704700BF00000020CF
:1007B000002307B50246019303480B4601A900F048
:1007C000E3F803B05DF804FB950701002DE9F84F4D
:1007D000B0F81890044619F008080DD001290CBF94
:1007E00049F0100949F02009A0F8189082F3118807
:1007F000BFF36F8FBDE8F88F09F00709022907D111
:10080000204604F01FFE0028F0D00128238B4AD197
:100810006769238B002F15DA2568C4E9008823F067
:10082000070343F0010323830026238B03F0070A09
:10083000CA4502D0A168002956D10DB9002E6DD04D
:10084000002152E003F00701481F01281CD823F0C3
:100850000703062925689BB2C4E900880AD13DB187
:100860002846618B0068013189B20028FAD1618382
:1008700043F002032383204604F0E4FD0028D3D094
:10088000238B43F02003CEE704290AD123F007038A
:1008900099B22183204604F0D5FD10B141F020012A
:1008A00021830025C0E7032809D1216923F007032C
:1008B0000E6843F00603002523832F46B5E704287E
:1008C00006D1216923F007034E6843F00403F2E7E1
:1008D000052806D1216923F007038E6843F005033C
:1008E000E9E700252E46E8E7012143F008032383CA
:1008F00082F31188BFF36F8FF9B985BB16B1214917
:100900002046B0474FF02003EFF3118283F31188A4
:10091000BFF36F8F238B23F008032383238BD90628
:1009200027D5012123F010032383B4F8189009F090
:10093000070900297FF462AF58E7A1680029DCD0DD
:10094000D1F80090D1F804B03B4652462046D84733
:10095000B9F1000FD1D04946D9F80090F2E7D5F8A7
:10096000009029463B465246204604F087FD4D46FE
:10097000C3E713F020011EBF23F0200323830221CD
:10098000D3E700BFA95401002DE9F04F0D46924670
:1009900098460024A3B004909AF8000010B92046AD
:1009A00000F0A6BD0AF1010325280C930BD02946BF
:1009B000049B98470028C0F29B8546460134B04608
:1009C000DDF830A0E8E71822002114A805F088F926
:1009D0009AF80130252B7CD000239E4618461F46EE
:1009E0009B461E469946DDF830C005930C93614640
:1009F0001CF8012B2B2A00F08F8000F28580202A22
:100A000000F08D80232A00F08D802EB19DF8586073
:100A100069F382068DF858600C9E2EB19DF85860DF
:100A200046F008068DF858602FB19DF858606BF3BA
:100A300004168DF8586030B19DF85800059E66F395
:100A400045108DF858002BB19DF858306EF3861381
:100A50008DF858309DF8583003F04400442803D1F5
:100A60006FF386138DF858309DF858302A2A43F0DA
:100A700080038DF8583071D19DF859204B1C42F0FD
:100A800001028DF859201A782E2A0CBF012100216D
:100A90009DF8592061F341028DF859206AD15A78A6
:100AA0002A2A60D000220A270133194611F8010BC7
:100AB000A0F13006092E40F284809DF8581018925B
:100AC000C1F3400040EAD27262F341018DF8581040
:100AD00050E00AF102020C928DF85B309DF859301B
:100AE000D80740F13081464656F8042B002A05927B
:100AF00080F230819DF8582042F004028DF8582091
:100B0000059A5242059225E12D2A0ED0302A7FF413
:100B10007CAF01239E466AE701220C9267E701271A
:100B2000BB4664E70120059061E70126B1465EE718
:100B300033460CFB0202303A1E4616F8010BA0F1B8
:100B40003007092FF4D999429DD09DF8581017927B
:100B5000D20F62F341018DF8581094E70B46002242
:100B60004FF00A0CE8E79DF85920023342F00402E6
:100B70008DF859209C461CF8012B6A2A4AD025D8AA
:100B80004C2A53D0682A2ED09C46624612F8013B6C
:100B9000672B0C928DF85B3079D8652B58D2582B87
:100BA00000F0AA804FD8412B52D003D3A3F14502C5
:100BB000022A4DD99DF8583043F001038DF8583082
:100BC00082E007FB02020B46303A6EE7742A29D016
:100BD0007A2A23D06C2AD7D15A786C2A9DF85920CA
:100BE00015D1042105E05A78682A9DF8592007D1CB
:100BF000012161F3C6028DF8592003F1020CC4E70C
:100C00001346022262F3C6038DF85930BDE713463E
:100C10000322F7E79DF859300522F3E79DF8593094
:100C20000622EFE79DF859300722EBE7BDF8583070
:100C300023F4F04323F0020343F4804343F0020320
:100C4000ADF85830A1E7632B56D028D8612BB1D12D
:100C500004219DF85A2003F0DF0361F30202A3F19F
:100C600041077B428DF85A209DF859207B4163F360
:100C7000C712D3B28DF859201A0662D403F0780255
:100C8000182A4AD16FF3C6038DF859301CE0702B37
:100C900023D01BD86E2B44D02ED8692B8AD10121AA
:100CA0009DF85A2061F302028DF85A209DF85920D0
:100CB00002F07802402A02BF9DF8581041F001016D
:100CC0008DF85810632B1BD000231CE0752B13D01C
:100CD000782B11D0732B7FF46DAF03229DF85A301F
:100CE00062F302038DF85A309DF8593013F0780FF3
:100CF00014BF0123002306E09DF85A200221D1E70A
:100D0000131C18BF01239DF85820C2F340010B4368
:100D100063F341028DF85820E0E613F0380FD3D08A
:100D200048E703229DF85A3062F302038DF85A30E7
:100D30009DF8593003F07803A3F1400673427341E4
:100D4000E1E70123DFE79DF95820002A14DA46463F
:100D5000179A0592590713D5334653F8048BB8F107
:100D6000000F38DA1E469DF859206FF341028DF8C6
:100D700059204FF0FF3807E046464FF0FF32C1E6FA
:100D80009A07F6D5DDF860800023CDE917339DF88A
:100D90005A3003F00703042B0BD19DF859309B0701
:100DA00007D49DF95930002BB4BF4FF00D084FF018
:100DB00006089DF85A309DF8592003F00703012BCF
:100DC000C2F3C3023ED1D31E042B14D8DFE803F0D4
:100DD000050D0D1313001E46D6E7334653F8040BDA
:100DE000C117CDE914011E461CE0073626F00703A3
:100DF000F3E80201F5E7334653F8040B012A4FEA02
:100E0000E071CDE914011E4605D19DF850301493D0
:100E10000023159306E0022A04D1BDF95000C11742
:100E2000CDE914019DF8580010F003073ED00C9B4B
:100E300052462946049804F019FD0028C0F2588350
:100E40000444BCE5022B20D1D31E042B0ED8DFE8CE
:100E500003F00309090D0D0000213068331D1490C3
:100E60001591C0E7F31D23F00703C1E7334653F89C
:100E7000041B012A14914FF000011E461591C4D0A5
:100E8000022ACFD1BDF85030C1E7042B07D1F31DA2
:100E900023F00706F6E80201CDE91401C2E7032BAF
:100EA000C0D1334653F8041B14919CE79DF85B9026
:100EB000B9F1670F00F21F81B9F1650F0ED2B9F1D8
:100EC000470F00F2D880B9F1450F07D2B9F1250FCD
:100ED00000F03681B9F1410F7FF471ADDDE91423E3
:100EE000002A73F10001C0F2A281010700F1A18183
:100EF00010F0100718BF2027C3F30A5AC3F31303D7
:100F000006920793DDE90623CDE91023BAF1000F1D
:100F100040F09181DDE90632134314BF4FF0010C1C
:100F20004FF0000C50460799B9F1460F4FEAC12324
:100F3000069908BF4FF06609CA0243EA51534AEACC
:100F400002010A91C11719430B91DDE90A0101431E
:100F5000CDE9102300F0E281BCF1000F40F0A28146
:100F6000109B4FF0050E0293119BAAF2FE3A43F03C
:100F700000430393DDE90223CDE9102300231A4641
:100F80001AF1020FC0F298811BB1DDE90201CDE92F
:100F90001001DDE91031BAF1000F00F3A781CAF1A9
:100FA000040A1199109BCAF1200C01FA0CFCAAF159
:100FB000200023FA0AF321FA00F043EA0C0303436A
:100FC00021FA0AF1CDE9103109F0DF03472B40F097
:100FD000AD81D31C02DB904580F2A381A9F1020907
:100FE000B8F1000F5FFA89F901DD08F1FF389DF8CB
:100FF0005830980600F19A81B8F1000FD4BF4FF035
:10100000000A4FF0010AB9F1660F4FF0100340F0EB
:10101000908112EB080B40F18E814FF0000B0F9383
:1010200000204FF00061CDE91201DDE912300BF133
:10103000FF3BBBF1FF3F40F0858110995B1808939F
:10104000119B40EB03030993DDE90801B1F1805FD7
:1010500008BF002880F08281CDE91001B9F1660F48
:1010600040F00082002A00F3888130230DF16D0BDF
:101070008DF86C3092E1B9F1610F3FF42FAF20D8B9
:10108000B9F1580F7FF49BACDDE914010DF1850334
:10109000009316AA1BAB04F09CFB8146B8F1000F2D
:1010A0000DF1850B48DB9DF85820ABEB09036FF37E
:1010B000861298458DF858203ED9A8EB0303179364
:1010C0003AE0B9F1630F48D0B9F1640F7FF477AC1F
:1010D000070779D410F0100718BF2027DDE9142383
:1010E000002A73F10001CFDA524263EB4303CDE9EA
:1010F00014232D27C8E7B9F1700F67D006D8B9F1CE
:101100006E0F7BD0C0D8B9F1690FDFE7B9F1750F69
:10111000BAD0B9F1780FB7D0B9F1730F7FF44FACF3
:10112000B8F1000FDDF8509013DB4146484604F05B
:1011300071FD002709EB000BB9F1000F14D13EE45B
:1011400029464846049B98470028C0F2D1810134C3
:1011500035E4484604F057FDEBE7149B0DF16D0BA9
:101160008DF86C300DF16C09ABEB090A0FB10AF187
:10117000010A9DF85A30D80640F1AE810AF1020A00
:10118000179A92445A0644BF189B9A44059B002B19
:1011900040F3BB81A3EB0A0A9DF85830C3F38008E3
:1011A000B8F1000F40F0EF815B0640F1A48147B138
:1011B00029463846049B98470028C0F29981474643
:1011C00001344FF0300898E12B2787E71498002866
:1011D00000F07C810DF18503009316AA1BAB394604
:1011E00004F0F7FABDF85A30814603F0EF0343F4F8
:1011F000F04343F01003ADF85A304FE7149B072A31
:101200003FF6DDABDFE802F0100407100A0A101009
:101210001C70FFF7D4BB1C80FFF7D1BB2046E11741
:10122000C3E90001FFF7CBBB1C60FFF7C8BB2D274C
:1012300062E62B2760E640F2FF739A452DD1DDE987
:1012400006231343A9F1410918D1B9F1190F95BF2C
:1012500044F6496346F66963ADF86C30ADF86C301E
:1012600094BF462366238DF86E309DF858300DF1FB
:101270006F0B6FF386138DF8583073E7B9F1190FC0
:1012800095BF44F24E1346F26E13ADF86C30ADF8D4
:101290006C3094BF4E236E23E5E74FF0000C41E61F
:1012A0000AF1FF3A92185B41002A73F10001F7DA64
:1012B000CDE9102354E6E246029B03995B08B3484C
:1012C00043EAC173490881420AF1010CCDE90231B8
:1012D000F1D8A3FB0EBCCDE902BC039B0AF1020AC4
:1012E0000EFB0133013A0393012349E6023341F136
:1012F000000110A80D92CDE9103104F034FADDE9B7
:1013000010010D9A0AF1FF3A0132001849410028F4
:1013100071F100030AF1FF3AF7DA38E6002292464B
:101320003DE6A8EB02084FF0660960E64FF0000AC0
:1013300069E608F1010BBBF1100F0F93A8BF4FF046
:10134000100B6DE65B0843EAC0734008CDE912302C
:1013500012A80D9204F007FA0D9A66E6089B0D920A
:10136000099A5B0843EAC273510810A8CDE910310D
:1013700004F0F9F90D9A013270E60DF16C0B0F9B38
:10138000002B09DD0FA910A80D9204F00BFA0D9A9D
:101390000BF8010B013AF2D1179200229DF8583058
:1013A000990602D4B8F1000F1DDD2E230BF8013B86
:1013B0009AB1B8F1000F16DD51424145A8BF414630
:1013C00000291791A8EB0108D4BF002101219DF845
:1013D0005A3061F345138DF85A30B8F1000F02DD31
:1013E0000F9B002B57DCBAF1000F62D1CDF8608063
:1013F00009F0DF03452B23D1002AB4BF2D232B2373
:101400005946B8BF5242632A01F8029B8BF801305B
:101410000ADD642092FBF0F300FB132203F1300C91
:101420000BF103018BF802C00A2092FBF0F38B460C
:1014300000FB132203F1300C30320BF802CB4A7060
:10144000179B002B40DC189B002BD4BF00230123EB
:101450009DF85A2063F3861200238DF85A208BF8EA
:1014600000307FE60FA910A80D9204F09BF90D9AA9
:101470009DF85830302818BF02F1FF329B068DF8D6
:101480006C0002D4B8F1000F10DD2E230DF16E0BAD
:101490008DF86D30A1E70FA910A80D9204F082F924
:1014A00008F1FF380BF8010B0D9A96E70DF16D0B63
:1014B00099E7002318935B461BF8011D3029FAD0E9
:1014C0002E2918BF9B4693E70123C1E7DFF8C0B080
:1014D0000746ABF1050947E6190748BF0AF1010ABB
:1014E0004EE6049B2946404698470028059B06DAAD
:1014F00023B0BDE8F08F4FF020085346A2445A1E97
:10150000002BAAEB03040592EBDC37B129463846E1
:10151000049B98470028EBDB01349DF85A305F06A6
:1015200040F194809DF95930002B33DBA4EB090482
:1015300099F800004F46A0F13003092B04EB09088D
:1015400009F1010954D99DF85A30DDF85C909806EC
:1015500008D44B4609EB080A002BAAEB030803F159
:10156000FF394BDC38782E280AD12946049B98474E
:101570000028BDDBB9F1000F08F1010846DC013796
:10158000A8EB07084FE0CDF814A0BEE732333333A1
:10159000F5650100A4EB0908CA4608EB090419F82F
:1015A000010B70281ED1189B03EB0408A8EB040361
:1015B000002B42DC5B4652462946049804F056F95B
:1015C000002895DB059B044423441F463B1B002B4E
:1015D0007FF7F5A929462020049B9847002887DB40
:1015E0000134F3E72946049B98470028D4DA7FE7C3
:1015F0002946049B984700289ADA79E7049B2946F4
:101600003020984700284B46A6DA71E7294630205B
:10161000049B984709F1FF39AAE72946049B98479C
:101620000028FFF665AFBA4608EB070417F8010B70
:10163000A0F13003092BF0D9B5E729463020049BEF
:1016400098470028FFF654AF0134AFE7D90601D41C
:101650001A0707D529463020049B98470028FFF633
:1016600047AF01349DF85A30DB0608D529469DF86E
:101670005B00049B98470028FFF63AAF0134179BA4
:1016800003EB0408A8EB0403002B02DC5B464A468C
:1016900092E729463020049B98470028FFF628AFA0
:1016A0000134EFE74FF02002EFF3118382F311884A
:1016B000BFF36F8F0121044AC2F8401583F31188EC
:1016C000BFF36F8F002070470090035020B1034B91
:1016D000800143F001031847704700BF40630100D9
:1016E00008B504464FF02002EFF3118382F311880E
:1016F000BFF36F8F04F06AF9204601F087F80348C2
:1017000003F093FE00F0BEFEFCE700BFF6650100AB
:1017100010B5074801F0D4FE064C074B1860204670
:1017200001F0CAFA2046FFF73DF8002010BD00BFC7
:101730001F6601003D170100680200200A2838B525
:101740000446074D04D1286883680D215B689847DB
:1017500028688368E1B25B689847204638BD00BFBF
:10176000680200200E4A70B5841A05460C200E4609
:101770004021A3100B4C5C43E4B200FB042008445E
:1017800004F096F8011E05DB074B03EBC404636805
:101790009847002128463346BDE87040184700BFEF
:1017A0007C020020B76DDBB65C6301002DE9F041DF
:1017B0000C25104E8046841BA3100F4C0F465C4333
:1017C000E4B2654305F140004021304404F089F85B
:1017D000011E09DB094A7319C3E90E27084B53F8A8
:1017E0003430BDE8F041184740463B46BDE8F04183
:1017F000184700BF7C020020B76DDBB645590100D9
:101800005C63010070B5002201210446052000F050
:10181000E1FD052000F0C0FD0F4801F03DFD0F4B3C
:10182000984215D104F0E3FAE6680D49304603F01A
:1018300059FE00280BDB01253564E468084904F1F2
:101840001C0003F04FFE002801DB0020E56470BDA2
:101850006FF00400FBE700BFFD1801000000AD0BB6
:101860006C63010001460C2300224B43084870B50D
:10187000C4184033D4E90E561844A26304F04FF85C
:101880002DB132462B46BDE870400248184770BD66
:101890007C020020BC00002008B54FF02003EFF3CD
:1018A000118183F31188BFF36F8F124A136843F0DD
:1018B000020013F0010310600CD04FF05022D2F858
:1018C0000C34D2F80C2413F0010303D00A4804F0BE
:1018D00026F8012381F31188BFF36F8F23B1BDE890
:1018E00008400020FFF7BEBF0120BDE8084001F01E
:1018F000E3BC00BFCC020020BC02002010B10128D4
:1019000004D07047034B1B6C5B0701D1FFF7AABFE4
:10191000704700BF7C020020074BD3E8EF2F22F076
:101920000201C3E8E01F0028F7D1D30702D4012049
:1019300001F0F4BC704700BFCC0200201FB50022AC
:101940000123CDE902236B46084ACDF800D0CDF83B
:1019500004D004F01EF8002805DB4FF48042002379
:10196000684602F0A1FB05B05DF804FB6559010073
:101970002DE9F843012205463849D1E8EF3FC1E897
:10198000E02F0028F9D133B9354936484B60CB6098
:101990008A6003F0BAFD6B1E012B30D8012D07D1F0
:1019A0004FF05023D3F81C3403F00303022B26D04E
:1019B00004F00DFB18B92C4B1B78002B46D14FF0CF
:1019C0002003EFF3118983F31188BFF36F8F012494
:1019D000264E274FDFF89C804FF05022D2F8183463
:1019E000D2F81824D2030CD503F00303022B01D044
:1019F000012D06D124B389F31188BFF36F8FBDE8A1
:101A0000F883C4B1484600F04BFD4FF05022D2F8A5
:101A10001835DBB2012BDFD131680029DCD0002181
:101A2000316031680221C2F818152022C7F88021E0
:101A3000C8F80030D0E70021212002F0EDFAE4E7F9
:101A40004FF050230222C3F80423D8E74FF050236D
:101A500002220446C3F808238146B9E7D0020020D9
:101A60006C020020980200208108002004510050E0
:101A700000E100E008500050044A1368C91A21F040
:101A80007F400344136002F0DFBC00BFE00200208F
:101A90002DE9F0474FF48037850000F1500405F13F
:101AA0005025A40005F58035A4B204F15024D5F8E2
:101AB0004025DFF86C80DFF86C9021F07F4604F55C
:101AC00080348740D8F804A5A2EB0A0222F07F42B6
:101AD0002AF07F43012AC5F8403502D1132004F0D3
:101AE0007CFA0AF10202B31A23F07F434B4528BF68
:101AF000164600232360236826F07F43C8F844730A
:101B0000C5F84035D8F804359A4507D0F31A023B9A
:101B100023F07F43B3F5000F3246D3D8BDE8F087FA
:101B20000050015001008000F8B5002427460F4EF8
:101B30000F4B104A1D68184604B1F8BDD2F80413C3
:101B4000C903FAD531680029F7D0346031684FF401
:101B50008031C2F84813D2F84015012425B11F6026
:101B60005A680020A847E3E70560E6E740510150C6
:101B7000D40200200050015038B500244FF48033C7
:101B80004FF400120D4D0121C5F80845C5F8043386
:101B90000B4B1520C3F88021224600F01BFC1520BA
:101BA00000F0FAFB0123074A02201360064A2B606B
:101BB0001360FFF7DDFE204638BD00BF0050015026
:101BC00000E100E008500150DC020020134BB0F1AE
:101BD000FF3F08BF1846013800281CDD9842A8BF07
:101BE00018460F4BD3F804250E4B1968521A12F4FD
:101BF000000F18BF002022F07F4301330A4A03443C
:101C00000A48106000205060044A934294BFC918EB
:101C10008918FFF73DBF0020E3E700BFFFFF7F000B
:101C200000500150E0020020D4020020791A010087
:101C30004FF02002EFF3118382F31188BFF36F8F0F
:101C4000064AD2F80405064A1268801A20F07F403E
:101C500083F31188BFF36F8F704700BF00500150AE
:101C6000E0020020F7B500281C4614BF4FF40053D3
:101C70004FF400438A4241D90D46214F00283AD003
:101C800005F5E07647F826406E1CB24231D15A4342
:101C90001C4800924B432A4603F0C7FB1A4B14F032
:101CA000100F1A491A4808BF194603F0BEFB14F07A
:101CB000040F14BF72212D21164803F0B6FB14F057
:101CC000020F14BF77212D21124803F0AEFB14F050
:101CD000010F0CBF2D2178210E4803F0A6FB6C21CB
:101CE0000C4803F0A2FB0C4803B0BDE8F04003F041
:101CF0009CBB3546C2E705F5C076C3E703B0F0BD2F
:101D00000030005045660100396601003066010070
:101D10004F6701005F6601009A69010008B543B290
:101D2000002B0CDB012200F01F018A405B091049E7
:101D3000203341F82320BFF34F8FBFF36F8F830011
:101D400003F1A04303F540533128D3F8002806D00F
:101D5000002A07DA02F00302023A012A02D8054AF1
:101D6000C3F80028012103F0E2FE002008BD00BFF7
:101D700000E100E00001008030B54FF4E13485B0AF
:101D80002E4D4FF4E1312E4803F04FFB21682D48D2
:101D900003F04BFB29682C4803F047FB102200217D
:101DA000684603F09DFF236868460093029400F0A4
:101DB0000DFF012000F03AFF002000F023FF00207B
:101DC00000F048FF0121002000F062FF00F056FF04
:101DD0002C681E4803F029FB0820FFF79FFF24F022
:101DE0000104BFF34F8FBFF36F8F64086400204678
:101DF000214622462346B7EE000AF7EE000AB7EE68
:101E0000001AF7EE001AB7EE002AF7EE002AB7EE36
:101E1000003AF7EE003AB7EE004AF7EE004AB7EEA6
:101E2000005AF7EE005AB7EE006AF7EE006AB7EE16
:101E3000007AF7EE007AFEF77FFC00BF04C20100D3
:101E4000666701007D67010092670100B0670100CD
:101E50002DE9F8433B4803F0E8FA002140F217135C
:101E600008460322FFF7FEFE40F20713202203215B
:101E70000020FFF7F7FE344803F0D7FA334B344A1B
:101E8000C3F3C431C3F30E03C3F50043C3F34313D9
:101E9000C2F80015C2F80435D2F80015D2F80425AE
:101EA0002C48520103F0C1FA274803F0BEFA03F0B0
:101EB0008EFD014610B1284803F0B7FA00242748E8
:101EC00003F0B3FA40F21713082200210120FFF7B4
:101ED000C9FE1F4D40F20713202208210120FFF701
:101EE000C1FE194803F0A1FAC5F880441C4803F06C
:101EF0009CFA1C4FC5F8C044DFF87C801A4DDFF80F
:101F00007C906E792A68002E14BF3B4643462146DA
:101F1000484603F08AFA66B91448013403F085FA9A
:101F20001A2C05F10805ECD10748BDE8F84303F089
:101F30007CBA2879FFF7F2FE08B10D48EDE70D48AD
:101F4000EBE700BF6D6601009A690100E07F0100C8
:101F50000030005091660100D7660100076701005C
:101F60002967010062660100786301005267010081
:101F700059670100616701003D6601004567010086
:101F80002DE9F0438146002685B0DFF838800C4FFC
:101F900001AD58F8044B97E807004C4485E807006A
:101FA0000C222946204603F04AFE00B91CB901362E
:101FB000052EEED10024204605B0BDE8F08300BF19
:101FC000F06201004864010070B50C4615460646F3
:101FD000B0BB6FF01500BDE87040714672467346A5
:101FE000B7EE000AF7EE000AB7EE001AF7EE001A95
:101FF000B7EE002AF7EE002AB7EE003AF7EE003A05
:10200000B7EE004AF7EE004AB7EE005AF7EE005A74
:10201000B7EE006AF7EE006AB7EE007AF7EE007AE4
:102020008EF3008C10B4F1EE10CA4FF66074C0F657
:10203000FF740CEA040CE1EE10CA10BCF4467447BD
:10204000002AC6D003F0DAFD0128C2D0B4F5803FE3
:1020500017D32B19B3F5813F06D90B4A94420AD9FD
:1020600002F61D22934209D82A462146304603F043
:102070000DFE0020AFE7054A944202D9044A93427C
:10208000F2D94FF0FF30A6E70302FF002F01FF0057
:102090003801FF0070B5054610460E46144603F0A1
:1020A000ADFD012837D16FF01503BDE8704018462B
:1020B000714672467346B7EE000AF7EE000AB7EEB5
:1020C000001AF7EE001AB7EE002AF7EE002AB7EE74
:1020D000003AF7EE003AB7EE004AF7EE004AB7EEE4
:1020E000005AF7EE005AB7EE006AF7EE006AB7EE54
:1020F000007AF7EE007A8EF3008C10B4F1EE10CA7D
:102100004FF66074C0F6FF740CEA040CE1EE10CADE
:1021100010BCF44674472846FFF732FF05463046A8
:10212000FFF72EFFCDB12A6A0E4B9A4215D148B166
:102130000123016A0B4A914202D13BB92370B4E7F3
:10214000002BB0D0012323700023AEE76B694269F6
:10215000934234BF00230123F5E70028A3D00023D6
:10216000E7E700BFFFFF0291014802F023BC00BF78
:102170005C64010008B5B0B14368042B0DD10022A6
:102180000368D3E8EF1F012903D1C3E8E02F00283B
:10219000F7D1074808BF104608BD3BB1006801F001
:1021A00087FB0020F8E76FF4E040F5E70148F3E72C
:1021B000E98FFFFFEA8FFFFF10B5044618B90D4BFA
:1021C0000D485B689847616808290DD031F0040319
:1021D0000AD011F0020108D02146084801F0C6FAE1
:1021E000002323600023636010BD1422206803F0E5
:1021F00077FDF7E770000020D7680100E4020020B7
:1022000010B5044618B9164B16485B6898476368C2
:10221000042B23D0082B21D0CBB92368BBB94FF0B6
:10222000FF324FF0FF3321460F4801F06DFA08B935
:1022300023681BB90A4B0D485B689847142200219C
:10224000206803F04DFD636843F00203636020687B
:1022500003F010FE636843F00103636010BD00BF2C
:1022600070000020D7680100E4020020FD68010032
:1022700008B5D8B14368042B0CD101220368D3E818
:10228000EF1F002903D1C3E8E02F0028F7D10BD1BD
:10229000002008BD6BB100684FF0FF324FF0FF33F4
:1022A00001F08EFA0028F3D00348F2E76FF4E04023
:1022B000EFE70248EDE700BFE98FFFFFEA8FFFFF7E
:1022C00008B5064940231422054803F0B8FDBDE8CF
:1022D00008400449044802F0BFBB00BF00030020CF
:1022E000E40200207464010064640100094A0A49A0
:1022F000936809689867D96708494B6843F0805329
:102300004B60002383F31188BFF36F8F9368D86FFE
:10231000704700BF20080020F464010000ED00E0D9
:1023200013498A684FF038001044EFF3098C80E8B5
:10233000F01F202080F31188BFF36F8F0D4F4FF0F7
:1023400000668A6A8A603E60906F0023936780F31C
:10235000118802F1380090E8F01F8CF3098802F12F
:10236000000004B503F011FCBDE804407047000014
:102370002008002004ED00E01EF0040F0CBFEFF376
:102380000880EFF30980816911F8021C0229FFD04F
:1023900001B503F000FC01BD43B2002B08DB0122B4
:1023A00000F01F0002FA00F0024A5B0942F8230025
:1023B000704700BF00E100E0054B420953F82220BE
:1023C000012300F01F0003FA00F01040704700BF27
:1023D00000E100E043B2002B01F10101A8BF03F1CD
:1023E00060434FEA4111B8BF054BC9B2ABBF03F51B
:1023F000614300F00F0083F800131954704700BFC9
:1024000014ED00E042F8203C009B0B4942F81C3CD4
:10241000019B21F0010142F8183C029B42F8081C84
:1024200042F8143C4FF0807342F8043C0023203AF9
:1024300082658367704700BF9D55010008B504465B
:102440000E4615460023E1EE103A00F055FA094B0E
:102450009C60A36E83F30B88284686F309880021CD
:1024600063B681F31188BFF36F8F0022002303F05E
:1024700095F800BF20080020014910220A6070472B
:1024800010ED00E072B6404080F31188BFF36F8F0B
:10249000BFF34F8F30BF62B6BFF36F8F704700BF7F
:1024A00072B6494081F3118820BF80F3118862B66B
:1024B000704700BF30BFFFF7FDBF00BF174A08B528
:1024C000174B22F07F029A60BFF34F8FBFF36F8FDD
:1024D000D3F8882022F47002C3F88820D3F888202B
:1024E00042F4A002C3F888200E4A536823F0404308
:1024F0005360BFF34F8FBFF36F8F0023E1EE103AAD
:10250000EFF3148323F0040383F3148801F030F80D
:1025100001F0A0FE00F0C2F901F04EF80002010047
:1025200000ED00E030EF00E001B572B60B4A506AF2
:1025300000281EBF0021516203F07FFC62B6EFF35A
:102540000580A0F110004FEAC0000549014409C907
:102550009847BDE8014003490847000020080020D3
:10256000E0600100F1270100002080F31488BFF330
:102570006F8F002080F30A8880F30B8803F08DF9B9
:1025800000200E490860BFF34F8F0D4880F3088884
:1025900000F05EF9202080F311880A484FF40061B2
:1025A000401880F30988EFF314800221084380F378
:1025B0001488BFF36F8FFFF781FF000094ED00E0F8
:1025C00088180020C8190020EFF30880EFF3098174
:1025D00001B5724600F074F801BD00BF0E4B9A6A57
:1025E0009A6A9A6A920708D55A6B9A6A120604D5B3
:1025F00018B19A6A22F080029A620020064B9A6A09
:102600009A6A9A6AD20658BF9A6A9A6A42F0FF0298
:102610009A620870704700BF00ED00E00D4B9A6AA7
:102620009A6A9A6A920508D59A6B9A6A120404D536
:1026300018B19A6A22F400429A620020054B9A6A05
:102640009A6AD20558BF9A6A9A6A42F47F429A629D
:102650000870704700ED00E0094B9A6A9A6A986A20
:102660009A6A9A6A9A6A9A6A9A6A10F480106FEA69
:1026700002426FEA124218BF02209A62704700BFFE
:1026800000ED00E00D4B9A695A695A69D0070FD4E2
:102690005A6991070CD45A69520709D45A6910072C
:1026A00006D45A69D10603D45A69920658BF5A69AA
:1026B0005A6942F0FF025A61704700BFD0ED00E056
:1026C000F0B5414B8BB05B680025C3F3080385F37D
:1026D0001188BFF36F8F02F07F44B4F17F4F1ED19A
:1026E00012F001041AD0560602F0080467D482F0F2
:1026F0000402C2F3800564B1EFF389860022033B34
:102700008DF80720042B4BD8DFE803F00B4C504129
:102710004800EFF38886F1E70E46EFE725462E46A0
:10272000ECE7294BDA6A92073AD4DC6A14F0804469
:1027300008D028331B78EBB101200DF10701FFF71A
:102740004DFF04469DF8073093B92022314602A878
:1027500003F09CFA099B6DB3C3F3080222B96FEA38
:1027600053236FEA4323099302A9204603F011FA89
:102770000BB0F0BD154B1B782BB101200DF10701FB
:10278000FFF74CFFDDE7124B1F88BFB217B1FFF711
:1027900063FFD6E70F4B5C69002CD3D0FFF772FFC5
:1027A0000024CFE70DF107010020C8E70DF1070174
:1027B0000020E5E723F4FF7323F00103D3E7002CA7
:1027C000AAD10646012599E700ED00E029ED00E0D9
:1027D0002AED00E0D0ED00E0044B5A6942F010020F
:1027E0005A615A6942F480625A61704700ED00E014
:1027F000044B9968986A884203D003494FF080528D
:102800000A6070472008002004ED00E0BFF34F8FFE
:102810000549064BCA6802F4E0621343CB60BFF37C
:102820004F8F00BFFDE700BF00ED00E00400FA0598
:1028300000231846054A1168C1F307218B4200D1D5
:102840007047936010610133F8E700BF90ED00E03E
:1028500010B572B6002484F31388FFF7E9FF0E4A1F
:10286000234611464FF0FF3403F120000133102BB3
:1028700042F82040F8D100234FF0FF3003F160020E
:102880000133102B41F82200F8D162B6BFF34F8F0D
:10289000BFF36F8F10BD00BF00E100E000232021D7
:1028A0000348C2180133412B82F80013F9D1704755
:1028B00000E100E008B50E4B9B68834207D1EFF3BF
:1028C000058393B10B4A536843F08053536001F082
:1028D000F5F94FF02003EFF3118083F31188BFF374
:1028E0006F8FBDE8084003F0CCBA01F093FC00BF45
:1028F0002008002000ED00E01FB5094C094A2346DE
:102900000121094800F004F900230393074B01213A
:10291000E41A01A80193029400F004F904B010BD78
:1029200000000120000000208864010060010020F8
:1029300010B50B680C7A23F01F0204F01F031A4332
:10294000CB68640923F01F03044943EA440343F0BE
:1029500001038860CA600B6110BD00BF90ED00E00C
:102960002DE9F04F88461446814600274B4D85B02F
:10297000474506DAD9F80460BEB31F2E05D86FF0BC
:102980001504204605B0BDE8F08FF306F7D1D9F85D
:1029900000A01AF01F0FF2D1504603F026F983462B
:1029A00006EB0A00013803F020F98345E7D11BF15B
:1029B000160FE4D0631E5B45E1DBC5F808B0E9689B
:1029C000C5F808B02E6921F01F01D9E900321A4478
:1029D000994246F01F0602F1FF3A1CD1564508D134
:1029E00049465FFA8BF003F0E1F8013709F10C0971
:1029F000BEE74946C5F808B0EB6822F01F0203F0B5
:102A00001F031A43EA60E0B203F0D0F810F1160F8A
:102A1000B5D0441CE9E7013B5645E0B223F01F0363
:102A2000C5F808B006D12A69494602F01F021343CF
:102A30002B61E9E7296901F01F010B432B6149462E
:102A400003F0B4F810F1160F99D0C5F808B0EA6891
:102A50009DF80830013E62F304038DF808302B69BD
:102A60009DF808205B0863F347128DF80820D9E928
:102A700000321344009323F01F0301301E44A6EBE1
:102A80000A06C4B226F01F060F2C03963FF677AF56
:102A900020466946FFF74CFF0134A6E790ED00E0C1
:102AA0000522034B5A60BFF34F8FBFF36F8F704700
:102AB00090ED00E0BFF35F8F0022014B5A6070473A
:102AC00090ED00E070B50E4D2E68102E15D8002444
:102AD000FFF7F0FF0B4B0C4A1A63A64205D10B4BD4
:102AE0001E70FFF7DDFF002070BD6968204601EB16
:102AF0000411FFF71DFF0134EFE74FF0FF30F3E75C
:102B00009464010090ED00E0AAFF440080080020DA
:102B100010B5034C2278FFF723FF207010BD00BFD3
:102B2000800800202DE9F74F254C8A468046002773
:102B3000A1464FF0140B234D57451ADAD8F804304C
:102B40000193002B36D0D8F800100846009103F00E
:102B50004CF8DDE9001306465818013803F045F833
:102B60008642194A08D014235F436FF0150349F8D1
:102B7000073003B0BDE8F08F16F1160F2660F8D0CD
:102B80001378B342F5DD0BFB0793AE60AE60E868E7
:102B9000197B60F3040119732969187B490861F3F3
:102BA00047101873EB6823F01F0363602B6923F051
:102BB0001F0323610137143408F10C08BCE700BF80
:102BC0000008002090ED00E08008002082680C4B97
:102BD0009A60036883F38888436883F38988027B5B
:102BE00002F00101EFF3948323F00303920748BF3F
:102BF00043F0020309B143F0010383F39488704763
:102C000000ED02E0084AD36848B123F400531B04E6
:102C10001B0C43F0BF6343F40033D36070479BB297
:102C200043F40053F5E700BF00ED00E0084AD36825
:102C300040B19BB243F4804343F0BF6343F400339D
:102C4000D360704723F480431B041B0CF4E700BFE0
:102C500000ED00E0084AD36840B19BB243F008039E
:102C600043F0BF6343F40033D360704723F008039D
:102C70001B041B0CF4E700BF00ED00E0034AD2F890
:102C80008C3043F44063C2F88C30704700ED00E0B4
:102C9000084B1A6818B142F001021A60704722F01E
:102CA00001021A601A6811B142F00202F5E722F03F
:102CB0000202F2E7D0ED00E0014B1860704700BF60
:102CC00024000020F0B54B79012B27D0032B22D113
:102CD00010268B79032B1ED1CC7924B1012C1AD16B
:102CE00043681B79BBB10A7912B1022A13D10E22B3
:102CF00047F612270B684568BB422D6863D029D878
:102D0000B3F5965F62D014D8B3F5167F60D007D8BC
:102D1000B3F5967F5FD06FF0220053E00026D8E72E
:102D2000B3F5966F5AD0B3F5166FF4D14FF41D2357
:102D30003CE0B3F5615F54D004D8B3F5165FEAD137
:102D4000334B33E0B3F5964F4DD0B3F5E14FE2D1BD
:102D5000304B2BE0B3F5E13F47D012D84DF6C027FA
:102D6000BB4245D005D8B3F5164FD4D14FF41D035F
:102D70001CE0B3F5614F3ED0B3F5963FCBD1264B67
:102D800014E0B3F5E12F39D008D8B3F5613F38D05E
:102D9000224FBB42BFD14FF0806307E0B3F5612FF4
:102DA00032D01F4FBB42B6D14FF08053C5F8243507
:102DB000C36834432243043303C9C5F86C2583E850
:102DC00003000020F0BD4FF40003EFE7154BEDE7E3
:102DD0004FF41C33EAE74FF4A033E7E74FF49E23A8
:102DE000E4E7114BE2E7114BE0E74FF0EB73DDE76F
:102DF0004FF46503DAE74FF46B03D7E74FF0E8636E
:102E0000D4E74FF06C73D1E74FF07063CEE700BFAB
:102E10000050270000C0750000903A0190D00300D8
:102E200040420F0000B0130000F03A0000A04E0036
:102E30002DE9F04106460F46C56803F0C8F8B8B959
:102E4000294B1B7883F001037268146893B14FF02B
:102E50002003EFF3118183F31188BFF36F8F3046A6
:102E600002F093FF48BB81F31188BFF36F8FEEE749
:102E70000123E9E74FF06408304602F086FF78B995
:102E8000012002F0B2FFB8F10108F5D100212120A4
:102E900001F0C2F8EEE781F31188BFF36F8FF5E719
:102EA0004FF02003EFF3118183F31188BFF36F8F8D
:102EB000304602F06AFF0028EDD00123002205F819
:102EC000107FC4F84455C4F84835C4F82021D4F81C
:102ED0002001C4F85821D4F85821A36081F3118847
:102EE000BFF36F8FBDE8F081810800204FF0000C28
:102EF00043682DE9F041C5681C680F46C4F800C559
:102F000006462860086801213D4B00F01F029140F1
:102F100099600321803243F822107A68511C1EBF49
:102F200002F01F01803143F821C0B968C4F80C05D4
:102F3000481C18BF0020C4F814251EBF01F01F0252
:102F4000803243F82200F868421C0CD04FF0010C8C
:102F500000F01F020CFA02FCC3F808C04FF0030C8B
:102F6000803243F822C0C4F80805C4F81015F1688F
:102F700030460431FFF7A6FE8046002839D1736839
:102F80009B799BB105F1120000F03EFA1D4B98426F
:102F900032D1AB7C43F00043C4F8A031C4F88C308C
:102FA0000123AA7C9340184AC2F804350823C4F8C8
:102FB00000357B6801330CD00023C4F81031D4F8FD
:102FC000103105F11103C4F834350123C4F8383544
:102FD000236073689B791BB94FF48073C4F8043382
:102FE00000231035C4F84455C4F848350123A360C4
:102FF000E3604046BDE8F0816FF00408F9E700BFE8
:10300000002584500000AD0B0070015030B585B034
:103010006C460546084B0FCB84E80F0000220121C7
:103020000820FFF7D7F90820FFF7B6F92146284610
:10303000FFF75CFF05B030BDFC62010030B585B024
:103040006C460546084B0FCB84E80F000022012197
:103050000920FFF7BFF90920FFF79EF9214628460E
:10306000FFF744FF05B030BD0C6301002DE9F043CC
:103070000025214C214E54F8048CDFF8889085B04F
:10308000A84503D8002005B0BDE8F083636A96E840
:1030900007001F6801AB83E807000C221946384679
:1030A00002F0CDFD90B98FB1636A21691B681A697E
:1030B00091420BD19A69A169914207D8E169914285
:1030C00004D962695B6932EA03030AD0276A67B1EF
:1030D0000B4802F0AAF9404080F311884FF0040039
:1030E00002DFE36801351C44CAE7484602F09DF957
:1030F000636A1F60F5E700BF3C0401001C63010028
:103100004069010069690100054B1868043B1B68B0
:10311000092B03D1431E5842584170470020704785
:103120003401FF004F4A08B5136843F002031360EF
:103130004D4B1B68092B01BF4FF050230022C3F8F1
:103140001421C3F81821FFF7DFFF30B10123474AEC
:103150001360A2F63822C2F87835434B1B68092B5E
:1031600007D1434B1B68012B1EBF0122414BC3F803
:103170007825FFF7C9FF10B10E223F4B1A603A4B7A
:103180001B68092B04D100223C4B1A6001225A60B3
:103190000022D30003F57F03D3F80013013108D0D8
:1031A000D3F800130132D3F80433B2F5807F0B60FB
:1031B000EFD1334BDA69D1073BD5324B1946D3F8FF
:1031C0000024012AFBD1C3F80425D1F80034012BD7
:1031D000FBD12B4BDA69D20708D5DA69294922F0ED
:1031E0000102DA61D1F80024012AFBD11A6A013206
:1031F0000AD11A6A22F0FF0242F020021A62214A22
:10320000D2F80034012BFBD100221E4BC3F8042559
:10321000D3F80024012AFBD1BFF34F8F1A491B4B6F
:10322000CA6802F4E0621343CB60BFF34F8F00BF64
:10323000FDE71B6A0133C0D0134BD3F88C2042F456
:103240004062C3F88C20D3F8882042F47002C3F89F
:103250008820BFF34F8FBFF36F8F0D4B0D4A1A605D
:1032600008BD00BFD0ED00E03001FF00384A00503B
:103270003401FF0000400050E4AE03500C47005002
:103280000080FF000090035000ED00E00400FA050C
:10329000500000200090D003044B1A7922B901227B
:1032A00018601A71024870470248704714080020DD
:1032B0000000AD0B0C00AD0B10B1012820D0704701
:1032C0004FF05022D2F81834D2F81814C90311D58F
:1032D00003F00303022B0DD1C2F8183500220D4B69
:1032E0001A601B6802224FF05023C3F80423012206
:1032F0009A6070474FF050230122C3F81825EDE77C
:103300000022054B1A601B684FF05023C3F80403DA
:1033100018607047045100500051005038B510B18A
:10332000012818D038BD4FF050230222012142F26B
:1033300010751C46C3F80823154A10601268154A18
:103340001160D4F81834DB03ECD5012002F04DFDF8
:10335000013DF6D1E6E74FF05024002242F210750D
:103360000D4BC4F808031A601B680C4B1860D4F8A6
:103370000C34D4F80C2403F00103D203D2D5002B73
:10338000D0D0012002F031FD013DF0D1CAE700BFED
:10339000045100500C500050005100500450005097
:1033A000164B10B51A6852B1002018601B68012234
:1033B0004FF05023C3F80823114B1B689847114B5B
:1033C0001A688AB100221A601B684FF05023D3F8A4
:1033D0001824D3F8181402F00302012A4FF0020156
:1033E00003D1C3F818159A6010BDC3F80813044B35
:1033F0000120BDE810401B68184700BF0051005075
:1034000014080020045100500B4A70B51668F143AF
:1034100089B271B10025ECB221FA04F3DB0705F1A2
:103420000105F8D50123A34033430470034813601A
:1034300070BD0348FCE700BF1C0800200000AD0B76
:103440000200AD0BF8B5104B104F53F8205001306F
:1034500053F82060AE4200D8F8BDD5E900342046CC
:10346000984770B16CB10123E41B2411084A61092B
:1034700052F8210004F01F0403FA04F4044342F854
:1034800021400835E6E700BFE0640100BC000020F1
:103490000C010020084BC01A0011084B420953F8D8
:1034A0002220012300F01F0003FA00F010420CBF9D
:1034B00018460020704700BFBC0000200C0100200F
:1034C000114970B505460E46104C8C4204D10F4C84
:1034D000B4420AD1002414E02046FFF7DBFF10B10C
:1034E0002368AB420DD01034EFE72046FFF7D2FF40
:1034F00008B91034ECE72168284602F094FB002854
:10350000F7D1204670BD00BF0C010020BC00002098
:10351000F8B505460027154E4FF02002EFF3118352
:1035200082F31188BFF36F8F286988B12F6183F30D
:103530001188BFF36F8F00F0C1FB4FF02003EFF352
:10354000118083F31188BFF36F8F02F09AFCE3E7D9
:1035500002F05DFD012104460228D8BF084602F0B2
:1035600066FD7462FEF78EFFD6E700BF20080020DC
:103570000248034A0021121A02F0B2BB6001002087
:1035800084080020012208B5094B02201A70FFF7B9
:1035900059FF00F053FE0320FFF754FF00F0DCFD5D
:1035A00001F01CFF034A137B23F00103137308BDD2
:1035B00081080020E00100202DE98048374BA7B0AA
:1035C00003F5006989F3088883F30A880024E0235F
:1035D000334D4FF0010B85F82230EC772C766C766A
:1035E000AC76EC766B6A2F4E43F4E0236B626B6A29
:1035F000DFF8CC8043F400236B62AC63FFF7ECF898
:10360000FEF73AFF4FF0FF33AB62EB6240F201137B
:10361000254DADF8243006ABAB602046CDE9204403
:10362000FFF710FF0120FFF70DFF00F09DFC1F4B7F
:10363000AE624FF480521E490593CDE9034B4346D9
:10364000CDE901440094304600F058FD737B82467A
:1036500023F004033046737302F03CFC0F23154F34
:10366000CDE902434FF4A072134B1449CDE904B4E1
:10367000CDE90054384600F041FD7B7BEF6023F03C
:1036800004037B7305F11C032C76C5F80490C5E98F
:103690000733424651463046FEF7D0FEC819002097
:1036A00000ED00E0E001002020080020A7690100F3
:1036B00088080020600100201135010088180020D2
:1036C0008535010070B50E4B0E4CA34201D300208E
:1036D00070BDD3E9030141EA000212F003020BD1ED
:1036E0009D685A61AA4201D11C33EEE75E6901323E
:1036F0000E6059610144F5E76FF01500E8E700BF7F
:103700001001002010010020D3B50C4616461F46BC
:103710004FF02003EFF3118183F31188BFF36F8F14
:1037200043695BB123601B68436183690133836133
:10373000002081F31188BFF36F8F11E056EA070272
:1037400003D123606FF00B00F3E70246CDE9006779
:10375000044800F077FB18B9034B9B685B69236052
:1037600002B0D0BD8208002020080020F8B5044631
:103770000D464FF02003EFF3118683F31188BFF35A
:103780006F8F47696FB902F0FDFB50B12A68C767B8
:10379000426102F09FFB3146BDE8F840074800F067
:1037A0000FB92B6862691A602B686361A369013BDA
:1037B000A36186F31188BFF36F8FF8BD82080020E4
:1037C0002DE9F341044616461F464FF02003EFF360
:1037D000118883F31188BFF36F8FC368324A6BB1CE
:1037E00080689168884219D056EA070318D188F397
:1037F0001188BFF36F8F6FF00F000CE0916891F9A3
:103800000E100133E36093682161A36088F311888F
:10381000BFF36F8F002002B0BDE8F0812169F0E7AF
:1038200090F90E3091F90E109942A8BF194621EA7D
:10383000E17199422CDA00F053FB0546CDE90067AF
:1038400022464146194800F0FDFA0028E3D04FF027
:103850002003EFF3118683F31188BFF36F8F236882
:103860002169A34207D033B193F90E309942A8BF22
:10387000194621EAE171A06890F90E30994209D108
:103880006DB13146094800F09BF86FF00A00C2E7BD
:103890000025D3E700F024FB0028F2D1F0E786F3FF
:1038A0001188BFF36F8FF0E7200800208208002006
:1038B00038B583680446002B36D01E4A926893427E
:1038C00035D1DA7B013ADA73C368012B05D0013BAD
:1038D000C36000F0D9F8002038BD4FF02003EFF3AB
:1038E000118583F31188BFF36F8F0169806890F9A8
:1038F0000E30994201D000F0F3FA204602F042FB6C
:10390000A06058B190F90E2022610022C26702F037
:10391000E1FA2946084800F053F8DAE7E06085F359
:103920001188BFF36F8FD4E76FF01500D4E74FF025
:10393000FF30D1E7200800208208002010B5084C95
:1039400023685BB1FEF774F92368064A1844506196
:103950000021BDE81040184602F069BB10BD00BF51
:103960005C08002020080020F8B50D464FF0200329
:10397000EFF3118483F31188BFF36F8F4FF400418D
:1039800040F2E73600270022E1FB0067094B304692
:103990005A6139464FF47A720023FCF74FFD064B0B
:1039A0001860064B1D60FFF7C9FF84F31188BFF351
:1039B0006F8FF8BD200800205C0800205808002008
:1039C00049B9EFF3058030B9054B9A6A9B689A4272
:1039D00001D0FEF78BBC81F31188BFF36F8F704766
:1039E000200800204FF02003EFF3118183F31188AA
:1039F000BFF36F8F044B9A68D37B013BD37381F382
:103A00001188BFF36F8F704720080020094B03F126
:103A10002C02824205D19B688B4202D14B7BDB0694
:103A200006D1D1E9003213605A600023C1E90033A6
:103A3000704700BF2008002038B5124C01462369AA
:103A4000A2680BB1E5680CE004F12C0002F03CFA2E
:103A50000546537B980644BF43F008035373002D7B
:103A6000F0D049B9537BDB0606D1AB6923B9D389C2
:103A70007F2B01D9A26238BD954201D0FFF75EFFCE
:103A8000A562F8E72008002010B54FF02003EFF3FF
:103A9000118483F31188BFF36F8F084B00209A685D
:103AA000D37B0133D373FFF7C7FF84F31188BFF3D0
:103AB0006F8FBDE8104002F0F0B900BF2008002071
:103AC00070B4437B1A0629D4DB0627D183692BBB4C
:103AD000134A02F12C01D2E90B348B4218D0BBB14E
:103AE00090F90E5093F90E60AE420CDD5A68C0E9B1
:103AF000003210605860437B63F07F03437370BCF7
:103B00000020FFF799BF9C4202D01B68002BE9D12F
:103B1000C0E90014136B18601063ECE770BC7047C9
:103B20002008002010B54FF02003EFF3118483F339
:103B30001188BFF36F8F437B590704D484F3118836
:103B4000BFF36F8F10BD23F004034373FFF7B8FF7B
:103B50002146BDE810400148FFF732BF820800202F
:103B600070B590F90D300446002B03DA0146164873
:103B7000FFF74CFF154A02F12C01D2E90B308B42C2
:103B80001CD0DBB194F90E5093F90E60AE4210DDFB
:103B90005968C4E900310C605C60637B906863F035
:103BA0007F036373031B58425841BDE87040FFF721
:103BB00043BF984202D01B68002BE5D1C4E9001036
:103BC000136B1C601463E8E74C08002020080020F9
:103BD00070B54FF02003EFF3118483F31188BFF326
:103BE0006F8F174A174993680D68AB42154606D187
:103BF000FFF7A4FE84F31188BFF36F8F70BD00261A
:103C00000E6011490968C1B1D9897F2915D8597B3E
:103C1000C90612D10D4993F90E6009688E420CDB7A
:103C20000B498B4209D05169814203DC1846FFF7EA
:103C300097FFDDE7091A5161DCE700236B61D9E7E3
:103C400020080020540800205C08002058080020AC
:103C50006001002070B50446183002F0C2F94FF040
:103C60002003EFF3118683F31188BFF36F8F94F96C
:103C70000D30002B07DA21460E48FFF7C7FE637BA5
:103C800003F07F0363730C4D637BA86843F010035C
:103C90006373031B58425841FFF7CEFE86F3118829
:103CA000BFF36F8FAB68A34203D1BDE8704002F051
:103CB000F4B870BD4C080020200800202DE9F04128
:103CC00004464FF02003EFF3118283F31188BFF312
:103CD0006F8F437B13F0280F05D082F31188BFF359
:103CE0006F8FBDE8F08143F02003437382F31188A6
:103CF000BFF36F8F183002F074F94FF02003EFF329
:103D0000118683F31188BFF36F8F637BD80616D1BA
:103D1000A269A2B9190607D521462648FFF776FE03
:103D2000637B03F07F036373234B9868021B50424D
:103D30005041FFF781FE04F1300800271DE09B078A
:103D4000F9D52146A068FFF761FE637B23F00203EB
:103D500063730023A360EEE705F1180002F041F958
:103D6000A8682946FFF752FE6B7BAF6023F0020381
:103D70006B73EF672846FFF7A3FE256B454501D01F
:103D8000002DE9D10C4B9A680C4B9A4202D10120CC
:103D9000FFF752FE637B43F008036373236E86F3E1
:103DA0001188BFF36F8F002B9BD02046BDE8F041F8
:103DB000184700BF4C0800202008002060010020A8
:103DC00010B590F90D300446002B07DA014608487B
:103DD000FFF71CFE637B03F07F036373054B98685A
:103DE000031B58425841BDE81040FFF725BE00BFF5
:103DF0004C080020200800202DE9F041064614461A
:103E00001D464FF02003EFF3118783F31188BFF3B2
:103E10006F8F02F08FF887F31188BFF36F8F6B1CE1
:103E200008BFB4F1FF3F08D022462B4606F1180028
:103E30000349BDE8F04100F077BABDE8F08100BF6A
:103E4000F55E010010B50C46064B11469868064B0E
:103E50001860DDE90223FFF7CFFF2046BDE81040E0
:103E6000FEF744BA20080020540800202DE9F04154
:103E70000646884602F0F5F804464FF02003EFF3BB
:103E8000118783F31188BFF36F8F124D124BA8680F
:103E900034441860FFF794FFA8681049324643463F
:103EA000183000F041FAAA683846537B002543F0E9
:103EB00010035373FEF71AFA02F0D3F8221A65F1D1
:103EC00000031946002A71F100031046B8BF002014
:103ED000BDE8F0812008002054080020F55E0100B4
:103EE0002DE9F04104464FF02003EFF3118883F3EE
:103EF0001188BFF36F8F437B4EB2DB062ED18369EF
:103F000063BB184D014605F12C073846FFF77EFDCF
:103F1000EB6AA673BB422A4619D0C3B1296B93F949
:103F20000E00B0420EDD5A68C4E9003214605C60D5
:103F30000120FFF781FD012088F31188BFF36F8F07
:103F4000BDE8F081994202D01B68002BE7D1136BCA
:103F500027606360136B1C601463E9E7A67300209D
:103F6000EAE700BF200800200021044B084603F1C7
:103F70002C02C3E90B22FFF7F7BC00BF200800208A
:103F8000F8B5234C234BA2689A4229D04FF0200366
:103F9000EFF3118683F31188BFF36F8F04F12C05C3
:103FA000A1682846FFF732FDE26AA368AA4228D03A
:103FB0003AB3206B93F90E1092F90E708F421BDD0D
:103FC0005168C3E900210B6053605A7B012062F005
:103FD0007F025A73FFF730FD86F31188BFF36F8FAE
:103FE0004FF02003EFF3118083F31188BFF36F8F3D
:103FF000BDE8F840FEF77AB9824202D01268002A82
:10400000DAD1226B1D605A60226B13602363DCE7F8
:104010002008002060010020B1F1FF3F08BFB0F18F
:10402000FF3F08B502460B4606D10B4B9868FFF7D9
:1040300011FE4FF0FF3008BD13430AD1FFF7A0FF78
:1040400000204FF47A7380FB0323D00B40EA4340F7
:10405000F1E7FFF70BFFF4E720080020014B986819
:10406000704700BF2008002038B504464FF02003F9
:10407000EFF3118583F31188BFF36F8F01F082FF97
:1040800048B10022C26701F025FF2946BDE838404B
:104090000448FFF795BCD4E902329A4218BF0133B5
:1040A000A360F2E78208002037B514461D464FF0A2
:1040B0002003EFF3118183F31188BFF36F8F8368BF
:1040C00043B1013B836081F31188BFF36F8F002000
:1040D00003B030BD54EA050306D181F31188BFF364
:1040E0006F8F6FF00F00F3E70246CDE900450248FD
:1040F000FFF7A8FEECE700BF82080020F0B500F152
:10410000300585B0C0E90C550E9D044605730425A5
:1041100045730D9D07328573002522F00702C0E923
:104120001A128E180C9AC573C0E9065505670292DB
:104130000B9A01920A9A00923246FEF763F9054BF8
:10414000C4E917559B6803B15B6F3046636705B0E0
:10415000F0BD00BF200800202DE9F0472A4E2B4D6E
:10416000B04686B0B54205F1300410D3FFF73AFCF3
:104170004FF4004940F2E7360027244CDFF890A0C6
:10418000444521D306B0BDE8F047FFF77DBC54F8A5
:10419000043C059354F8103C049354F8143C0393E6
:1041A00054F8183C029354F81C3C019354F8203CFA
:1041B000009354E90A2354E90C01FFF79FFF54F8D8
:1041C000303CDD652546CDE7636A5A1C0DD030468C
:1041D000394623EAE373C9FB0301B94208BFB04281
:1041E000256804D12846FFF79DFC3034C8E74FF41A
:1041F0007A720023FCF722F902460B4605F11800FB
:10420000514600F091F8F0E7100100201001002065
:10421000F55E010008B54FF02003EFF3118483F33E
:104220001188BFF36F8F044B98681861FFF712FD78
:104230002046FEF75BF800BF20080020024A034931
:10424000034801F0F2B800BF38660100AC69010014
:10425000B969010008B50648064A0749121A01F073
:1042600015FDBDE80840054A0549064801F00EBDA8
:104270000000002060010020E4690100000000004F
:10428000E469010000000020034B1B680BB9FDF737
:10429000CFBC0020704700BF6008002030B5036825
:1042A00068B10A4A5268904209D043B1D3E9042167
:1042B000D0E90445121945EB0101C3E90421426824
:1042C00013605A600023C0E9003330BD5400002061
:1042D00038B5134B1C689C4208BF0024FFF7D4FF7D
:1042E000C4B1D4E90423141A63EBE075012C75F111
:1042F000000312DB6FF000420023A242204673EB62
:10430000050400DA1046074B5B6913B19842A8BF59
:10431000184638BD6FF00040F5E70020F3E700BF16
:1043200054000020200800202DE9F74F0191591C6E
:1043300008BFB2F1FF3F824673D0541C43F1000521
:104340006FF001034FF0FF3BB3EB04086BEB050983
:10435000B8F1000F79F100030FDBFFF795FF6FF065
:104360000103364AD2E9001C5B1A6BEB0C021E1BE0
:1043700062EB0507341A67EBE075019BCAF8083059
:104380004FF02003EFF3118683F31188BFF36F8F93
:10439000FFF77AFF012C75F100032146B8BF012118
:1043A0002A46B8BF0022264B0C1842EBE0751A686B
:1043B000CAE904459A4201D05F6852B95A68CAF8FE
:1043C0000030CAF804205A68C2F800A0C3F804A05C
:1043D00014E0D2E90489DAE90445444575EB0901A2
:1043E00022DAB8EB040069EB0501C2E90401516867
:1043F000CAE90021C1F800A0C2F804A01A689A42D4
:104400000BD0924509D1FFF763FF18B10D4B5B69E3
:10441000834202D00021FDF7D9FB86F31188BFF358
:104420006F8F03B0BDE8F08FB4EB080065EB0901B6
:10443000BA42CAE90401C1D01268BEE76002002096
:1044400054000020200800202DE9F74F0446FFF714
:10445000BFFB4FF02003EFF3118583F31188BFF307
:104460006F8F2C4BDFF8B0909846CB46DFF8ACA0AE
:104470001C60D8F800C0DAF800406646D9E900238D
:104480005445CDE900234FEAE6770CD05CB1D4E97E
:1044900004128C4577EB02031BDAB1EB0C0062EBE4
:1044A0000701C4E904010024009BC8F80040F21889
:1044B000019B47EB0303CBE90023FFF709FF2146EC
:1044C000FDF784FB85F31188BFF36F8F03B0BDE860
:1044D000F08F0022DDE9006700237618ACEB0100C5
:1044E00047EBE177C8F80000C4E904232046C9E996
:1044F0000067FFF7D3FE85F31188BFF36F8FA368C2
:1045000098474FF02003EFF3118583F31188BFF331
:104510006F8FAEE76008002060020020540000208A
:104520002DE918484FF02003EFF3118483F311882D
:10453000BFF36F8FFDF77CFB074BD3E9002312EB32
:10454000000B43F1000C5846614684F31188BFF319
:104550006F8FBDE8188800BF6002002038B5064C98
:10456000064DAC4201D3002038BDD4E901122046EB
:1045700001F07BFD1434F4E710010020100100204D
:1045800001F06DBB0A46002101F0AABB10B511482D
:1045900000F048F800B110BD0F4800F043F80028C3
:1045A000F9D10E4C204600F03DF80028F3D10C4B19
:1045B0000C481C6000F036F801460028EBD100F0F2
:1045C0002DF8044608B1204610BD00F051F82046F1
:1045D000FAE700BF680000205C00002064000020B3
:1045E0006C0000206000002008B5084800F024F8A6
:1045F000074800F021F8074800F01EF8064800F0D0
:104600001BF8BDE8084000F00BB800BF68000020B0
:104610005C00002064000020600000200020704743
:10462000704700BF08B5034B02681B6810689847C5
:10463000002008BD8000002008B5034B02685B68BD
:1046400010689847002008BD80000020024B0268D7
:104650009B681068184700BF8000002008B5034B16
:104660000268DB6810689847002008BD80000020C1
:1046700070B5094C094D2069AB68984718B1084BD3
:1046800008485B6898470021074AEB681160206979
:10469000BDE87040184700BF900000208000002057
:1046A00070000020F86401006408002070B51A4D05
:1046B0001A4E0446B26828699047F0B95CB1184CAC
:1046C0002368ABB1012B1AD0013B23602869F36842
:1046D0009847002070BD124C216839B90120114B58
:1046E000114AC3F800051368002BFCD10131216089
:1046F000F36828699847002070BD0C4870BD0A4ACD
:104700001368002BFCD1074A6FF07E40C2F80035D9
:1047100000F020F82368D7E79000002080000020F8
:10472000640800200000845010198450E98FFFFFB6
:104730000020704700207047430503D54FF0FF323B
:10474000024B1A60024B1860704700BF081184507A
:10475000081A8450014B1860704700BF041A845037
:1047600008B100F003B84FF47500704702460748DF
:1047700003681342FCD021B1054B06481B680B604F
:104780000360054B00201A60704700BF001A845078
:104790000411845008118450081A845000F09EB807
:1047A00038B131B1002201440346013081421A7010
:1047B000FAD170472DE9F041ADF51A7D0E4605920C
:1047C0000021144612A84FF408721D4601F088FA21
:1047D0000021282208A8069101F082FA002E3CD080
:1047E000002D3AD0002C38D0042106A8FFF7CAFECD
:1047F00008A82821FFF7C6FE08A800F031F878B114
:104800004FF0FF374FF4087112A8FFF7C9FF0421DA
:1048100006A8FFF7C5FF38460DF51A7DBDE8F08103
:1048200012AB0DF11C080246CDE90153039005AB14
:1048300008A9CDF8008006A800F02AFD0028DFD1E5
:104840002B68A342DCD3D8F8001007462246304636
:104850000831FFF795FE2C60D4E74FF0FF37DAE719
:104860001C2330B583B001A90446019300F0E4F99C
:10487000054638B9019B1C2B07D0164D20461C213C
:10488000FFF780FE284603B030BD0121D4E9003295
:10489000003B18BF0123E1610AB143F00203A268A3
:1048A00032B9E26842B9C4E908328BB90A4DE5E78A
:1048B000E26843F004033AB10022284643F00803BB
:1048C000C4E9083203B030BD1546C4E90832D9E75F
:1048D0001546D7E7370CF0000E0CF00010B50C4C65
:1048E000236813B10B4B1B682BB900F065F930B985
:1048F0000122084B1A6001230020236010BD0138FB
:10490000062801D9044810BD044B53F8200010BDFF
:10491000680800206C080020FE8FFFFF186501006A
:1049200010B50A4C23681BB101230020236010BD81
:1049300000F0AEF80028F7D00138062803D8044B61
:1049400053F8200010BD034810BD00BF68080020C8
:1049500018650100FE8FFFFFBFF34F8F0549064B1F
:10496000CA6802F4E0621343CB60BFF34F8F00BF0D
:10497000FDE700BF00ED00E00400FA054FF0FE3354
:10498000002130B4064A074D074C2B6013602360AA
:10499000064A074CEB606368C2F8001530BC184744
:1049A000041484500014845008148450000084506F
:1049B00070000020024BD0E90012C3E900127047DA
:1049C0007000002048B143682BB1BFF35F8F002314
:1049D000036018467047024870476FF4E040704724
:1049E000EA8FFFFF10B5044628B1636813B10023B6
:1049F0002360636010BD024B02485B689847F4E790
:104A0000700000203465010010B5044630B100226A
:104A10006368226043F00103636010BD0148FFF743
:104A2000ADFFF4E75C65010080B1436863B101222A
:104A3000D0E8EF3FC0E8E12F0029F9D1012BF7D0F2
:104A4000BFF35F8F00207047024870476FF4E0406B
:104A5000704700BFEA8FFFFF70B40B4B0668C26857
:104A6000D0E90154C3E90242C3E90065D1E9030278
:104A70000E68064BD1E90154C3E90065C3E9024061
:104A80001A6170BC704700BF8000002090000020B9
:104A900010B5FFF74DFE20B10324FFF7A5FD20461A
:104AA00010BDFFF773FD90B9FFF700FE90B90F4BF3
:104AB0001B681B0EF02B08D10D4A0E4B12689A4250
:104AC0000AD00724FFF736FEE7E70624FAE70424B6
:104AD000204610BD0024F5E70120FFF7E7FD04465E
:104AE0000028F7D1044B1860D9E700BF281984507B
:104AF000241A84500000E0200C1A845030B5ADF523
:104B0000157D4FF4087200210CA801F0E9F800218E
:104B1000282202A8019101F0E3F802A8FFF7A0FE05
:104B200020B1052420460DF5157D30BD1D4D4FF0FB
:104B3000FF312868FFF78AFD0446E8B90020FFF737
:104B4000B5FD58BB0CAA02A901A800F0EDFB044674
:104B50000120FFF7ABFDE8B92868FFF77FFD28B912
:104B6000002CDED120460DF5157D30BD0E48FFF737
:104B700005FF002CF6D0D4E70C48FFF7FFFE012C10
:104B8000DCD12868FFF76AFD0028CAD00648FFF785
:104B9000F5FEC6E70648FFF7F1FEDDE70548FFF73B
:104BA000EDFECFE76C0000209865010080650100F4
:104BB000D0650100B065010008B5FFF7B9FD18B177
:104BC000FFF712FD032008BDFFF7E0FCC0B9FFF7B7
:104BD0006DFDB8B9144B1B681B0EF02B0AD1134A9C
:104BE000134B12689A4217D0FFF7A4FDFFF7FCFCA5
:104BF000072008BDFFF79EFDFFF7F6FC062008BD65
:104C0000042008BDFFF796FDFFF7EEFCFFF776FFE7
:104C1000002818BF052008BD0120FFF747FD002828
:104C2000F0D1044B1860F1E728198450241A8450FD
:104C30000000E0200C1A8450002866D0002964D0BF
:104C40000B681C2B61D14FF47F033B4AD3F8101C37
:104C500091425CD0D3F8102C013258D0D3F8102CEC
:104C60004FF47F030260D3F8141C344A914260D0A1
:104C7000D3F8142C01325CD0D3F8142C4FF47F03FA
:104C80004260D3F8182C12F5947F4FD0D3F8182C2B
:104C900001324BD0D3F8182C4FF47F038260D3F845
:104CA0001C1C274A91423ED0D3F81C2C01323AD02A
:104CB000D3F81C2C4FF47F03C260D3F8002C703261
:104CC0002FD0D3F8002C01322BD0D3F8002C4FF486
:104CD0007F030261D3F8042CAF3220D0D3F8042C28
:104CE00001321CD0D3F8042C4FF47F034261D3F877
:104CF000081C144A91420DD0D3F8082C013209D077
:104D0000D3F8083C8361002070470120704740F6CB
:104D1000FC02A5E740F2373383610020704751223F
:104D2000E2E79022D3E742F60412C3E740F6D862E6
:104D3000B2E742F2D002A1E7FCF8FFFFD020FFFF6C
:104D40000429FFFF37F3FFFF2DE9F843002877D050
:104D50000C46002974D01D46002B71D006461AB1AE
:104D6000012200232A6003602B68002B64D02946AF
:104D7000204600F015FB074600285ED12146286832
:104D800000F0F0FA0746002857D12B68082B66D0B0
:104D9000042B67D0A3F10208B8FA88F84FEA581834
:104DA00001239C46314A3249136010460B60943A05
:104DB000C0F800C0636A136011688B42F8D14FF0ED
:104DC00000092C4B4FF0FF30C3F80090FFF7B4FC04
:104DD000294B2A4A48461A60FFF7BCFC284A294B4F
:104DE000C2F80080186840F48060FFF7B3FC0A2224
:104DF000254B1A60089A2369012A616A24D0234A44
:104E0000A2FB03231B09012203FB01F303EB430372
:104E10001F49DB039B090B60164B38461A60336849
:104E20002A6823F07F4343EA026333602A6843EA37
:104E300002233360BDE8F883164F3846BDE8F88397
:104E4000154F3846BDE8F8834FF47F03D3F80C2C98
:104E5000013202D0D3F80C3CD1E71623D3E74FF050
:104E600003089DE74FF002089AE700BFC411845081
:104E7000401184502C11845000118450FEFFFF0F0C
:104E80000C118450041A845038118450ABAAAAAA79
:104E9000D8118450310CF100350CF100F0B400242D
:104EA000C9002646274601F1FF3C06E09F4215D087
:104EB0000126654518D82C461F46630950F8233053
:104EC00004F01F01CB401F2904F1010518BF03F0B6
:104ED0000103002CEAD101263546ECE70136964263
:104EE000E7D10348F0BC70470020F0BC704700BF1A
:104EF000360CF10000285FD02DE9F0414C1EB4F5CE
:104F0000047F26D22BB322B3CC00012B04F1FF3E49
:104F10002FD000218C460F460D4603F1FF384C0977
:104F200050F8244001F01F06F4401F2E18BF04F073
:104F3000010421B90125AC4629462746EFE7AB42DB
:104F400013D0A74201D10CF1010C454504D16245B3
:104F500002D21A48BDE8F0813C4601318E4505F188
:104F60000105EAD20020BDE8F08100254FF0010CD8
:104F7000F3E70026B446374631464B0950F8233054
:104F800001F01F05EB401F2D18BF03F0010339B1DD
:104F90005FB99C4501D0634608E06346013605E0F1
:104FA000012631469C460127E7E73E46B242D0D370
:104FB0000131A142F6D1D5E700487047370CF10026
:104FC0002DE9F04F8DB0189E07460C46179D002E18
:104FD0004CD1D1F810B000211D60169B1960002A39
:104FE00000F01E819A4A9B4B1168626A1B689A42C4
:104FF00047D10A2945D1FB7804930423B84602938C
:10500000954BA3FB0B234FEA930A0AEB4A0305F1E6
:1050100008020392ABEB430A169BC3F800B0BBF146
:10502000000F00F0C3805D464FF00009039E00F0C2
:10503000C7F900230593B8F1000F00F0E580002CBC
:1050400000F0E280049B002B00F0DC80204604A9E5
:1050500000F0A6F9B8B1814B984240F0A7800290C9
:1050600000F0AEF902980DB0BDE8F08F4FF47F016B
:10507000D1F80C0C01300CBF4FF4047BD1F80CBC00
:10508000A9E77748EBE72146049800F06BF9002880
:10509000E1D1049F082F00F0B980042F00F0B88000
:1050A000A7F10207B7FA87F77F09012319466D4870
:1050B000036040F8843C6B4B66481960636A036088
:1050C00000688342F7D10023674A4FF0FF30136036
:1050D000FFF732FB002365491846654B1960FFF75F
:1050E00039FB6449644B0F6018685B4F40F4806083
:1050F000FFF730FB0A210122554B604819602169F6
:10510000636AA7FB01C1090903FB01F303EB430336
:10511000DB039B090360544B05A81A600499D8F877
:1051200000200B0243EA016322F07F421343C8F8D8
:10513000003000F007F900288DD1514BA7FB05275F
:105140001A681433069253F8102CB9EB970F079294
:1051500053F80C2C089253F8082C099253F8042C9D
:105160000A921B680B9302D1BAF1000F41D11822A9
:1051700030460DEB0201FFF703FA183D183609F12E
:105180000109002D7FF453AFBBF5047F5DD8039D6B
:10519000594628466269FFF781FE00284BD000235C
:1051A000169A13602D4B98423FF459AF049D082D79
:1051B00034D0002204AB214640466D000092049595
:1051C000FFF7C2FD2F4B984224D000287FF447AF51
:1051D000D8F80020130A03F47F03134323F07F431E
:1051E000C8F80030029B013B02937FF415AF00200A
:1051F00035E73046524606A9FFF7C2F9A5EB0A0586
:105200005644BCE71F4826E71F4824E703274CE71E
:1052100002274AE7236A002B3FF421AF1B481EE711
:10522000012221463846009604ABFFF78DFD002889
:105230003FF4E3AE13E74FF4806359462846A26972
:10524000FFF758FE0028AAD1D1E7169B1D60ADE7F5
:105250003811845030118450ABAAAAAA020CF10074
:10526000300CF100C41184502C118450FEFFFF0F4C
:10527000001184500C118450041A8450D8118450A9
:1052800014118450310CF100350CF100320CF10096
:105290002DE9F0411F4E84B004460D4630684FF0B2
:1052A000FF3190460C9FFFF7D1F9D8B90020FFF7E6
:1052B000FDF9F8B900230B9A20460092029342466A
:1052C00029460A9B0197FFF77BFE04460120FFF762
:1052D000EDF9D0B93068FFF7C1F978B9204604B0CC
:1052E000BDE8F0810C48FFF749FB0020FFF7DEF92D
:1052F0000028DFD00948FFF741FBDBE70848FFF74C
:105300003DFB204604B0BDE8F0810648FFF736FBC0
:10531000E0E700BF6C00002080650100B06501007F
:1053200098650100D065010010B5012486B005AB79
:10533000CDE901240093002204ABFFF741FE06B043
:1053400010BD00BF014608B54FF48060FFF708FAB2
:1053500000230249024A0B60136008BDC811845043
:105360002C1184500138072805D8DFE800F00A0E18
:1053700004120404040609487047CB6800204B62FD
:1053800070470B6800204B6270474B6800204B62EF
:1053900070478B6800204B62704700BF310CF100F2
:1053A0000B6802E0082B0B6006D8026A13424FEA32
:1053B0004303F7D00020704700487047310CF100DC
:1053C00000230449044A0B604FF480601360FFF728
:1053D000B3B900BF2C118450C411845008B5FCF738
:1053E00037FDBDE80840FCF7C7BC60B1436803F077
:1053F0000303012B03D0032B05D103681BB100234A
:105400008360184670476FF0150070474268034686
:1054100002F00302032A4FF0000281600CBF006813
:1054200010465A607047002070470FB407B504A9B2
:1054300051F8040B0191FBF7BBF903B05DF804EBE5
:1054400004B07047038B13F0070305D10368002BEA
:105450000CBF002003207047022B05D1438B002B8B
:1054600014BF002004207047012B05D10368002BD6
:105470000CBF002005207047002070472DE9F04147
:105480000D4607461946281D90461E46FFF7BEFFEB
:10549000044638B13346424629463846A446BDE85C
:1054A000F0416047BDE8F08110B44FF02004EFF305
:1054B000118284F31188BFF36F8F41615DF8044B53
:1054C0000121FBF783B910B50C4640B139B1081D75
:1054D000FFF78BFF28B9A36833F0030301D06FF007
:1054E000150010BD38B50C46054658B151B10B68D2
:1054F00043B14B6833B11C22002100F0F1FB0020C6
:105500002C6138BD6FF01500FBE770B504460D4601
:10551000FFF7D9FF061E31DB4FF02003EFF31181B7
:1055200083F31188BFF36F8F4FF6FF76638B208B69
:10553000B34200F007022ED0022A0ED1013363835A
:105540001646012381F31188BFF36F8FB3B1002397
:1055500029462046FFF792FF10E0830701D0062A74
:105560000ED100232B60636893B9C4E90055164639
:1055700062B90A4620460221FBF728F9304670BD81
:10558000052A0CBF6FF022066FF004060023D9E74E
:105590001D606560EBE76FF00A06F7E7044608B5A3
:1055A000084611461A46A047FEF758FDFDF782F956
:1055B000836800EBC101B3F5004F2CBF51F8220006
:1055C00031F81200704700EBC1018068B0F5004F60
:1055D0002CBF41F8223021F81230704708B5012263
:1055E000FFF7E6FF400808BD836800EBC101B3F593
:1055F000004F08D34B681AB143F001034B6070476A
:1056000023F00103FAE74B881AB143F001034B8002
:10561000704723F00103FAE753000122FFF7D3BFDD
:105620008368481CB3F5004F2CBF02230123C01A26
:10563000B0FA80F0C0F11F0070472DE9F041044638
:105640000D46FFF7CBFFA3680146B3F5004F01D32A
:10565000012835D02046FFF7E3FF04EB80021669EE
:105660009EB9012303FA00F0E36829460343E3608F
:10567000204615612B460222FFF7A5FF032229468B
:105680002046BDE8F041FFF79EBF0222314620468A
:10569000FFF78EFF07460346022229462046FFF702
:1056A00092FF3346032229462046FFF78CFF032250
:1056B00039462B462046FFF786FF02223146DFE7B8
:1056C000BDE8F081B2F5802FF8B52CBF0825042580
:1056D0000023551B0022CC1D0D4424F0070425F0A7
:1056E00007052D1BED0804602946C4E90023C4E921
:1056F00002522046FFF794FF134686001B36471CD4
:10570000F60804F11001BB4229DB32462046002195
:10571000FFF782FFAF1B204601220021FFF764FF45
:105720003A463146FFF778FF33463146204600229D
:10573000FFF749FF294620460022FFF76DFF3B4651
:10574000294620460022FFF73EFF29462046012237
:10575000FFF74AFF3146BDE8F840FFF76EBF41F85A
:10576000042B0133CFE72DE9F048D0E900244FF0B6
:105770003333A2FB03BC1BEB03064CEB03052F46A4
:105780000026A4FB03451BEB04024CEB0501D219D8
:10579000324646EB0101631845EB0202C0E90032D4
:1057A000BDE8F0880B6870B5002B10DD013B0B6085
:1057B0000A2102684468A2FB015601FB046626F038
:1057C0007043C0E90053310F3031084670BD3021BD
:1057D000FBE72DE9F74F9946D37814466F2BA3F1D9
:1057E000410206460F4601922DD028D8582B0CBFF7
:1057F00010250A25AA464FF0000BDDF830805246EE
:105800005B4630463946FAF719FE092AD3B221D849
:1058100030335F45DBB208BF564508F8013D01D380
:10582000C84514D823789B0605D5082D18D1A37830
:1058300043F00803A370404603B0BDE8F08F702B1F
:1058400003D0782BD3E70825D4E71025D2E7064606
:105850000F46D4E7019A192A94BF37335733D8E754
:10586000102DE8D1A37843F01003E3E72DE9F041D0
:105870000746884615461E461446B442A4EB05006A
:1058800002D33EB923782BB1414614F8010BB84737
:105890000028F2DABDE8F0817047FDF743BC0C2325
:1058A000C268C9B201FB0323186C00F007007047FF
:1058B0004FF02003EFF3118283F31188BFF36F8F52
:1058C000036813F0C00301D08B4207D101230360AA
:1058D000002082F31188BFF36F8F70474FF0FF30C5
:1058E000F7E710B54FF02003EFF3118283F311882F
:1058F000BFF36F8F036803F00704012C06D101602A
:10590000002082F31188BFF36F8F10BD03F0C00336
:105910008B4214BF4FF0FF306FF04400F1E74FF0BF
:105920002003EFF3118283F31188BFF36F8F0368B5
:1059300003F0C00343F00203036082F31188BFF356
:105940006F8F7047C3681C2010B4CCB204FB0030CA
:1059500000215DF8044B10470020FDF7ADBC00208E
:10596000FDF7DCBC1046FEF77FBB38B50C23CCB28C
:1059700063430546C068403380211844FFF798FF11
:10598000002805DB696801EBC4014B6898470020DB
:1059900038BD2DE9F8430C25CEB27543C4680746DF
:1059A00005F140008021204491469846FFF799FF79
:1059B000002807DB2C44C4E90E987B6853F8363086
:1059C00098470020BDE8F883704770477047002370
:1059D00007B501A88DF80430FEF7E0FE03B05DF8CE
:1059E00004FB70B506460C46154600F007F9012881
:1059F00036D16FF01500BDE87040714672467346AF
:105A0000B7EE000AF7EE000AB7EE001AF7EE001A3A
:105A1000B7EE002AF7EE002AB7EE003AF7EE003AAA
:105A2000B7EE004AF7EE004AB7EE005AF7EE005A1A
:105A3000B7EE006AF7EE006AB7EE007AF7EE007A8A
:105A40008EF3008C10B4F1EE10CA4FF66074C0F6FD
:105A5000FF740CEA040CE1EE10CA10BCF446744763
:105A6000284600F0CBF80128C3D0902CC1D12B469A
:105A7000224631460020FEF79DFEBCE738B50546BC
:105A80000C46B1BB6FF01500BDE838407146724658
:105A90007346B7EE000AF7EE000AB7EE001AF7EE0B
:105AA000001AB7EE002AF7EE002AB7EE003AF7EE3A
:105AB000003AB7EE004AF7EE004AB7EE005AF7EEAA
:105AC000005AB7EE006AF7EE006AB7EE007AF7EE1A
:105AD000007A8EF3008C10B4F1EE10CA4FF66074A9
:105AE000C0F6FF740CEA040CE1EE10CA10BCF446D8
:105AF000744700F083F80128C4D1204600F07EF8F6
:105B00000128BFD02846FCF73BFA014628B13C22C9
:105B1000204600F0BBF80020B6E76FF00D00B3E7B9
:105B20000020FBF7DDBD0021012000F032B843B2B8
:105B3000C9B9002B15DB01215B099B0003F1604310
:105B400003F56143D3F8802200F01F00814022EA70
:105B50000102C3F88022D3F88012C14001F0010194
:105B6000C9B208467047002B0DDB01225B099B0080
:105B700003F1604303F56143D3F8801200F01F0086
:105B800082400A43E5E70021EBE7836E83F30B884D
:105B9000704700F037B90146006800F033B908B526
:105BA000FCF788FCBDE80840FCF722BE7FB50B6817
:105BB0004D689DF808200E890093498923F01F0342
:105BC000013D66F304022B4461F3471223F01F03E7
:105BD0000F288DF80820039304D86946FCF7A8FE27
:105BE00004B070BD6FF01500FAE740E800F313F45D
:105BF000803FD8B208BF6FF01500704740E800F052
:105C0000C0F3805070470023C25C0AB91846704741
:105C10000133F9E70023C25C0AB18B4201D1184677
:105C200070470133F7E70138013910F8013F11F8E7
:105C3000012F934201D1002BF7D1981A704710B56C
:105C40005AB10139841810F8012B11F8013FA04214
:105C500001D09A42F7D0D01A10BD1046FCE7431A83
:105C6000934210B500EB020308D3024601399A4271
:105C70000BD011F8014F02F8014BF8E70A4412F873
:105C8000014D8A4203F8014DF9D110BDF0B581EA0A
:105C90000004A50703460BD0013B0A4491421AD1E8
:105CA000F0BD002AFCD011F8014B013A03F8014B7A
:105CB0009C07F6D19508AC001E1F0F19B94205D1FB
:105CC0006FF00306234406FB0522E5E751F804CBF9
:105CD00046F804CFF2E711F8014B03F8014FDDE776
:105CE000034670B5C9B29C0710D141EA012444EAC9
:105CF0000445940803EB8406B3420DD16FF003050D
:105D000005FB04241C44A34209D170BD002AFCD029
:105D100003F8011B013AE6E743F8045BECE703F8FC
:105D2000011BF0E74FF0FF30704743681B68D3F862
:105D30000423D20518D5D3F82021AAB14FF02001B1
:105D4000EFF3118281F31188BFF36F8FD3F8201125
:105D500031B10021C3F82011D3F820110121D960FD
:105D600082F31188BFF36F8F70470A46C36804330C
:105D700093E8030082E803000020704743681B6833
:105D8000D3F88004C3F88004704742681368D3F8DE
:105D9000580138B9927932B9D3F82001003018BFD0
:105DA00001207047012070474368C2681B68D3F820
:105DB000100148B10020527C0A70C3F81001D3F8DA
:105DC000102101221A6070474FF0FF30704708B56C
:105DD0000020FCF71BFD08B5FCF7C6F9FCF770FACC
:105DE000BDE80840FEF79CBD004700F0F6B808B5D6
:105DF0000520FCF7E1FA20B9BDE808400520FCF7D2
:105E0000CBBA08BDF8B506460F464FF02003EFF3B6
:105E1000118583F31188BFF36F8FFEF71FF93946A1
:105E200004463046FFF7D3FF85F31188BFF36F8F29
:105E30002046BDE8F840FCF73DBDFFF7C6BD30B5D4
:105E40000024846141EA020414F00304C0E9023230
:105E500001610CD14461A34203D1C0E900000020DC
:105E600030BD456901340D6041611144F3E76FF0C5
:105E70001500F5E703460020C3E90033C3E902003B
:105E80007047034620B9EFF305820AB9FCF72EBA32
:105E900083F31188BFF36F8F70474FF02003EFF348
:105EA000118083F31188BFF36F8FFFF7EABF10B53E
:105EB000044601468068FDF7A9FD637B23F00203D9
:105EC00063730023A36010BD0368984214BF184693
:105ED0000020704710B54FF02003EFF3118483F3D7
:105EE0001188BFF36F8FFDF7EBFD84F31188BFF3CB
:105EF0006F8F10BD70B504464FF02003EFF311868D
:105F000083F31188BFF36F8F50F8103CA0F1180590
:105F100013B12846FFF7CBFF14F80B3C284623F0BB
:105F2000140304F80B3CFDF7CBFD86F31188BFF397
:105F30006F8F70BD38B504460D46FDF741FF637B9A
:105F400043F0020363737DB12B68A5609D4212D0BC
:105F50008BB194F90E2093F90E10914205DD5A6829
:105F6000C4E9003214605C6038BD69688B4202D0BD
:105F70001B68002BEFD16B68256063606B681C6049
:105F80006C60F1E738B54FF02003EFF3118283F333
:105F90001188BFF36F8FFFF797FF044682F31188D4
:105FA000BFF36F8F88B14FF02003EFF3118583F3B8
:105FB0001188BFF36F8FFFF77AFF85F31188BFF366
:105FC0006F8F04F1180000F00CF8204638BDEFF395
:105FD0000580003018BF0120704708B1FBF776BB81
:105FE000704710B54FF02002EFF3118482F311884F
:105FF000BFF36F8F03683BB1FEF750F9002084F3C5
:106000001188BFF36F8F10BD6FF01500F7E710B563
:106010004FF02003EFF3118483F31188BFF36F8FE8
:10602000FEF756F984F31188BFF36F8F10BD70B57A
:1060300004460E464FF02003EFF3118583F31188D9
:10604000BFF36F8FFEF744F9012805DDA04203DDA1
:1060500031462046FBF7BAFD85F31188BFF36F8FF9
:1060600070BD08B5FEF75CFA08BD10B400F10C0471
:10607000C0E903445DF8044BFFF724BB7047FFFF02
:10608000ECA3FF7F01000000A51601000000000046
:10609000C5360100000000005D4501000000000061
:1060A000C52A01000000000005180100BC00002006
:1060B0003D300100CC0000200D300100DC0000204C
:1060C0001117010000000000791B0100EC00002006
:1060D000D75D0100FC0000206D30010000000000D1
:1060E00000000000275B010000000000275B0100AA
:1060F00000000000275B010000000000275B01009A
:1061000000000000275B0100A1330100E95D0100F0
:1061100000000000275B010000000000275B010079
:10612000DC0000202B5D0100CC0000202B5D010075
:1061300000000000275B010000000000275B010059
:1061400000000000275B010000000000275B010049
:1061500000000000275B010000000000275B010039
:1061600000000000275B010000000000275B010029
:1061700000000000275B010000000000275B010019
:1061800000000000275B010000000000291B010047
:1061900000000000275B010000000000275B0100F9
:1061A00000000000275B010000000000275B0100E9
:1061B00000000000275B010000000000275B0100D9
:1061C00000000000275B010000000000275B0100C9
:1061D00000000000275B010000000000275B0100B9
:1061E00000000000275B010000000000275B0100A9
:1061F00000000000275B010000000000275B010099
:1062000000000000275B010000000000275B010088
:1062100000000000275B010000000000275B010078
:1062200000000000275B010000000000275B010068
:1062300000000000275B010000000000275B010058
:1062400000000000275B010000000000275B010048
:1062500000000000275B010000000000275B010038
:1062600000000000275B010000000000275B010028
:1062700000000000275B010000000000275B010018
:1062800000000000275B010000000000275B010008
:1062900000000000275B010000000000275B0100F8
:1062A00000000000275B010000000000275B0100E8
:1062B00000000000275B010000000000275B0100D8
:1062C00000000000275B010000000000275B0100C8
:1062D00000000000275B010000000000275B0100B8
:1062E00000000000275B0100FFFFFFFFFFFFFFFF33
:1062F000DEE61E284CBBCE8F025B00001D000000B6
:106300001C0000001A0000001B000000010000003B
:10631000000000000F0000000E000000DEE61E2856
:10632000EAAC45B8025B0000DEE61E284CBBCE8F0F
:10633000025B000000000000000000000000000000
:106340000338FDD8704700003D1901006B5901006A
:1063500093590100000000009F58010099180100A6
:1063600019190100595901005F590100AD170100C9
:106370006517010000000000DB670100420100001A
:10638000E267010005010000EC6701001401000054
:10639000F567010015010000FE67010039010000EA
:1063A0000768010009010000126801000A000000EE
:1063B0001D6801000A010000276801000B010000B0
:1063C000316801000F0100003C680100100100006D
:1063D0004768010011010000526801000E01000031
:1063E0005C680100210100006568010022010000D5
:1063F0006E6801002301000077680100240100009D
:106400008068010018010000886801002A0100006E
:10641000906801003A010000986801002C0100001A
:10642000A06801001C010000A96801001D01000016
:10643000B268010017010000BC68010004010000FF
:10644000CB680100310100000000000000020000E4
:106450000004000000080000001000000000000020
:10646000215B010001220100B9210100712201001C
:10647000752101001C0000200400002014000020F1
:10648000000000000C0000200000002000000000C0
:1064900006000100020000009C64010000000000F2
:1064A0002A69010006000000E0FF0F000000002044
:1064B0003269010021000000E0FF0020A95D010019
:1064C000312E01007D5D0100C52C01006B5D0100D6
:1064D00000800050060001000090005006000100FE
:1064E00088600100C8600100D0600100E060010028
:1064F000E0600100F5FFFFFF436F756C64206E6F75
:1065000074206C6F636B20706F7765722073617697
:1065100065206D7574657800FF8FFFFFFF8FFFFFAB
:10652000FE8FFFFFFE8FFFFFFD8FFFFFFC8FFFFF42
:10653000FC8FFFFF6D757465785F6672656520631B
:10654000616C6C65642077697468204E554C4C20F2
:10655000706172616D6574657200000043616E2741
:106560007420696E697469616C697A65206D7574EF
:1065700065782C20776173204E554C4C0D0A000035
:106580004661696C20746F20616371756972652062
:106590006D757465780A00004661696C20746F201F
:1065A00072656C65617365206D757465780A0000AD
:1065B0004661696C20746F20696E637265617365F2
:1065C00020504D20636F756E7465720A00000000E4
:1065D0004661696C20746F206465637265617365E0
:1065E00020504D20636F756E7465720A00000000C4
:1065F000286E696C29004661696C656420746F209F
:106600007265626F6F743A207370696E6E696E673F
:1066100020656E646C6573736C792E2E2E0A00559E
:106620004152545F30007379735F636C6F636B002A
:106630005365637572650909004E6F6E2D5365636E
:10664000757265090025303275202530327520308D
:1066500078253035782030782530357820090025A8
:1066600063004E6F6E2D53656375726500466C61F5
:10667000736820726567696F6E730909446F6D6195
:10668000696E09095065726D697373696F6E730A7B
:10669000004E6F6E2D7365637572652063616C6C5F
:1066A00061626C6520726567696F6E203020706C66
:1066B0006163656420696E20666C61736820726531
:1066C00067696F6E20256420776974682073697A22
:1066D000652025642E0A00436F756C64206E6F740C
:1066E00020696E697469616C697A65207365637588
:1066F00072652073657276696365732028657272AE
:10670000202564292E0A005352414D207265676985
:106710006F6E0909446F6D61696E09095065726D8C
:10672000697373696F6E730A00506572697068658A
:1067300072616C0909446F6D61696E090953746176
:106740007475730A002530327520252D323173257A
:10675000730009534B49500A00094552524F520ADF
:1067600000094F4B0A0053504D3A204E5320696D9B
:1067700061676520617420307825780A0053504D98
:106780003A204E53204D53502061742030782578A4
:106790000A0053504D3A204E5320726573657420A1
:1067A000766563746F7220617420307825780A00F2
:1067B00053504D3A207072657061726520746F207D
:1067C0006A756D7020746F204E6F6E2D5365637502
:1067D000726520696D6167652E0A004E52465F50F2
:1067E00030004E52465F434C4F434B004E52465F83
:1067F00052544330004E52465F52544331004E5281
:10680000465F4E564D43004E52465F5541525445E9
:1068100031004E52465F554152544532004E524669
:106820005F5457494D32004E52465F5350494D33E5
:10683000004E52465F54494D455230004E52465F1D
:1068400054494D455231004E52465F54494D4552D0
:1068500032004E52465F5341414443004E52465F20
:1068600050574D30004E52465F50574D31004E52FA
:10687000465F50574D32004E52465F50574D3300E1
:106880004E52465F574454004E52465F49504300B3
:106890004E52465F564D43004E52465F465055009D
:1068A0004E52465F45475531004E52465F4547556B
:1068B00032004E52465F4450504943004E52465FAC
:1068C000524547554C41544F5253004E52465F4734
:1068D00050494F544531006D757465785F696E6934
:1068E000742063616C6C65642077697468204E5510
:1068F0004C4C20706172616D6574657200436F75F8
:106900006C64206E6F7420616C6C6F6361746520C1
:106910006D75746578206265666F726520696E6951
:106920007469616C697A696E6700464C4153485FCF
:1069300030005352414D5F3000554152545F310099
:106940004552524F523A2043616E6E6F7420667505
:106950006C66696C6C204558545F415049207265E3
:1069600071756573742E0D0A005741524E494E479A
:106970003A204F7074696F6E616C204558545F41C6
:1069800050492072657175657374206E6F7420664E
:10699000756C66696C6C65642E0D0A0048575F4320
:1069A000433358585F30006D61696E0076322E3483
:1069B0002E39392D6E637331002A2A2A20426F6FD7
:1069C00074696E67205A6570687972204F5320622F
:1069D00075696C64202573202573202A2A2A0A00F1
:1069E00000000100275401001001002001000000F8
:1069F00024010020010000003801002001000000F7
:106A00004C01002001000000255D01000000000095
:106A100000C20100000103000000000000000000AF
:106A20000000000000C2010000010300000000009F
:106A3000000000000090D00354000020540000200B
:106A400094000020A000002098000020900000206A
:106A50006400002000000000594901007008002077
:106A600001000000094A0100E5490100294A01002E
:106A7000C5490100B400002078000020AC000020CF
:106A800000000000A40000207408002001000000A5
:106A900078080020010000007C08002001000000B0
:106AA000E66701005C630100486301007C0200208E
:106AB00039690100D8640100BC6401003C00002079
:106AC0001F660100D0640100BC64010028000020A2
:106AD0002666010000000000000000000000000029
:106AE0009C690100000000000000000000000000A0
:106AF0000000000010010020100100200000000034
:106B0000000000000F0000002401002024010020EC
:106B100000000000000000000F000000380100200D
:106B20003801002000000000000000000F000000FD
:106B30004C0100204C01002000000000000000007B
:106B40000F000000FFFFFFFFFFFFFFFFFFFFFFFF42
:106B5000FFFFFFFFFFFFFFFFFFFFFFFFFFFFFFFF45
:106B60000000000000000000000000000000000025
:106B70000000000000000000000000000000000015
:106B80000000000000000000000000000000000005
:107FE0007FE97FE9FDF74ABD7FE97FE9FDF7F9BC4D
:107FF0007FE97FE9FAF74EB87FE97FE9F9F7E4BF57
:10800000FFFFFFFFFFFFFFFFFFFFFFFFFFFFFFFF80
:10801000FFFFFFFFFFFFFFFFFFFFFFFFFFFFFFFF70
:10802000FFFFFFFFFFFFFFFFFFFFFFFFFFFFFFFF60
:10803000FFFFFFFFFFFFFFFFFFFFFFFFFFFFFFFF50
:10C20000A0550220556D02003FF20300B56D0200FB
:10C21000B56D0200B56D0200B56D0200B56D02008E
:10C22000000000000000000000000000E9690200BA
:10C23000B56D020000000000356902004165020092
:10C24000156D0200156D0200156D0200156D0200DE
:10C25000156D0200156D0200156D0200156D0200CE
:10C26000156D0200156D0200156D0200156D0200BE
:10C27000156D0200156D0200156D0200156D0200AE
:10C28000156D0200156D0200156D0200156D02009E
:10C29000156D0200156D0200156D0200156D02008E
:10C2A000156D0200156D0200156D0200156D02007E
:10C2B00051970200DB060400156D0200156D0200A7
:10C2C000156D0200156D0200156D0200156D02005E
:10C2D000156D0200156D0200156D0200156D02004E
:10C2E000156D0200156D0200156D0200156D02003E
:10C2F000156D0200156D0200156D0200156D02002E
:10C30000156D0200156D0200156D0200156D02001D
:10C31000156D0200156D0200156D0200156D02000D
:10C32000156D0200156D0200156D0200156D0200FD
:10C33000156D0200156D0200156D0200156D0200ED
:10C34000156D020000000000000000000000000069
:10C3500000000000000000000000000000000000DD
:10C3600000000000000000000000000000000000CD
:10C3700000000000000000000000000000000000BD
:10C3800000000000000000000000000000000000AD
:10C39000000000000000000000000000000000009D
:10C3A000000000000000000000000000000000008D
:10C3B000000000000000000000000000000000007D
:10C3C000000000000000000000000000000000006D
:10C3D000000000000000000000000000000000005D
:10C3E000000000000000000000000000000000004D
:10C3F000000000000000000000000000000000003D
:10C40000DEE61E284CBBCE8F025B00003C00000025
:10C41000D82903000100000000C2010000C2010091
:10C42000FFFF02910000000000000000000000007B
:10C43000000000000000000000000000FFFFFFFF00
:10C4400081F0004102E000BF83F0004330B54FEAC5
:10C4500041044FEA430594EA050F08BF90EA020F32
:10C460001FBF54EA000C55EA020C7FEA645C7FEAC5
:10C47000655C00F0E2804FEA5454D4EB5555B8BFE8
:10C480006D420CDD2C4480EA020281EA030382EA59
:10C49000000083EA010180EA020281EA0303362DEB
:10C4A00088BF30BD11F0004F4FEA01314FF4801CBE
:10C4B0004CEA113102D0404261EB410113F0004FD0
:10C4C0004FEA03334CEA133302D0524263EB430387
:10C4D00094EA050F00F0A780A4F10104D5F1200E25
:10C4E0000DDB02FA0EFC22FA05F2801841F1000180
:10C4F00003FA0EF2801843FA05F359410EE0A5F154
:10C5000020050EF1200E012A03FA0EFC28BF4CF084
:10C51000020C43FA05F3C01851EBE37101F000453A
:10C5200007D54FF0000EDCF1000C7EEB00006EEB47
:10C530000101B1F5801F1BD3B1F5001F0CD34908D1
:10C540005FEA30004FEA3C0C04F101044FEA445228
:10C5500012F5800F80F09A80BCF1004F08BF5FEAAF
:10C56000500C50F1000041EB045141EA050130BD8F
:10C570005FEA4C0C404141EB010111F4801FA4F132
:10C580000104E9D191F0000F04BF01460020B1FA87
:10C5900081F308BF2033A3F10B03B3F120020CDABF
:10C5A0000C3208DD02F1140CC2F10C0201FA0CF09D
:10C5B00021FA02F10CE002F11402D8BFC2F1200C02
:10C5C00001FA02F120FA0CFCDCBF41EA0C019040B8
:10C5D000E41AA2BF01EB0451294330BD6FEA040401
:10C5E0001F3C1CDA0C340EDC04F11404C4F12002EC
:10C5F00020FA04F001FA02F340EA030021FA04F3FE
:10C6000045EA030130BDC4F10C04C4F1200220FA54
:10C6100002F001FA04F340EA0300294630BD21FA92
:10C6200004F0294630BD94F0000F83F4801306BF58
:10C6300081F480110134013D4EE77FEA645C18BF4C
:10C640007FEA655C29D094EA050F08BF90EA020FE3
:10C6500005D054EA000C04BF1946104630BD91EADB
:10C66000030F1EBF0021002030BD5FEA545C05D1DE
:10C670004000494128BF41F0004130BD14F580041D
:10C680003CBF01F5801130BD01F0004545F0FE4191
:10C6900041F470014FF0000030BD7FEA645C1ABFC6
:10C6A000194610467FEA655C1CBF0B46024650EAFD
:10C6B000013406BF52EA033591EA030F41F4002129
:10C6C00030BD00BF90F0000F04BF0021704730B5AF
:10C6D0004FF4806404F132044FF000054FF0000184
:10C6E00050E700BF90F0000F04BF0021704730B545
:10C6F0004FF4806404F1320410F0004548BF40421A
:10C700004FF000013EE700BF42004FEAE2014FEA6E
:10C7100031014FEA02701FBF12F07F4393F07F4F49
:10C7200081F06051704732F07F4208BF704793F04C
:10C730007F4F04BF41F40021704730B54FF460745F
:10C7400001F0004521F000411CE700BF50EA010262
:10C7500008BF704730B54FF000050AE050EA01020B
:10C7600008BF704730B511F0004502D5404261EB7B
:10C7700041014FF4806404F132045FEA915C3FF4BC
:10C78000D8AE4FF003025FEADC0C18BF03325FEA59
:10C79000DC0C18BF033202EBDC02C2F1200300FA0A
:10C7A00003FC20FA02F001FA03FE40EA0E0021FA2F
:10C7B00002F11444BDE600BF70B54FF0FF0C4CF41D
:10C7C000E06C1CEA11541DBF1CEA135594EA0C0FCF
:10C7D00095EA0C0F00F0DEF82C4481EA030621EA0A
:10C7E0004C5123EA4C5350EA013518BF52EA033545
:10C7F00041F4801143F4801338D0A0FB02CE4FF0F7
:10C800000005E1FB02E506F00042E0FB03E54FF026
:10C810000006E1FB03569CF0000F18BF4EF0010E1E
:10C82000A4F1FF04B6F5007F64F5407404D25FEA1A
:10C830004E0E6D4146EB060642EAC62141EA5551CD
:10C840004FEAC52040EA5E504FEACE2EB4F1FD0C0F
:10C8500088BFBCF5E06F1ED8BEF1004F08BF5FEA8D
:10C86000500E50F1000041EB045170BD06F000463F
:10C8700046EA010140EA020081EA0301B4EB5C04EC
:10C88000C2BFD4EB0C0541EA045170BD41F48011E4
:10C890004FF0000E013C00F3AB8014F1360FDEBF09
:10C8A000002001F0004170BDC4F10004203C35DAE5
:10C8B0000C341BDC04F11404C4F1200500FA05F368
:10C8C00020FA04F001FA05F240EA020001F0004209
:10C8D00021F0004110EBD37021FA04F642EB06017F
:10C8E0005EEA430E08BF20EAD37070BDC4F10C04A9
:10C8F000C4F1200500FA04F320FA05F001FA04F26D
:10C9000040EA020001F0004110EBD37041F1000158
:10C910005EEA430E08BF20EAD37070BDC4F1200563
:10C9200000FA05F24EEA020E20FA04F301FA05F2CB
:10C9300043EA020321FA04F001F0004121FA04F273
:10C9400020EA020000EBD3705EEA430E08BF20EA43
:10C95000D37070BD94F0000F0FD101F0004640007D
:10C9600041EB010111F4801F08BF013CF7D041EAFF
:10C97000060195F0000F18BF704703F00046520003
:10C9800043EB030313F4801F08BF013DF7D043EAD4
:10C990000603704794EA0C0F0CEA135518BF95EA8A
:10C9A0000C0F0CD050EA410618BF52EA4306D1D111
:10C9B00081EA030101F000414FF0000070BD50EA30
:10C9C000410606BF1046194652EA430619D094EABA
:10C9D0000C0F02D150EA013613D195EA0C0F05D1A4
:10C9E00052EA03361CBF104619460AD181EA0301F8
:10C9F00001F0004141F0FE4141F470014FF00000B0
:10CA000070BD41F0FE4141F4780170BD70B54FF04A
:10CA1000FF0C4CF4E06C1CEA11541DBF1CEA1355CA
:10CA200094EA0C0F95EA0C0F00F0A7F8A4EB0504AC
:10CA300081EA030E52EA03354FEA013100F08880A3
:10CA40004FEA03334FF0805545EA131343EA12636C
:10CA50004FEA022245EA111545EA10654FEA002621
:10CA60000EF000419D4208BF964244F1FD0404F5DA
:10CA7000407402D25B084FEA3202B61A65EB030536
:10CA80005B084FEA32024FF480104FF4002CB6EBF3
:10CA9000020E75EB030E22BFB61A754640EA0C0073
:10CAA0005B084FEA3202B6EB020E75EB030E22BFB3
:10CAB000B61A754640EA5C005B084FEA3202B6EBF4
:10CAC000020E75EB030E22BFB61A754640EA9C00B3
:10CAD0005B084FEA3202B6EB020E75EB030E22BF83
:10CAE000B61A754640EADC0055EA060E18D04FEA41
:10CAF000051545EA16754FEA06164FEAC30343EAE1
:10CB000052734FEAC2025FEA1C1CC0D111F4801FAD
:10CB10000BD141EA00014FF000004FF0004CB6E7A6
:10CB200011F4801F04BF01430020B4F1FD0C88BF45
:10CB3000BCF5E06F3FF6AFAEB5EB030C04BFB6EB50
:10CB4000020C5FEA500C50F1000041EB045170BD43
:10CB50000EF0004E4EEA113114EB5C04C2BFD4EB70
:10CB60000C0541EA045170BD41F480114FF0000EF4
:10CB7000013C90E645EA060E8DE60CEA135594EA70
:10CB80000C0F08BF95EA0C0F3FF43BAF94EA0C0F73
:10CB90000AD150EA01347FF434AF95EA0C0F7FF4E8
:10CBA00025AF104619462CE795EA0C0F06D152EA3C
:10CBB00003353FF4FDAE1046194622E750EA410620
:10CBC00018BF52EA43067FF4C5AE50EA41047FF431
:10CBD0000DAF52EA43057FF4EBAE12E74FF0FF3C96
:10CBE00006E000BF4FF0010C02E000BF4FF0010C67
:10CBF0004DF804CD4FEA410C7FEA6C5C4FEA430CE0
:10CC000018BF7FEA6C5C1BD001B050EA410C0CBF2E
:10CC100052EA430C91EA030F02BF90EA020F002090
:10CC2000704710F1000F91EA030F58BF994208BFF7
:10CC300090422CBFD8176FEAE37040F001007047B4
:10CC40004FEA410C7FEA6C5C02D150EA013C07D10B
:10CC50004FEA430C7FEA6C5CD6D152EA033CD3D056
:10CC60005DF8040B704700BF8446104662468C4650
:10CC70001946634600E000BF01B5FFF7B7FF002883
:10CC800048BF10F1000F01BD4DF808EDFFF7F4FFAC
:10CC90000CBF012000205DF808FB00BF4DF808ED37
:10CCA000FFF7EAFF34BF012000205DF808FB00BF5A
:10CCB0004DF808EDFFF7E0FF94BF012000205DF87C
:10CCC00008FB00BF4DF808EDFFF7CEFF94BF012031
:10CCD00000205DF808FB00BF4DF808EDFFF7C4FF2A
:10CCE00034BF012000205DF808FB00BF4FEA41027D
:10CCF00012F5001215D211D56FF47873B3EB6252AE
:10CD000012D94FEAC12343F0004343EA505311F0D4
:10CD1000004F23FA02F018BF404270474FF0000066
:10CD2000704750EA013005D111F0004008BF6FF0A4
:10CD3000004070474FF00000704700BF4A0011D21A
:10CD400012F5001211D20DD56FF47873B3EB625265
:10CD50000ED44FEAC12343F0004343EA505323FA71
:10CD600002F070474FF00000704750EA013002D1E6
:10CD70004FF0FF3070474FF0000070474FEA41021C
:10CD8000B2F1E04324BFB3F5001CDCF1FE5C0DD929
:10CD900001F0004C4FEAC0024CEA5070B2F1004F73
:10CDA00040EB830008BF20F00100704711F0804F76
:10CDB00021D113F13872BCBF01F00040704741F43B
:10CDC00080114FEA5252C2F11802C2F1200C10FA3F
:10CDD0000CF320FA02F018BF40F001004FEAC12323
:10CDE0004FEAD32303FA0CFC40EA0C0023FA02F3C7
:10CDF0004FEA4303CCE77FEA625307D150EA01339D
:10CE00001EBF4FF0FE4040F44000704701F000406C
:10CE100040F0FE4040F40000704700BF7BB972B99B
:10CE20000029BEBF00204FF0004106E008BF0028E7
:10CE30001CBF6FF000414FF0FF3000F0F1B9ADF1D1
:10CE4000080C6DE904CE002909DB002B1ADB00F089
:10CE500083F8DDF804E0DDE9022304B070474042C6
:10CE600061EB4101002B1BDB00F076F8DDF804E0FC
:10CE7000DDE9022304B0404261EB4101524263EB21
:10CE800043037047524263EB430300F065F8DDF85B
:10CE900004E0DDE9022304B0404261EB4101704748
:10CEA000524263EB430300F057F8DDF804E0DDE99C
:10CEB000022304B0524263EB4303704753B94AB9AB
:10CEC000002908BF00281CBF4FF0FF314FF0FF3092
:10CED00000F0A6B9ADF1080C6DE904CE00F03CF805
:10CEE000DDF804E0DDE9022304B0704738B5002224
:10CEF000002304460D46FFF7D1FE28B920462946F7
:10CF0000BDE8384000F00AB8204605F1004100F0C5
:10CF100005F8404261EB410138BD00BFD0B50022A9
:10CF20000B4B06460F46FFF747FCFFF707FF04468B
:10CF3000FFF7C8FB0022074BFFF73EFC02460B46FB
:10CF400030463946FFF780FAFFF7F8FE2146D0BD9C
:10CF50000000F03D0000F0412DE9F04F099E04462D
:10CF60008946002B40F083808A42154645D9B2FAA3
:10CF700082F24AB1C2F1200701FA02F395409440CF
:10CF800020FA07F747EA03094FEA154E230C1FFA68
:10CF900085F8B9FBFEFC0EFB1C990CFB08F143EA7B
:10CFA000094399420AD9EB182CBF0120002099426D
:10CFB00002D9002800F01D810CF1FF3C591AA3B2E0
:10CFC000B1FBFEF00EFB101100FB08F843EA014430
:10CFD000A04505D92C1902D2A04500F20E810138D6
:10CFE000A4EB080440EA0C4000271EB1D440002303
:10CFF000C6E900433946BDE8F08F002A51D0B2FAA5
:10D0000082F2002A40F0AF80491B4FEA154E1FFA0A
:10D0100085F80127230CB1FBFEFC0EFB1C1108FB5D
:10D020000CF043EA014398420AD9EB182CBF0121C6
:10D030000021984202D9002900F0D7800CF1FF3C72
:10D04000191AA3B2B1FBFEF00EFB101108FB00F899
:10D0500043EA0144A04505D92C1902D2A04500F2AB
:10D06000C1800138A4EB080440EA0C40BDE78B42C4
:10D0700008D9002E74D00027C6E900013846394689
:10D08000BDE8F08FB3FA83F767B98B42C0F0A48094
:10D09000824240F2A1803846002EABD0C6E900495A
:10D0A000A8E7FFDEC7F12005BB4002FA07FC01FA42
:10D0B00007F4EA4020FA05F8E94000FA07FE1A43AF
:10D0C00048EA04044FEA1248200C1FFA82F9B1FB27
:10D0D000F8FA08FB1A110AFB09FB40EA01418B45EB
:10D0E0000AD951182CBF012300238B4502D9002BEC
:10D0F00000F088800AF1FF3AA1EB0B01A4B2B1FB6A
:10D10000F8F008FB101100FB09F944EA01418945D8
:10D1100004D9511801D289457BD8013840EA0A4028
:10D12000A1EB0901A0FB0C89494544464B4602D3BB
:10D1300006D1C64504D20138B8EB0C0469EB0203F2
:10D14000002E5DD0BEEB040261EB030101FA05F590
:10D1500022FA07F3F94000271D43C6E9005149E7C9
:10D160003746304646E7C2F12000954001FA02F703
:10D1700021FA00F34FEA154E24FA00F11FFA85F860
:10D1800094403943B3FBFEF00F0C0EFB103300FB51
:10D1900008FC47EA03439C4507D9EB182CBF01273D
:10D1A00000279C4500D98FB30138A3EB0C0389B24B
:10D1B000B3FBFEF70EFB173307FB08FC41EA034104
:10D1C0008C4504D9691801D28C4525D8013FA1EBC3
:10D1D0000C0147EA00471DE7841A61EB03030120B5
:10D1E000994659E702382C443CE7ACF1020C2B4439
:10D1F00026E7ACF1020C2B44E0E602382C44EFE6C3
:10D200003746F7E6AAF1020A114475E702382B44C3
:10D21000CBE70238114481E7023F2944D7E700BF3A
:10D22000704700BF4FEA410C7FEA6C5C02D150EAC4
:10D23000013C0AD14FEA430C7FEA6C5C02D152EA0E
:10D24000033C02D14FF0000070474FF001007047DF
:10D2500010F8012B11F8013B012A28BF9A42F7D0A0
:10D26000D01A7047034613F8012B002AFBD1181A75
:10D2700001387047000000002DE9F041284B294D8E
:10D28000294CA846E41AD5E900231343C4F3C90482
:10D2900018D020F0E3FDD5E90032C61A61EB020791
:10D2A0001DA3D3E90023B242BB410BDB4FF00000CA
:10D2B00002231E4963F3070064F38F10BDE8F041B9
:10D2C00021F020B903234FF0000063F3070064F35B
:10D2D0008F10174921F016F9164A002307CA09F0E2
:10D2E000C1FA024658B101214FF0000061F3070076
:10D2F00064F38F101049BDE8F04121F003B920F02C
:10D30000ADFD0323C8E900014FF0000063F30700FF
:10D3100064F38F100949D1E77FEE3600000000006A
:10D320000C450400205D01201C450400655E0400DE
:10D33000915E0400208B0120A75E0400CF5E0400F4
:10D3400070B596B025F0FFFC4FF47A74A0FB04563C
:10D3500004FB0166EA0B524C42EA4642F30BCDE96C
:10D360001423206883680321DB689847014678B15D
:10D3700001234FF000004B4A63F307004A4B4B492F
:10D380009B1ADB0863F38F1021F0BCF816B070BD58
:10D3900006AA206820F07FFD60B101234FF0000055
:10D3A000404A63F30700404B41499B1ADB0863F393
:10D3B0008F10E9E708AA0121206820F06CFD002801
:10D3C000EBD10AAA0221206820F065FD0028E4D1F3
:10D3D0000798FFF787F930A3D3E90023FFF716FB7F
:10D3E000044606980D46FFF77DF902460B46204697
:10D3F0002946FFF72BF8CDE90E010998FFF772F9DE
:10D4000025A3D3E90023FFF701FB044608980D4646
:10D41000FFF768F902460B4620462946FFF716F843
:10D42000CDE910010B98FFF75DF91BA3D3E90023A9
:10D43000FFF7ECFA04460A980D46FFF753F9024647
:10D440000B4620462946FFF701F80022194B0446F7
:10D450000D46FFF737FC90B10123CDE912456C462C
:10D460008DF83030144B10AD1E680FCD0FC495E809
:10D47000030084E803000CAB0FCBB04786E7002223
:10D480000E4B20462946FFF713FC08B10223E4E7C0
:10D490000323E2E7AFF300800000000080842E4108
:10D4A000888B01200C450400D4450400046104006D
:10D4B0001F610400000014408C8B0120000014C088
:10D4C0002DE9F04F8DB06A4B00AF1A68C7F804D051
:10D4D0003B60002A5CD04FF0000B664B664A674CFD
:10D4E0009B1AC3F3C903664E3B6107F11805236815
:10D4F000186A198B8368DB6898478046A8B1BB8A95
:10D5000023F03F0242F0010262F307033A699BB243
:10D5100062F38F13BB822368D86921F006F8434673
:10D5200002465849B88A20F0EDFF2368186A198B23
:10D5300083682A461B6998472368814660B32AF0AE
:10D540003F0242F0010262F3070A3A69D86962F3C6
:10D550008F1A20F0EAFF4B4602464A49504620F017
:10D56000D1FF0BF1010BBBF1030F04F1040405F132
:10D570000805BCD1444B1B6803B19847434B1B784B
:10D58000002B6ED13B68186805F0E8F9D7F804D095
:10D590003437BD46BDE8F08F03F124084FF0200377
:10D5A000EFF3118283F31188BFF36F8F40469146EA
:10D5B0001DF054FA68B97C2332463549354820F0CD
:10D5C000E1FC4146344820F0DDFC7C21304620F06F
:10D5D00088FF40461DF060FA6868FFF783F822A3D1
:10D5E000D3E90023FFF712FAC7E902012868FFF721
:10D5F00079F802460B46D7E90201FEF727FFD4F877
:10D600000080C8E9020125F09EFB4FF47A7CA0FB64
:10D610000C23C7E90223FB680CFB0133FB60BB68EA
:10D62000DA0BFB6842EA4342DB0BC8E904232368B8
:10D6300003F1240840461DF01FFA68B9A7233246BB
:10D640001649144820F09EFC4146154820F09AFCEB
:10D65000A721304620F045FF89F31188BFF36F8F73
:10D660007FE7142090E700BF0000000080842E4177
:10D67000F0540120844504000C450400C048040017
:10D6800011670400E9660400B08B01200BEB012058
:10D6900037670400695C04004C6704006467040099
:10D6A0007B670400000000002DE9F04305469BB0B5
:10D6B0000F4616460021302202A825F042FC002D1C
:10D6C00000F08780002E00F084801B238DF8083046
:10D6D00025F039FB4FF47A730024A0FB038903FB88
:10D6E00001994FEAD8304FF47A72002340EA49405A
:10D6F0002146FFF7E3FB3C4A0244130A110201F4FE
:10D700007F0103F47F430B4343EA026343F0830347
:10D710002A610C93E8683022CDE90044234602A92F
:10D7200021F087FA00280FDB214630220EA825F0D1
:10D7300008FCA9683A46284607F074FCA04206DABD
:10D7400021F0CCFD006840421BB0BDE8F08337D02B
:10D75000E8683022CDE9004423460EA921F09CFA66
:10D760000028EDDB30282ED1149B2A691BBA9A427F
:10D7700002D06FF01500E7E79DF8383003F007039B
:10D78000042BF6D19DF8393003B3189B199A1BBAB4
:10D7900012BA53EA0201ECD0002BB2600CDA134A41
:10D7A0009342E6D90CA1D1E90001C41841F100056A
:10D7B000C6E900450020C7E709A1D1E90001F4E767
:10D7C0006FF07300C0E76FF07900BDE76FF00F00F6
:10D7D000BAE76FF00D00B7E78081557CFFFFFFFFD0
:10D7E0008081557C00000000807EAA837F7EAA8312
:10D7F0002DE9F043054693B00C4609B9002024E01A
:10D8000008680028FAD08B686268191D91420BD80D
:10D810000422B149184425F076FD28B90423EB60B1
:10D82000A3680433A36074E0A3686268591D914241
:10D830000ED820680522A949184425F064FD38B99E
:10D840000120A368E8600533A36013B0BDE8F0834E
:10D85000A3686268191D91420DD820680422A0496E
:10D86000184425F050FD30B902230120EB60A36875
:10D8700068610433E8E7D4E90172BA42BED2206895
:10D88000835C222B04D1214628460BF0BBF9DCE750
:10D890002D2B03D0A3F13006092E50D8002301937D
:10D8A0000028ABD0BF1A02AE9F4202EB03010ED09C
:10D8B000415C39292FD8302905D22D2903D02E29B2
:10D8C00001D02B2903D1F15401333F2BECD112AA03
:10D8D0001344002201A9304603F8402C1EF0E6FF55
:10D8E000019F59EC108BB74288D079A3D3E900236C
:10D8F00085ED060B10EE100A4946FFF7E3F970B10B
:10D900006FF000436B610823BE1BA768EB603E44C9
:10D91000A660012099E74529D5D06529D2E70022E4
:10D92000704B40464946FFF7C3F910B14FF0004332
:10D93000E8E740464946FFF7D9F96861E3E75B2B22
:10D9400053D1E368B3F57A7FBFF458AF0133E36096
:10D95000835C5B2B7FF452AF0132A260204622F041
:10D9600088FDD4E90123934262D22268D25C5D2A09
:10D9700009D10026E368013BE3602023C5E9026387
:10D98000A36801334EE74FF000084646013BA36011
:10D99000206922F0A8FD074600B3EEB1C8F80000E8
:10D9A000C0F80480A36820460133A36022F061FD23
:10D9B00021463846FFF71CFF98B1204622F059FD5A
:10D9C000D4E9012393420CD22268B846D35C2C2BB5
:10D9D000DED05D2B05D1CDE70646E3E7002E3FF410
:10D9E0000DAF30460BF018FD08E77B2B7FF406AF38
:10D9F000E368B3F57A7FBFF401AF0133E360835C82
:10DA00007B2B7FF4FBAE0132A260204622F031FD79
:10DA1000D4E9012393420BD22268D25C7D2A0AD139
:10DA20000027E368013BE3604023C5E90273A7E7F1
:10DA3000013BA360E2E64FF000084746C146013BC8
:10DA4000A360206922F04FFD0646002839D0B7B305
:10DA5000C8F80000C0F80480A36820460133A36022
:10DA600022F007FD214630460BF0CCF860B320468B
:10DA700022F0FFFC3369C6F810903362D4E9012329
:10DA8000934221D22268D25C3A2A1DD10133A3608D
:10DA9000204622F0EEFC21463046FFF7A9FE98B161
:10DAA000204622F0E6FCD4E9012393420CD22268FE
:10DAB000B046D35C2C2BC4D07D2B05D1B1E70746F3
:10DAC000CAE7002F3FF49AAE38468BE7AFF30080E9
:10DAD0000000C0FFFFFFDF41737D04008A7D04006A
:10DAE000907D04000000E0C1174BD0B5186857ECDA
:10DAF000106B22F0F8FC044670B10823C0E90667F9
:10DB0000C36039460EA3D3E900233046FFF7DAF8A5
:10DB100020B16FF0004363612046D0BD00220B4B63
:10DB200030463946FFF7C4F810B14FF00043F2E732
:10DB300030463946FFF7DAF86061EDE7AFF3008071
:10DB40000000C0FFFFFFDF41AC5501200000E0C135
:10DB50002DE9F0412DED028B0E468CB091B90123D9
:10DB60004FF00000BC4A63F30700BC4BBC499B1A52
:10DB7000DB0863F38F1020F0C5FC0CB0BDEC028B0A
:10DB8000BDE8F0810024B74F57F8045B2846FFF743
:10DB900069FB31460246284625F0B5FB0546A0BB89
:10DBA000E4B2012C00F02F81022C00F0C7814FF06D
:10DBB00009080A2107A8CDF8088023F020F80446B8
:10DBC00038B301234FF00000A34A63F30700A34BCF
:10DBD000A5499B1ADB0863F38F10224620F092FCC4
:10DBE00001234FF000059C4A63F307059B4B304629
:10DBF0009B1ADB0863F38F1520F097FC224603463F
:10DC00009A49284620F07EFCB7E70134032CBBD1AB
:10DC1000B3E7014607AA304622F0EEFF044600288B
:10DC200062D001234FF000008B4A63F307008B4B57
:10DC30008F499B1A2246DB0863F38F1020F062FCA9
:10DC400007A822F0EFFF002CCAD105F0FB07012F37
:10DC500002D188481CF0C0FC874C2368002B8CD074
:10DC6000864A1178A94207D0157000228DF82850F5
:10DC70008DF8242009A89847814E03AD082231462B
:10DC8000284625F030F960B195E8030004238DF8AB
:10DC900024300CAB03E9030086E80300236809A8DD
:10DCA0009847012F7FF469AF764E05AD08223146C3
:10DCB000284625F018F958B195E803000CAB8DF80B
:10DCC000247086E8030003E90300236809A8984745
:10DCD0000023694A1268002A3FF44FAF002B3FF43B
:10DCE0004CAF09A8904748E701AA012107A823F0F3
:10DCF00049F8044668B101234FF00000564A63F327
:10DD00000700564B60499B1ADB0863F38F102246CD
:10DD100094E79DF804505A2D6BD007A823F070F8B3
:10DD2000032866D902AB09AA022107A823F041F80B
